:020000040800F2
:104000000050002019F3000885C4000889C4000886
:104010008DC4000891C4000895C400080000000089
:104020000000000000000000000000009DC4000827
:1040300099C4000800000000A1C40008E99200082B
:10404000A5C40008A9C40008ADC40008B1C4000894
:10405000B5C40008B9C40008BDC40008C1C4000844
:10406000C5C40008C9C40008CDC400080000000091
:104070000000000000000000000000000000000040
:104080000000000000000000EDC40008F1C40008BA
:1040900001C5000811C5000821C5000831C5000888
:1040A00035C5000839C500083DC5000841C50008F0
:1040B00045C5000849C500084DC5000851C50008A0
:1040C00055C5000859C500085DC5000861C5000850
:1040D00065C5000869C50008ED89000871C50008BC
:1040E0009949000879C500087DC500080000000056
:1040F00000000000000000000000000000000000C0
:0C41000000000000000000005FF800005C
:1041100030BF704720BF704740BF7047BFF36F8FFD
:104120007047BFF34F8F7047BFF35F8F704701DF5A
:104130007047EFF31480704780F31488BFF36F8FDC
:104140007047EFF30980704780F309887047EFF3F9
:104150000880704780F30888704772B6704762B66F
:10416000704771B6704761B6704780F31188704729
:10417000EFF31280704740BA704700BA70470000F2
:1041800010B500F033FC0B4C0B490C4A0C4B48B1FA
:104190004FF0010C0B4884F800C00B4C1860146001
:1041A000086006E020700948086009491160094A62
:1041B0001A6010BD200B0020480B00202C0C0020A2
:1041C000BC0B0020618C0008619A0008F58C000887
:1041D000319200087991000837B509F06FFD6A4BFC
:1041E00000254FF480301D7009F088FD09F0ECFEC9
:1041F0000128044627D1102009F04AF8284609F082
:10420000CDFD284609F0DEFD4FF4806009F0D0FDB9
:104210004FF440304FF4E01109F09CFD204609F0C6
:10422000A5FD392009F0BAFE0028FAD0022009F0D5
:1042300017F8022009F0A0FD09F0A8FD0828FBD11D
:10424000514B01221A700420012109F05DFE032365
:104250008DF80630153301A94C488DF807304FF41E
:104260008073ADF8043009F047FA062009F090FE9B
:104270000120014609F048FE454C4FF480414FF0C3
:10428000006009F03DFC4FF4407009F09BFB00F02A
:104290000FFC00F093FDFFF773FF00F0FBF805F053
:1042A0004DF905F0ADF804F0CFFA00F077F820787A
:1042B00004F0FCFBE07804F055FB364B1B7823B987
:1042C00022696079A16804F0AFFD324B1B780BB115
:1042D00005F06EFC06F0E2F900F010FA07F0A4FE1B
:1042E000012000F0B7FB00F04FF901F033FE05F0BC
:1042F00067FC06F019FA284B4FF400425A6105F0AA
:1043000079F8044603F020FC06F01CFA05F092FC54
:1043100005F070F8001B0028B8BF4042B0F57A7F66
:1043200024DD1C4D2B782C4683B100F05FFB68B96F
:10433000287005F0FDFB05F0E3FAFFF721FF144BB1
:104340001A695879996804F06FFD0CE0237853B925
:1043500000F04CFB38B104F02BFD01232370FFF774
:104360000FFF05F025FC05F045F8044600F048F97C
:1043700000F03AF90028C5D006F090F901F0EAFD06
:1043800006F0D2F9BEE700BF1C0C00200008014077
:1043900008000020200B002000100140114B82B0CB
:1043A0001B78E3B1104B04225A6102221A610023E8
:1043B00001E0019B01330193019A0C4B9A42F8D919
:1043C000094B04221A6102225A61002301E0019B79
:1043D00001330193019A054B9A42E3D8F7E702B003
:1043E000704700BF5C0B0020000C01403F0D030034
:1043F00010B1012809D104E0044B4FF400625A6166
:1044000003E0024B4FF480621A617047000C0140D8
:1044100010B1012809D104E0044B4FF400621A6185
:1044200003E0024B4FF480625A617047000C014078
:1044300038B50546002455FA04F2E3B212F0010F34
:10444000184602D0FFF7E4FF01E0FFF7D1FF013487
:10445000082CF0D138BD00BF18B1012806D00020CB
:104460000AE0064BD868C0F3C02005E0034BD868CB
:1044700080F48060C0F38020704700BF000C0140D2
:1044800008B1002003E0024B9868C0F3C0007047F9
:10449000000C014062B6704772B6704718B9024B03
:1044A0004FF400425A6170470010014018B9024BA6
:1044B0004FF400421A6170470010014008B100201B
:1044C00005E0034BD3E90023100A40EA036070477C
:1044D000600B0020F8B50D460446B8B9FFF7DCFFC5
:1044E0000B492A464FEAE273C1E90023D1E900678C
:1044F0003B0243EA16633202C1E90023054B1C600C
:10450000054B1C60054B9C84FFF7C4FFF8BD00BF42
:10451000600B0020680C0020400B002000080040C9
:1045200010B9024B09011960704700BF680B0020E9
:1045300020BB11F0040F10D011F0100F04D0104B5D
:104540009A6842F400420CE00D4B9A6822F4004253
:104550009A60DA6842F4004207E0094B9A6822F454
:1045600000429A60DA6822F4004211F00801DA6031
:10457000044B02D001221A7000E01970704700BF8E
:104580000004014030020020084B4FF400721A6012
:10459000074B10B50024204610211C60FFF7C0FF18
:1045A00020462146FFF7C4FF10BD00BF500B00207E
:1045B0004C0B002010B9024B09011960704700BF75
:1045C0000400002008B9014B5970704730020020E8
:1045D000044B98780138C0B201288CBF002001201C
:1045E000704700BF30020020044B9878012801D0AA
:1045F000002001E002229A70704700BF30020020C4
:10460000082008B504F014FF592804D9064B9A78FD
:104610004AB9013206E0082004F00AFF542802D803
:10462000014B00229A7008BD3002002008B5032813
:1046300003D8DFE800F0040D1217002016E0002078
:1046400004F0F6FEB0F5006F94BF002001200DE0ED
:10465000074B9868C0F3C01008E0054B9868C0F39A
:10466000801003E0034B9868C0F3C03008BD00BF62
:10467000000C01400008014038B500242546E0B296
:10468000FFF7D4FF20B10123A34043EA0505EDB2B3
:104690000134082CF3D1284638BD00BF38B50D4B86
:1046A0000D4C9A6812F0200201D0606810E0FF21E2
:1046B000032000F00DFBFF2105460122032000F03E
:1046C00007FBA36840EA052003EA9000181A60601F
:1046D00038BD00BF000C01403002002008B5FFF7D4
:1046E000DDFF052801D8012007E0FFF7D7FF40F2E2
:1046F000F933984294BF0020012008BD38B51E4C04
:10470000002021694909FFF755FF2169002001F0C8
:104710001F01FFF757FFFE210022032000F0D8FA07
:1047200040210122032000F0D3FA00210A46032091
:1047300000F0CEFA002104460122032000F0C8FA5E
:10474000082C0E4B05D14FF40062DA6040F6FF7280
:1047500004E04FF40072DA6040F2FF329A60FFF733
:104760009DFF064B040224464FEAE475C3E9084561
:10477000C3E90645186138BDC00B00203002002097
:104780002DE9F84304F036FE624CA062FFF786FF85
:104790002369E06298423EDDE268C11A91420BDA79
:1047A0005D4B256B1A684D195143D4E9086772189F
:1047B00047EBE17325632BE094F801C0564A1CF0E7
:1047C000040F12D0A3681668C31A5E432CF0040CC1
:1047D00036464FEAE677236300220023C4E90867E0
:1047E00084F801C0C4E906234EE0A56816685A198A
:1047F0000132121A7243D4E90867236BED43ED18B6
:10480000B6EB020867EBE27942464B466918216332
:10481000C4E9082338E037DAE1681A1A8A420EDA66
:104820003D4D216B2D68C91A6A43D4E90867B6EB80
:10483000020867EBE27942464B460918E7E76178E0
:10484000354A11F0040F0FD0126821F004014243E1
:1048500012464FEAE273C4E9082300220023617084
:10486000C4E9062320630FE0A16812680131CB1A66
:104870001B185A43D4E90867B61847EBE277226B56
:10488000C4E908679B182363224B1D6B5A6B996B15
:10489000AA1A82EAE27CACEBE27C8C452CD942F28B
:1048A00010714A439E6ADC6B3C21341B92FBF4F28C
:1048B00051434FF4807C91FBFCF181EAE172A2EB61
:1048C000E172596440F6B8318A42DE635D631C646C
:1048D00001DDC82219E0B2F57A7F01DD642214E01F
:1048E000322A01DD0A2210E00A2A01DD05220CE04D
:1048F000012A0BDD012208E0996ADA6B8A1AB2F507
:10490000FA6F03D900225A6401329A63014B18618D
:10491000BDE8F883300200200400002038B50D46C1
:1049200018BB124CFFF72CFFD4E90801002901DB6A
:10493000A26803E0A268404261EB41011202124604
:104940004FEAE2730DF008FBC4E9062328464FEA5C
:10495000E071064C0B02020243EA1063D4E906013F
:10496000801841EB0301C4E9080138BD3002002082
:1049700008B508B100200CE0FFF702FF054BD3E9B2
:104980000601D3E90823121A63EB0103100A40EA77
:10499000036008BD3002002008B54FF4004008F065
:1049A00059FC0C4A002313600B4A002013600B4A89
:1049B0000021C2E900010A4A93840A4B1B7843B9DB
:1049C000094B9A6822F400429A60DA6822F40042A5
:1049D000DA6008BD680C0020400B0020600B00204E
:1049E00000080040300200200004014008B5084BD8
:1049F000587E10F0010005D0002006F027FF80F05F
:104A0000080001E006F022FFC0F3C00008BD00BFAF
:104A10000800002037B5044658B1002003240246A0
:104A200034212346009407F087F900202A21084A00
:104A30000AE00325024634212B46009507F07CF955
:104A400020462A2140F2FF7207F030F93EBD00BF38
:104A500001F8FFFF37B5044658B100200324024691
:104A600054212346009407F067F900204A21084AA0
:104A70000AE00325024654212B46009507F05CF915
:104A800020464A2140F2FF7207F010F93EBD00BFF8
:104A900001F8FFFF08B510B109F03CF801E009F09A
:104AA00041F808BD08B5C90805F062FA08BD00BFA5
:104AB0002DE9F0457F488BB0DFF80482012108F032
:104AC000ABFE09AD0420012109F01EFA03241026D3
:104AD000404642F206032946ADF824308DF82640C0
:104AE0008DF8276008F008FE0623734F4046C8F88B
:104AF00014304FF0040A4CF208632946ADF8243014
:104B00008DF826408DF827A008F0F6FD0820012139
:104B100009F0FAF941F6164338462946ADF8243033
:104B20008DF826408DF8276008F0E6FD41F2164327
:104B30003B614FF40063384629467B614FF0E80340
:104B4000ADF8243008F500688DF827A08DF82640D0
:104B500008F0D2FD3046012109F0D6F94EF20003EB
:104B600029464046ADF824308DF826408DF8276060
:104B700008F0C2FD4FF460430121C8F810304F48DF
:104B800008F04AFE00231A4619464D4C4FF40055D2
:104B900065612046A468013314F4804F4FF400543B
:104BA0000461806808BF013110F4804F18BF0132E2
:104BB0000A2BEAD10A2903D10A2A01D1012200E0F5
:104BC0000022404B01211A703A4808F025FE0420CB
:104BD00001213D4C09F098F900214FF4805008F074
:104BE0001BFE0121042009F09DF903AD20460AF0C7
:104BF0006BF9284609F05EFD294620464FF0000576
:104C00004FF0FF33ADF81030ADF80C50ADF8125046
:104C1000ADF80E5009F0F6FB0022134603212046A2
:104C200009F0FEFD684609F059FD4FF008072046DF
:104C30006946ADF808700AF0E3F84FF004036946DE
:104C40002046ADF800300AF0DBF8204641F65F61FF
:104C50000AF02CF820460121A58409F053FD00201C
:104C60000F2108F007FE012406A84FF40043069325
:104C70008DF81D708DF81C508DF81E4008F084FAD8
:104C8000124B08A89A686E4622F480629A60DA682D
:104C90008DF8234022F48062DA6028238DF82030DA
:104CA0008DF822508DF8215008F096FE0BB0BDE82B
:104CB000F08500BF00023000000C0140000430000D
:104CC000000801405C0B0020000800400004014087
:104CD00070B504460D461646032864D8DFE800F098
:104CE0000205080D4FF480520FE04FF4804201E0BE
:104CF0004FF400522D4B5A611AE02D4A138823F0CD
:104D000002031B041B0C138010222A4B5A612848F3
:104D1000022109F05BFA0028F9D02946244809F05D
:104D2000F9F92348012109F051FA0028F9D00FE0E0
:104D30002148022109F04AFA0028F9D029461E48E4
:104D400009F0E8F91C48012109F040FA0028F9D0DF
:104D5000E6B1032C27D8DFE804F002070A0F154B51
:104D60004FF480521A6119E04FF4804201E04FF491
:104D700000520E4B1A610FE00E4A0D4B10211161CB
:104D80001A8892B242F002021A8007E0032C0AD875
:104D9000DFE804F004020204074800E0044809F0D8
:104DA000BBF9C0B200E0002070BD00BF00100140A0
:104DB00000380040000C0140003001402DE9F04F68
:104DC00001218BB04FF4804009F0ACF8494C012030
:104DD00009AF014609F098F803264FF0180B20465A
:104DE00039464AF20003DFF81491ADF824304FF051
:104DF000040A8DF826608DF827B008F07DFC204667
:104E000039464FF480430DF11008ADF824308DF889
:104E100026608DF827A008F06FFC4FF48273002401
:104E200002224FF4007C012548464146ADF812307D
:104E30004FF00803ADF81620ADF81AC00392CDF874
:104E400008C0ADF81C30ADF81040ADF81440ADF816
:104E50001850ADF81E40ADF8204009F0E7F848467C
:104E6000294609F01FF929464FF4805009F04CF803
:104E700009F550492846214608F0CEFC48463946F7
:104E80004FF0A003ADF824308DF827B08DF82660E0
:104E900008F032FC484639464FF04003ADF8243064
:104EA0008DF826608DF827A008F026FC039ADDF81F
:104EB00008C04FF482734146ADF812300E484FF0EF
:104EC0002803ADF81620ADF81AC0ADF82040ADF8B3
:104ED0001040ADF81440ADF81850ADF81C30ADF8E6
:104EE0001E4009F0A3F80448294609F0DBF80BB08E
:104EF000BDE8F08F000C0140003001400038004058
:104F0000014B1878704700BF780200202DE9F84562
:104F1000054614460E4600294BD0002849D0814250
:104F200047D04FEA42185FFA88F848F0060739463A
:104F3000002006F075FD48F00C018246002006F0C6
:104F40006FFD804628460CF0C9FD054630460CF042
:104F5000C5FD014628460CF0CDFE064650460CF035
:104F6000BDFD31460CF0C6FE0CF0D6FF05464046AE
:104F70000CF0B4FD31460CF0BDFE0CF0CDFF0E4937
:104F8000002814BF80464FF001083046002D08BFAE
:104F900001250CF099FF18B14146204606F0BAFFF2
:104FA00039462A46002006F0EDFD044BE4180123A3
:104FB0002371BDE8F88500BF0000A0417802002001
:104FC00070B50D4D044645192B799BB1C6B20B4BFC
:104FD000710141F0060153F8202001F0E6010020A4
:104FE00006F064FE064B304653F8241006F092FF9C
:104FF00000232B7170BD00BF780200201C0B002025
:105000001807002013B5A64CA078002840F01F8395
:105010006378A52B00F0448259D8852B00F0E980F5
:1050200027D8072B00F01D810FD8032B00F0E1805B
:1050300005D8012B00F0B58000F2BD80ABE0052B58
:1050400000F0EF8000F20281D9E0812B00F0A9800E
:1050500009D80D2B00F03281802B00F09C800C2BA6
:1050600040F0F3820AE1832B00F0C98000F2A380B4
:1050700036E1952B00F0688115D88C2B00F0558116
:1050800008D8872B00F03681C0F0CB808A2B40F007
:10509000DC8235E1932B00F0118100F2EF808D2B43
:1050A00040F0D3824AE1A12B00F0DB8109D89A2B92
:1050B00000F07A81A02B00F0CE81992B40F0C582C0
:1050C0005DE1A32B00F0D78100F2DB81CDE1B72BAE
:1050D00000F06D8228D8AD2B00F0248210D8A92BC7
:1050E00000F0068205D8A72B00F0F68100F2FA81C5
:1050F000E3E1AB2B00F00582694C00F20882FBE192
:10510000B12B00F02F8206D8AF2B00F01582644C33
:1051100000F218820AE2B52B00F02E8200F23482EF
:10512000B22B40F0928221E2CC2B00F0798115D88D
:10513000C22B00F0578108D8C02B00F0928000F2FB
:105140004C81B82B40F0818235E2C72B7ED0C82B32
:1051500000F05681C32B40F0788249E1D52B00F056
:105160006E8109D8D22B00F03582D42B00F05F81FC
:10517000D12B40F06A8224E2D82B00F0408203D881
:10518000D62B40F062825EE1D92B00F04182DA2B0F
:1051900040F05B8251E2424B00205A680146DB78C6
:1051A00004E03F4B00205A68DB78022143EA0222E8
:1051B00006F0E8FC4EE23A4C0020E37862680821F1
:1051C00043EA022206F072FDE378A17862684901A1
:1051D00043EA0222002A41F00601B8BF524201F020
:1051E000E601002006F062FD2E4AA378D3180122C2
:1051F000DFE12B4B00205A680A21DB7875E0284C50
:105200000020E3786268062143EA022206F04EFDA0
:10521000E2786068A37842EA0020224A22499A187C
:105220000FE01F4C0020E378616843EA012106F09B
:1052300071FEE2786068A37842EA0020194A1B49AF
:105240009A1841F823000023137103E2144B184A03
:10525000D978184B01201B781070174A022B517215
:10526000D8E00F4B0122D978124B1878104B1A70E6
:10527000114B9972002840F0ED81CEE014210020FE
:1052800001AA06F01FFC064A9DF805305168D27845
:1052900052EA012114BF43F0020323F0020362E04B
:1052A00094060020780200201C0B00201807002024
:1052B000240C0020280C0020C00B0020142100200A
:1052C00001AA06F0FFFBA24A9DF805305168D2788A
:1052D00052EA012114BF43F0010323F0010342E02D
:1052E0009B4B00205A68DB78042143EA022206F037
:1052F000DDFCAFE1964B00205A680E21DB78F4E725
:1053000001AC22461421002006F0DCFB904B224623
:105310009978DB78490141F0140101F0F401002093
:105320008DF8063006F06AFD94E1E378894AC3F10E
:105330000801C9B2D37205F035F98BE1844B002026
:105340005A681A21DB78D0E7142101AA06F0BAFBCB
:105350006168E2789DF8053052EA012114BF43F0FC
:10536000040323F004038DF80530794B002099786D
:1053700001AA490141F0140101F0F401D2E701ACA6
:1053800022461821002006F09DFB714A9DF8053049
:105390009178D278490102F00F0223F00F0341F017
:1053A000180142EA030311E001AC22461821002053
:1053B00006F088FB664A9DF805309178D27849015D
:1053C00003F00F0341F0180143EA021301F0F80162
:1053D000224600208DF80530A4E75D4BDA785D4B5E
:1053E0001A7237E1E378626843EA0222594B2AE1F4
:1053F000574B5A68DB7843EA0222564B5A6029E140
:10540000534B554AD978554B01201B781070514A9F
:10541000032BD17740F01E810138FFF743FB19E1E0
:10542000E378626843EA02224A4BDA8112E1484B90
:105430005A68DB7843EA0222464B5A610AE1E27875
:10544000444B9A7706E1424B5A68DB7843EA0222E2
:10545000404B9A83FEE03E4B0020D97805F094F84B
:10546000F8E0E17805F086F8F4E0394B0020D978CF
:1054700004F060FFEEE0364B0020D97804F04EFFD8
:10548000E8E0002004F00CFC314C20B9E178A07871
:1054900004F02CFFDEE0E178A07804F0F7FED9E01C
:1054A00004F0FEFBE178A37818B9184604F012FF67
:1054B000D0E0184604F0D2FECCE0002004F0F0FB6F
:1054C000234C20B9E178A07804F0F8FEC2E0E1783E
:1054D000A07804F0CFFEBDE01D4B0020D97804F089
:1054E000E1FEB7E01A4B0020D97804F0E5FDB1E009
:1054F000E17804F0D5FDADE0E178002004F0C4FDD2
:10550000A8E0134B0020D97804F0B2FDA2E0E178C6
:10551000002004F0A1FDA178114BE27803EBC10358
:105520005A7197E0E17804F03BFD93E094F90310A1
:10553000002004F029FD8DE0054B0020D97804F00F
:10554000BDFF87E0E178002004F0ACFF82E000BFFF
:1055500094060020C00B0020240C0020280C002002
:10556000300B0020E17804F091FF73E03A4B00200B
:10557000D97804F07FFF6DE0374B5A68DB7843EA57
:105580000222364B9A6165E0334A354B5068D27837
:1055900042EA0020186010B9597904F05DFD2E4BE5
:1055A000304A9878125C012A54D1D97835E7E278EC
:1055B0002B4B1A714EE0284B0020D97804F0A2FE44
:1055C00048E0254B00205968DB7843EA0121FFF7CA
:1055D000A5F93FE0204C0020E378626803F01F014A
:1055E00043EA02221D4B1A61FEF7ECFFE378616883
:1055F000A07843EA01214911FEF7DCFF2AE0164BAF
:1056000000205968DB7843EA0121FEF763FF21E0BF
:10561000114C0020E378626803F01F0143EA022284
:10562000114B1A60FEF784FFE3786168A07843EAC3
:1056300001214911FEF774FF0CE0074B5A68DB7833
:1056400043EA0222094B1A6004E0032200E004222C
:10565000074B1A701CBD00BF94060020C00B002031
:10566000300B0020280C0020500B00204C0B002099
:105670000C07002013B5814B9A78002A40F0628213
:105680005B787F4CDA2B00F23E82DFE813F0DB0020
:10569000DE00E400E700EC00EE00F000F3000101A2
:1056A0001E01350123010A0114013C023C023C02A7
:1056B0003C023C023C023C023C023C023C023C02FA
:1056C0003C023C023C023C023C023C023C023C02EA
:1056D0003C023C023C023C023C023C023C023C02DA
:1056E0003C023C023C023C023C023C023C023C02CA
:1056F0003C023C023C023C023C023C023C023C02BA
:105700003C023C023C023C023C023C023C023C02A9
:105710003C023C023C023C023C023C023C023C0299
:105720003C023C023C023C023C023C023C023C0289
:105730003C023C023C023C023C023C023C023C0279
:105740003C023C023C023C023C023C023C023C0269
:105750003C023C023C023C023C023C023C023C0259
:105760003C023C023C023C023C023C023C023C0249
:105770003C023C023C023C023C023C023C023C0239
:105780003C023C023C023C023C023C023C02DB008C
:10579000DE004201EC00E400E700EE0045013C02BF
:1057A0003C0248013C02500156013C023C023C02D2
:1057B0003C023C0214010A0159013C023C023C0239
:1057C00063016D012301350101013C023C02AB0183
:1057D000AF01B301B701BB01C901D701E501E9017F
:1057E000ED01F101F501F901FC01000205020902D8
:1057F0000D021102150219021C021F0221022402CD
:105800003C023C023C023C023C023C023C02F300F3
:10581000760179017B017E0180013C02F00082016A
:105820003C023C023C0285013C0288018A01A00145
:1058300028022C023C02A201A501A8012F0232027B
:10584000360238020020014601E00020022106F065
:10585000E7F8606079E10020082101E000200A21DA
:1058600006F018F9F5E7074B4AE1074B48E1074B0B
:105870005B7A46E1054B9B7A43E100BF940600202A
:105880000C0700201C0B002018070020C00B002074
:10589000002005F0DBFF9D4B9B785B0050FA03F383
:1058A00010E00020142101AA06F00CF99DF8053043
:1058B000C3F3400325E10020142101AA06F002F9F8
:1058C0009DF8053003F001031BE1914B9B68C3F386
:1058D000C03316E17C21002001AA06F0F3F88B4BBF
:1058E00002219A789DF80630520011FA02F21A420B
:1058F0000CBF0023012304E101AA00207C2106F053
:10590000E1F8824B9DF806209B785B0052FA03F386
:10591000D8E700200421A3E700200E21A0E7002003
:10592000142101AA06F0CEF89DF80630E9E0002027
:1059300004F096F9C0F108008BE700201A218FE7E8
:105940000020142101AA06F0BDF89DF80530C3F32C
:105950008003D6E00020182101AA06F0B3F89DF8D4
:10596000053003F00F03CCE00020182101AA06F057
:10597000A9F89DF805301B09C3E0664B1B7AC0E00F
:10598000644BBDE0634B5B68BBE0634BB8E0634BCB
:10599000B6E0604BDB7FB4E05E4BDB89B1E0604B8F
:1059A000AEE0604B00221B78626013B15E4B0132A7
:1059B0005A605E4B5B4A1B780021117023B15A4B31
:1059C0005A6842F002025A600022584BBCE0584B21
:1059D00077E0504B5B6994E04E4B9B7F91E04D4BE1
:1059E0009B8B8EE0002004F043F932E7002004F0A6
:1059F00047F92EE7002004F04BF92AE7002004F0D5
:105A00004FF926E7002004F04BF9474C3F4B18B9FB
:105A1000987804F055F91CE7987804F071F918E7C4
:105A2000002004F03DF9404C384B18B9987804F048
:105A30004FF90EE7987804F073F90AE7002004F0B4
:105A40002FF9394C314B18B9987804F049F900E72F
:105A5000987804F05DF9FCE6002004F049F9F8E6D6
:105A6000002004F065F9F4E6002004F069F9F0E69E
:105A7000002004F06DF9ECE6002004F071F9E8E68E
:105A80002C4B5B793DE0002004F07AF9E1E6002040
:105A900004F07EF940B2DCE6002004F08BF9D8E691
:105AA000002004F08FF9D4E6002004F093F9D0E64A
:105AB000002004F097F9CCE6002004F0A3F9C8E632
:105AC0001D4B1B781DE0134B9B691AE0194B17E027
:105AD000184B1B7915E0002004F0EAF8B9E6002025
:105AE000FEF746FFB5E60B4B1B690AE0FEF7D6FD55
:105AF000AFE60020FEF7E2FCABE6104B00E0104BF7
:105B00001B68636021E0032323701EE094060020DD
:105B100000080140C00B0020240B0020E40B0020F3
:105B2000580B0020B40B00200C0700203C0B002079
:105B3000B80B0020300B00202C0B0020500B002055
:105B40004C0B00200A4B04221A700A4B1B786BB1D5
:105B5000074B09495A68094B0A601AB91A6842F09A
:105B6000080202E01A6822F008021A601CBD00BF99
:105B70000C07002006070020F40600209C060020E9
:105B800010B51B4A5378142B2DD8917871B95468ED
:105B9000D078184A1849927E40EA042041F8230040
:105BA00022B31BB303F5C270013013E0FF2918D1F3
:105BB00063B94FF4C364114920460919042204341F
:105BC00002F07AFCB4F5CD6FF5D10FE003F5C270A9
:105BD0000949013001EB83018000042202F06CFCD2
:105BE00004E0042200E00322054B1A7010BD00BF40
:105BF0009406002008000020A00600208C00002051
:105C00000C07002038B51F4C6578142D36D8A078C5
:105C100010F0800F18D010F0010F06D000200221E4
:105C200005F0FEFE184B43F82500184B9B7E43B34E
:105C3000144B5B782BB303F5C2701349013001EBB1
:105C400083018000042214E0B0B9022105F0E8FECF
:105C50000E4A0D4B927E43F8250092B1617881B1D6
:105C6000A0780422091801F5C270013003EB81010C
:105C7000800002F021FC04E0042200E00322044B37
:105C80001A7038BD94060020A006002008000020ED
:105C90000C07002038B5654CA07808B10422C2E09A
:105CA0006378952B1DD8932B7DD20D2B0AD80C2B06
:105CB00079D2052B4FD001D8042B09E0062B66D0F2
:105CC000072B1EE0862B46D005D8822B6ED0832B67
:105CD00040F0A88028E08C2B6CD08D2B40F0A28067
:105CE00079E0C32B00F087800ED8B52B77D004D88D
:105CF000993B012B00F296806FE0C12B72D077D8D0
:105D0000C02B40F08F8048E0CC2B7AD005D8C72B31
:105D10003DD0C82B40F0868070E0D52B78D0D62BB4
:105D20007AD0D42B7ED16FE0404D0020062106F0C2
:105D3000CFF8AC780020610141F0060101F0E601E6
:105D400005F0A8FE3A4AAB78D3183A4A42F8240044
:105D500000221A7169E0354D00200C2106F0B8F8D8
:105D6000AC780020610141F00C0101F0EC0105F07C
:105D700091FEAB78304A2E4942F8240018465B1851
:105D800052F8201000221A7106F0C4F84DE04920A4
:105D900002F07AFB294B587247E04A2002F074FB6C
:105DA000264B987241E00020142100E0042106F007
:105DB0008FF83AE04B200122214902F041FBA37801
:105DC0001E4A184602EB4313D97AC1F10801C9B241
:105DD00004F0E8FB29E01A21E9E71821E7E7582059
:105DE000184913E0482002F04FFB144B18721CE0D6
:105DF000402012490AE04420134907E05F2013497C
:105E000008E04E20124909E012495420042206E01D
:105E100011495E20012202E010495C20022202F0BA
:105E20000FFB02E003220E4B1A7038BD94060020CF
:105E3000780200201C0B002018070020C00B002057
:105E4000CB0B0020D80B0020C40B0020DF0B002060
:105E5000CE0B0020D40B0020DE0B0020DC0B00203A
:105E60000C07002010B51E4A5378142B34D89278B2
:105E7000AAB91C4A1C4952F823201C4B4A601B78C3
:105E8000002B2CD01A491B4B0A601AB91A6842F031
:105E9000080202E01A6822F008021A601FE0FF2AD6
:105EA00018D163B94FF4C364134920460919042279
:105EB000043402F0C5FAB4F5CD6FF5D10FE003F567
:105EC000C2700849013001EB83018000042202F016
:105ED000B7FA04E0042200E00322034B1A7010BD5D
:105EE00094060020A00600200C07002006070020D2
:105EF000F40600209C0600208C00002037B5134CCF
:105F0000657815B1012D1DD112E0042240F2FB701D
:105F100001A902F095FAE378626843EA0222019B44
:105F20009A420B4B02D101225A600EE05D600CE0F8
:105F3000A3782A2B06D1E11C40F2FB70042202F068
:105F4000BBFA02E0024B03221A703EBD9406002009
:105F50000C070020364900230B603649364A0B6097
:105F6000364910B50B6093749360D3601374537407
:105F7000334A4FF0FF3142F82310324A0024D45400
:105F800001332F2BF4D10731204605F049FD2E4B6C
:105F90000C211860204605F043FD2C4BD97A2C4B80
:105FA000C1F108011860C9B2204604F0FBFA294B80
:105FB0000022E2500434B4F5806FF8D1264B9B7E6A
:105FC0005BB104F5067425492046091904220434FE
:105FD00002F036FAB4F5CD6FF5D11F4BDB7E5BB91D
:105FE0004FF4A7641E49204609190422043402F024
:105FF00027FAB4F5C36FF5D1174B1B79012B03D0EA
:10600000112B01D0212B01D1012200E000220A4BEB
:1060100083F8D020104B5B7D23B1FEF7D9FA08B18D
:10602000012200E00022044B83F8D12010BD00BF04
:10603000F406002014070020780200209C060020AF
:106040008C020020380C00201C0B0020C00B00200C
:10605000180700201C070020080000208C000020EA
:10606000E401002008B50B4B5A7892B9997881B9B0
:106070005A68DB7843EA022240F2D2439A4208D1BE
:1060800040F2FF7002F096FA02F058FB0120FEF792
:1060900001FD08BD9406002010B59B4B9A78022A9A
:1060A00000F05581032A00F05B81002A40F0EB816B
:1060B0005A784D2A00F0B78023D8452A70D00ED8E0
:1060C000422A56D005D8402A45D0412A40F0D981ED
:1060D00046E0432A53D0442A40F0D38156E0482A70
:1060E0007CD005D8462A61D0472A40F0CA816AE0B0
:1060F0004B2A00F0858000F28F80492A40F0C18150
:1061000072E0542A00F0DE8011D8512A00F0AB80F2
:1061100006D84F2A00F08D80502A40F0B2819BE0D3
:10612000522A00F0B280532A40F0AB81B7E0832AB4
:1061300000F0F08006D8552A00F0D180572A40F0B0
:10614000A081D9E0852A00F0F580C0F0EB80FF2A1D
:1061500040F09781F7E06C4B40F2FF70D97805E092
:10616000694B6A4ADB7800201946137002F022FA64
:106170008CE1DB78654A194601205370F6E7624BE3
:10618000624ADB78042019461371EFE75E4B5F49E2
:106190005A68DB781C2043EA022341F81C3F0EE0DA
:1061A000DB785A4A194605205371DFE7564B5749A9
:1061B0005A68DB780C2043EA022341F80C3F0422A2
:1061C00002F07AF962E1504B504C5A68DB78214674
:1061D00043EA022341F8083F08206AE0DB784B4994
:1061E000262001F8263F78E0474A484BD27812B182
:1061F000474901224A60DA75444B1720D97DB5E73B
:10620000414B424CDB7803201946E37002F0D2F98F
:10621000E07802F0A7FB39E13B4B3C4ADB780220F7
:1062200019469370A2E7DB78384A19461520537552
:106230009CE7354B354CDB7819201946637602F024
:10624000B9F9607E10F0010002D00020012100E0C9
:10625000014605F019FD19E12B4B2C4ADB7816207D
:106260001946937582E7294A127D12F0010F05D075
:10627000DB7813F0010F01D102F060FA224B234AC0
:10628000DB7814201946137570E71F4B1F495A68B5
:10629000DB78202043EA022341F8203F8FE71A4BA6
:1062A0001A4C5A68DB78214643EA022341F8103F32
:1062B0001020042202F000F922696079A16802F03E
:1062C000B3FDE3E05A68DB7843EA0222012A00F2D8
:1062D000DA800E491A2001F81A3F012270E70A4BB2
:1062E0005A68DB7843EA0222012A00F2CC8007498F
:1062F0001B2001F81B3FF0E7034B0449DB78272004
:1063000001F8273FE9E700BF9406002008000020BD
:106310000C0700205A68DB7843EA02225C4BC3F882
:10632000D420B3E05B4B5A68DB7843EA02225A4B35
:106330001A60ABE0574B5A68DB7843EA0222544BB1
:10634000C3F8D820A2E0534BDA78544B9DE058684C
:10635000D9785A78524B41EA002143F8221095E04F
:106360005A78272A59D00ED8022A33D004D8CAB175
:10637000012A40F0868021E01B2A3ED01C2A44D00E
:10638000092A7ED132E02B2A5FD005D8292A50D0A5
:10639000D978444A54D847E02D2A64D05CD32E2AB9
:1063A0006FD167E05A68DB7843EA02223D4B1A60FE
:1063B00003F020F8364BC3F8DC0067E05A68DB785E
:1063C00043EA0222374B5A6003F014F8304BC3F80B
:1063D000E0005BE05A68DB7843EA0222314B9A60C6
:1063E00003F008F82A4BC3F8E4004FE05A68DB7862
:1063F00043EA02222B4BDA6048E05968DB78002040
:1064000043EA012105F03AFD40E05968DB780020BD
:1064100043EA012105F006FD38E05A68DB7843EADB
:106420000222204B1A6131E05B6841EA032151618D
:106430002CE05A68DB7843EA02221A4B9A6125E085
:106440005B6841EA0321D16120E05A68DB7843EAC6
:106450000222144B1A6219E05A68DB7843EA0222DE
:10646000104B5A6212E05A68DB7843EA02220D4B65
:106470009A620BE05A68DB7843EA0222094BDA623F
:1064800004E0032200E00422074B1A7010BD00BF95
:10649000780200209406002008070020050700204D
:1064A0001C070020E80B00200C07002008B5824BD9
:1064B0009A78022A00F0B980032A00F0BB80002AF3
:1064C00040F01E815B78502B6ED022D8462B54D0E2
:1064D0000ED8422B47D005D8402B3DD0412B40F061
:1064E0000D813EE0442B43D0744B754A43D83DE0C8
:1064F0004B2B4DD006D8482B43D040D3492B40F0EE
:10650000FD8042E04D2B49D045D34F2B40F0F68023
:1065100047E0812B5FD010D8542B4ED005D8522B9A
:1065200047D0664B664A46D841E0572B4BD0802B6C
:106530004DD0552B40F0E28042E0852B5DD004D851
:10654000832B53D05D4B55D84DE0FE2B64D066D8DD
:10655000F02B40F0D3805FE040F2FF7001F094FF39
:106560009CE0574B59E0564B5A78C4E01279C3E08F
:10657000534BDA69BFE05279BEE0514B85E0504B96
:1065800080E04F4B93F82620B5E04D4BDA7D48E094
:106590004B4BDA78AFE04A4B9A78ACE0484B5A7DE7
:1065A000A9E0474B5A7EA6E0454B9A7DA3E0127DB9
:1065B000A2E0434B95E012699EE0414B9A7E9AE03F
:1065C0003F4BDA7E97E03E4B93F8272093E03D4B1C
:1065D00093F8D1208FE03B4B93F8D120042A14BFCD
:1065E0000022012287E0374A926885E0354BD3F8D4
:1065F000D42080E0344A12687EE0324A334BD2F82D
:10660000D8104B4303F5405339332C4923F0004055
:106610004860C2F8D83076E02D4B1A786BE02D4BED
:106620001A78003A18BF012265E05A782A4B53F8CD
:10663000222060E05B78272B33D00DD8022B20D0AE
:1066400003D8C3B1012B59D118E01B2B1FD01C2B31
:1066500021D0092B52D117E02B2B41D005D8292B63
:1066600024D0164B1D4A24D81EE02D2B3ED03AD301
:106670002E2B43D13DE0194B1A683CE0174B5A686A
:1066800039E0164B9A6836E0144BDA6833E00020A4
:1066900005F042FA02E0002005F02AFA074B5860A4
:1066A00031E00E4B1A6926E0526925E00B4B9A69DE
:1066B00021E0D26920E000BF940600200C070020F2
:1066C0000800002078020020080700206D4EC64117
:1066D0001C0C0020050700201C070020E80B0020F0
:1066E000124B1A6A07E0114B5A6A04E00F4B9A6A80
:1066F00001E00E4BDA6A0E4B5A6004E0032200E020
:1067000004220B4B1A700B4B1B786BB1084B0A49D8
:106710005A680A4B0A601AB91A6842F0080202E085
:106720001A6822F008021A6008BD00BFE80B0020BA
:106730000C07002006070020F40600209C0600201D
:1067400010B5154CA07818BB6378012B16D003D375
:10675000022B124C19D114E004F010FDA17839B1CC
:106760000F4A937FBBB102EB4112927F9A4212D142
:106770000C4B01221A71013A0B4B0BE004F006FDA1
:1067800009E004F00BFD606005E00323237002E0E4
:10679000024B04221A7010BD940600200C07002042
:1067A000C00B0020780200203C0B002037B5504B76
:1067B0001A7CA2B94F494868CA7842EA0022B2F16D
:1067C000FF3F04BF4C4A12680A214A43C3F8E8203D
:1067D00002F010FE464B01221A74C3F8EC00454B40
:1067E0005B78042B00F28280DFE803F003353F4F33
:1067F000130002F0FFFD3E4BD3F8EC10D3F8E82075
:10680000411A0029B8BF494291426CD900221A743A
:106810006CE0384B364C987804F0C0FC30B9374AFD
:106820002074136823F0100313605FE0D4F8E8309D
:10683000002B57D002F0DEFDD4F8EC20D4F8E8307D
:10684000821A002AB8BF52429A424BD92B4B0021E0
:106850001A68217442E0002004F0F8FF254B244C14
:106860009D786D0050FA05F51CE000207C2101AAFE
:1068700005F028F91F4B02229D789DF806306D0027
:1068800012FA05F51A4C1D400EE001AA00207C21E9
:1068900005F018F9174A9DF806309578144C6D00EC
:1068A00053FA05F515F0010506D0144B00211A68BE
:1068B000217422F0100213E0D4F8E83093B102F012
:1068C00099FDD4F8EC20D4F8E830821A002AB8BF39
:1068D00052429A4206D9094B25741A6842F01002B6
:1068E0001A6003E0024B9A68013A9A603EBD00BF0D
:1068F0007802002094060020F40600209C06002068
:1069000008B5184B9A7812B1022A26D106E05868C9
:10691000DB7843EA0020FEF79DF821E0587807284D
:106920000AD85A68DB7853EA022202D1FDF760FDEB
:1069300016E0FDF76DFD13E0FF280CD15868DB78F9
:1069400043EA0020B0F1FF3F0ABF074BC0B21878FE
:10695000FDF76EFD04E0032200E00422034B1A70F1
:1069600008BD00BF94060020F40600200C0700209C
:1069700010B5224B9A78012A23D003D3022A204C47
:1069800028D122E05878082802D8FDF74FFE15E0FC
:106990000A2801D100220AE00B2802D1FDF79EFE51
:1069A0000CE00C2806D1174B9A68C2F3C032144B86
:1069B0005A6011E0FF280FD1FDF75EFE104B5860C2
:1069C0000AE0587802F034FDF8E75878FDF744FD06
:1069D000606001E0042323700B4B1B786BB1084B04
:1069E0000A495A680A4B0A601AB91A6842F0080242
:1069F00002E01A6822F008021A6010BD9406002016
:106A00000C0700200008014006070020F4060020C3
:106A10009C06002010B5204B5A78812A3AD19A78EA
:106A2000922A37D19A79A32A34D15A79B42A31D10A
:106A30001A79C52A2ED1DB78D62B2BD1174B4FF4E0
:106A400000421A6103F074F802F0D4FC044602F02C
:106A5000D1FC001B0028B8BF4042B0F57A7FF6DBBE
:106A6000FDF71AFD06F07CFF002007F0A9FC0021CD
:106A70000B4806F02BFB0A4806F088FA094805F097
:106A800043FF06F073FB4FF0804008F01DFA002032
:106A9000FEF700F810BD00BF940600200010014072
:106AA00008000240002401402DE9F3479D4A9E4D15
:106AB000D0785168137840EA01204FF0640C222B03
:106AC00085F800C06B70686000F0798554D80F2B92
:106AD00000F0358324D8072B00F00A8210D8032B4E
:106AE00000F0F88006D8012B00F0A680022B40F0C1
:106AF000A787C8E0052B00F0F38100F2F58101E1E2
:106B00000B2B00F0DF8205D8092B00F0D38200F2B6
:106B1000D582CBE20D2B00F00A8300F20C83EAE26F
:106B2000192B00F0B38412D8152B00F0BF8306D8C0
:106B3000132B00F00883142B40F082876BE3172B94
:106B400000F08484794B00F2948400F078BC1E2B12
:106B500000F0C68409D81B2B00F0BA84C0F0A684CC
:106B60001C2B40F06D8700F0B6BC202B00F0BE84DB
:106B700000F2BF8400F0B7BC812B00F0CE852ED888
:106B8000412B00F0B08515D8252B00F05E8507D885
:106B9000232B00F02085242B40F0528700F027BDE6
:106BA000272B00F08985C0F05B85402B40F048879B
:106BB00000F096BD452B00F0A28506D8432B00F0CF
:106BC000988500F2998500F091BD472B00F09D85D6
:106BD000C0F09885802B40F0338700F099BD882B5A
:106BE00000F03D8612D8842B00F0E28507D8822B76
:106BF00000F0AB85832B40F0238700F0ABBD862BE4
:106C000000F0F08500F24A8600F0E7BD8C2B00F022
:106C10008F8606D88A2B00F0728600F2848600F0F8
:106C20006BBEF22B00F0DC86FF2B00F0FB868D2B79
:106C300040F0068700F07FBE9378FBB93B4B4FF0E6
:106C4000010C83F804C03A4B00241C70394B2146D8
:106C50001C702046022204F0BDFE2046062140F2B0
:106C6000FF7205F023F82F4B20465A68DB78082185
:106C700043EA022205F01AF800F0E5BE2A4B04228E
:106C80001A7000F0E0BE274DAC78F4B9274B4FF0F6
:106C9000010C83F804C0264B21461C70254B20466E
:106CA0001C70022204F096FE2046062140F2FF727C
:106CB00004F0FCFF6A68EB78204643EA0222524265
:106CC000082104F0F3FF00F0BEBE174B04221A7037
:106CD00000F0B9BE94788CB9154B20461C70154B4A
:106CE0001C7004F053FA20462146022204F072FE82
:106CF0002046082104F0EEFF00F0A5BE04232B700F
:106D000000F0A1BE074B9A78002A40F0E4805B783F
:106D1000032B00F2DB80DFE813F00F004900940042
:106D2000BA0000BF940600200C0700207802002063
:106D3000B40B00203C0B0020A54D0020FEF740F9CD
:106D4000A44EAB7800246868EA78F454A24E590146
:106D500042EA0022F45401F0E001204604F012FF60
:106D6000A9782246204604F035FEA9789B4A02EB1A
:106D700041139B7F002B00F06686002900F063869C
:106D8000927F9A4240F05F862046FEF719F96A68C2
:106D9000EB78204643EA0222214604F0F3FE204627
:106DA0002146224604F016FE00F04DBE884D00201C
:106DB000FEF706F9AB78874A00245901D454864A75
:106DC00041F00201D45401F0E201204604F028FE13
:106DD000EB786E68A97843EA06268619490101F026
:106DE000E0013246204604F0CDFE2046A978224636
:106DF00004F0F0FDA878794A794902EB40139B7FB3
:106E00004E60002B00F01F86002800F01C86927F49
:106E10009A4240F01886FEF7D3F80221204604F08B
:106E2000FFFD6A68EB78214643EA02228218204679
:106E300004F0A8FE20462146224604F0CBFD00F0D7
:106E400002BE634CE378626843EA0223142B19DC28
:106E5000644A002052F82360FEF7B2F8A378324665
:106E60005C4E0025F5545C4E5901284601F0E001C6
:106E7000F55404F087FE2846A1782A4604F0AAFDBE
:106E800000F0E1BD564B04221A7000F0DCBD504CFE
:106E90000020E3786268002543EA0222514B53F850
:106EA0002260FEF78DF8A37832464A4E5901F55418
:106EB000494E284601F0E001F55404F063FE2846EF
:106EC000A1782A4604F086FD00F0BDBD444B0322A4
:106ED0001A7000F0B8BD424B04221A7000F0B3BD26
:106EE000FEF790F800F0AFBDFEF7C4FB00F0ABBDBD
:106EF000907818B104232B7000F0A5BD53789A2B1D
:106F000021D8992B80F08280822B6DD00BD8062B54
:106F10004AD003D8042B3BD0052B0AE0072B4AD0DC
:106F20000C3B012B0CE08C2B63D005D8832B2FD08E
:106F3000862B40F0B68031E08D2B61D0933B022B45
:106F400000F2AF803EE0C72B2ED00ED8C12B69D007
:106F500005D8B52B5FD0C02B40F0A3802BE0C22B0F
:106F600067D0C32B40F09D806AE0D22B7DD005D83E
:106F7000C82B6CD0CC2B40F094806FE0D52B00F068
:106F80008280D62B00F08680D42B40F08A8073E07C
:106F90000020062104F0D4FD00F055BD00200C2196
:106FA00004F0CEFD00F04FBD0C4B4920597A01F0A2
:106FB00001FB00F048BD094B4A20997A01F0FAFA2A
:106FC00000F041BD0020142104F0BAFD00F03BBDEB
:106FD000940600203C0B0020B40B0020C00B0020C6
:106FE0000C070020A0060020042104F0A9FD00F0F9
:106FF0002ABD4B209E49012201F05EFA00F023BD1C
:1070000000201A2104F09CFD00F01DBD182104F0A1
:1070100097FD00F018BD58209649042201F04CFA63
:1070200000F011BD944B4820197A01F0C3FA00F02A
:107030000ABD40209049042201F03EFA00F003BD51
:1070400044208E49042201F037FA00F0FCBC5F2096
:107050008B49012201F030FA00F0F5BC4E2089493D
:10706000022201F029FA00F0EEBC502086490422E9
:1070700001F022FA00F0E7BC54208449042201F018
:107080001BFA00F0E0BC5E208149012201F014FAF5
:1070900000F0D9BC5C207F49022201F00DFA00F01B
:1070A000D2BC7D4B03221A7000F0CDBCFEF7F2FD7E
:1070B00000F0C9BCFEF7F0FF00F0C5BCFFF7F6F921
:1070C00000F0C1BC9378022B11D15378372B0AD82A
:1070D000724903F5A77001EB83018000042201F0DF
:1070E000EBF900F0B0BC03232B7000F0ACBC042320
:1070F0002B7000F0A8BC6A4B9A78022A12D15B78F8
:10710000372B0AD8654903F5A77001EB830180008E
:10711000023201F095F900F096BC5F4B03221A7021
:1071200000F091BC5C4B04221A7000F08CBCFFF79D
:1071300007FB00F088BCFFF7E3FB00F084BCFFF71F
:1071400017FC00F080BC5278564B092A53D8DFE870
:1071500002F0050D151D26313941494C504A196878
:107160005068D27842EA0022521843E04C4A19682B
:107170005068D27842EA00228A1A3BE0484A1968ED
:107180005068D27842EA00224A4333E0444A196800
:107190005068D27842EA002291FBF2F22AE040489D
:1071A00019684468C27842EA042291FBF2F002FBBB
:1071B00010121FE03A4A19685068D27842EA002259
:1071C0000A4017E0364A19685068D27842EA00222D
:1071D0000A430FE0324A19685068D27842EA002226
:1071E0004A4007E01A68D24304E02D4A5168D27839
:1071F00042EA01221A602B4A2B4B12682AB91A68FC
:1072000042F008021A6000F01EBC1A6822F0080260
:107210001A6000F018BC224B224A5968DB781268C9
:1072200043EA01239A4206DD1F4B1A6842F004022A
:1072300022F003020CE01C4B05D11A6822F0060272
:1072400042F0010204E01A6822F0070242F0020252
:107250001A60144A144B126822B91A6842F00802E4
:107260001A60F0E31A6822F008021A60EBE300BF2C
:10727000CB0B0020D80B0020C00B0020C40B00203B
:10728000DF0B0020CE0B0020D00B0020D40B002001
:10729000DE0B0020DC0B00200C0700201C07002068
:1072A00094060020F40600209C06002053780C2B46
:1072B00000F2C983DFE813F00D001B00290037003E
:1072C0004500530061006F007D008B009900A7000E
:1072D000B500944B1B6813F0080F00F0B483924B79
:1072E0005A68DB7843EA0222904B9A60ABE38D4BFD
:1072F0001B6813F0080F40F0A6838B4B5A68DB78AD
:1073000043EA0222894B9A609DE3864B1B6813F087
:10731000010F00F09883844B5A68DB7843EA02221D
:10732000824B9A608FE37F4B1B6813F0010F40F094
:107330008A837D4B5A68DB7843EA02227B4B9A6052
:1073400081E3784B1B6813F0040F00F07C83764BCD
:107350005A68DB7843EA0222744B9A6073E3714BFC
:107360001B6813F0050F00F06E836F4B5A68DB78D3
:1073700043EA02226D4B9A6065E36A4B1B6813F087
:10738000020F00F06083684B5A68DB7843EA022200
:10739000664B9A6057E3634B1B6813F0030F00F0D2
:1073A0005283614B5A68DB7843EA02225F4B9A6052
:1073B00049E35C4B1B6813F0100F00F044835A4BF9
:1073C0005A68DB7843EA0222584B9A603BE3554BFC
:1073D0001B6813F0200F00F03683534B5A68DB789C
:1073E00043EA0222514B9A602DE34E4B1B6813F087
:1073F000400F00F028834C4B5A68DB7843EA0222A6
:107400004A4B9A601FE3474B1B6813F0800F00F054
:107410001A83454B5A68DB7843EA0222434B9A6051
:1074200011E3404B1B6813F4807F00F00C833E4B4C
:107430005A68DB7843EA02223C4B9A6003E33A4AFB
:107440005168D27842EA01229A60FCE2374BDA684E
:10745000072A00F2F88234499C684868C97841EAF2
:107460000020511C03EB8202C2F8F0409860D96002
:10747000E9E2DA682D4B002A00F0E582013A03EBDD
:107480008201D1F8F010DA609960DCE253782E2B9B
:1074900003D8274A0121D154D5E2FF2B03D1234B36
:1074A00001225A74CFE203232B70CCE21E4B5B788F
:1074B0002E2B03D81E4A0021D154C4E2FF2B03D146
:1074C0001A4B00225A74BEE21A4B03221A70BAE217
:1074D000FFF76CF9B7E2154B002283F8D120B2E236
:1074E000FEF74EFBAFE2FEF7BDFCACE2FEF78AFB17
:1074F000A9E20D4A104B52780A2A52D8DFE802F06E
:10750000060B20252B33393F45494C000B491A689F
:1075100009688A1803E0094A196812688A1A1A6009
:107520003FE000BF9C060020940600207802002067
:10753000380C00200C070020F4060020140700205F
:10754000934A196812684A43E9E7914A1968126830
:1075500091FBF2F2E3E78E4A1968126891FBF2F0B0
:1075600002FB1012DBE78A491A68096801EA020285
:10757000D5E787491A68096841EA0202CFE78449DA
:107580001A68096881EA0202C9E7814B1A68D24386
:10759000C5E71A687E4BC2E77D4A1868116810601B
:1075A00019607C4A7C4B126822B91A6842F00802C2
:1075B0001A6048E21A6822F008021A6043E2754B2A
:1075C00001F07F4118681B7841EA10215160D370A7
:1075D000FDF718FD37E26F4B01F07F4118681B780B
:1075E00041EA10215160D370FEF756FD2BE26B4B40
:1075F0005B78052B00F22782DFE803F003090F1503
:107600001B21654B1A6802F00F021A601BE2624BE5
:107610001A6822F010021A6015E25F4B1A6822F015
:1076200020021A600FE25C4B1A6822F040021A60D6
:1076300009E2594B1A6822F080021A6003E2564BA5
:107640001A6822F480721A60FDE153782E2B04D858
:10765000534A02EB83035861F5E103232B70F2E1F7
:107660004F4BDFF830C1D3F810914E4993F82C21DD
:10767000D3F814A1CCF80090DFF814C1D3F8187136
:10768000D3F81C81D3F82061D3F82451D3F82841D2
:10769000CCF800A0885CDFF800C19F60CCF80080C7
:1076A0001E74C3F8EC50C3F8E84008B101238B54B2
:1076B0003B4B00229A74C6E193786BB9374B5B78E9
:1076C000142B05D8334A1168374A42F82310BAE11F
:1076D000364B03221A70B6E1344B04221A70B2E121
:1076E00002F070FAAFE102F06FFAACE102F06EFA6C
:1076F000A9E102F06DFAA6E102F06CFAA3E102F052
:107700006BFAA0E102F06AFA9DE102F069FA9AE1EF
:10771000234B002283F8D12095E1537813B1012B3C
:1077200010D104E01E4B012283F8D1208BE1B0F58B
:10773000006F04D21A4A906082F8D13083E10423AA
:107740002B7080E103232B707DE1154B022283F81F
:10775000D12078E1124B002199745974104A4FF0EE
:10776000FF3402F1140040F821400E480023435436
:1077700001312F29F2D1084913740B60054982F8B1
:10778000D1300B60024993600B60D3605BE100BFB6
:1077900014070020F40600209C0600209406002018
:1077A00078020020380C0020A00600200C070020E2
:1077B0008D4B1B7D13F0020F0CD1B0F5006F06D27C
:1077C0008A4B0422C3F8300183F8D1203BE1042323
:1077D0002B7038E108232B7035E1844B002283F8AD
:1077E000D12030E1804B01219A78814BB0F5006FB8
:1077F0001970804B1A7028D27B4B1C7D0C4024D111
:10780000694600F0DFFF7B4B9DF800709DF801603A
:107810009DF802509DF806C09DF805009DF80410E3
:107820009DF803201C725F709E70DD7083F804C0A9
:1078300058719971DA7101236E4A985C117A01339B
:107840004118082B1172F7D1FDE00123694A00218C
:1078500099540133082BF9D113781372F3E053785C
:107860008BB9614A01209178634A1468604A1070AC
:10787000604A11700133E21812F8011C5D4A082BAE
:107880009954F7D1DFE0012B40F0DD801B222A71F3
:107890000422EA717032AA716B71D4E0574B5B78A5
:1078A000032B00F2D080DFE803F002101D224F4AC4
:1078B000534BD2F8301192F8D1C0107C0A0A1971DA
:1078C00083F807C098715A71BDE0484A4C4B9168E3
:1078D00092F8D1C0107C0A0A197183F807C0987118
:1078E0005A71B0E0474B1A68454B5A60ABE0464BC3
:1078F0001A68434B5A60A6E0FEF7B4FBA3E0527847
:10790000424B02B101221A703C4B414AD878374BA6
:10791000107093F834113F4A002311703E4A1370DF
:107920003E4A13708FE0314B012283F835218AE003
:10793000FEF7E4FA87E0314B5B78032B4CD8DFE8A5
:1079400003F00C023C472D4B28495A68DB78D1F8EC
:10795000381143EA022C00232BE0244BD3F83821C2
:10796000092A0CD82549501C4C68C97803EB8202BF
:1079700041EA0421C2F83C11C3F8380163E0204B0E
:1079800009221A705FE052F82340581C64450FD159
:1079900002EB8002013904E052F8040C013342F892
:1079A000080C04328B42F7D3104BC3F838114AE06D
:1079B00003468B421A4AE6D345E00C4A0023C2F83C
:1079C0003831174A0021D1500433282BF9D13AE03D
:1079D0000B4B0A225A6036E0094B03221A7032E040
:1079E000FFF718F82FE000BF080000207802002001
:1079F000F8060020FC06002000000020940600206D
:107A00000C070020F406002014070020280B00209B
:107A1000540B0020260C00206C0C0020440B00208E
:107A2000B4030020094B5A68DB7843EA022240F293
:107A3000D2439A4207D1064B012283F8642102E027
:107A4000044B02221A70BDE8FC8700BF9406002098
:107A5000780200200C07002073B5204B02464078C6
:107A60001F4D1870907800265870D078EC469870AA
:107A700010790C4698715079587192F806E095E8A3
:107A8000030083F804E0D2798CE80300DA70154B28
:107A90001E70FFF709F8144B1B7873B963702370DD
:107AA0002B78A3706B78E370EB792371AB796371FA
:107AB0006B79A3712B79E37108E0012B06D10B4B95
:107AC0009B195B78A3550136082EF8D1044B6A4602
:107AD00092E8030083E803007CBD00BF9406002009
:107AE0000C07002006070020F8060020FC060020F6
:107AF000F7B5114D114C6F684FF0000C07F07F4740
:107B000047EA13276F600E4F6E4687F800C0287053
:107B10006970AA7094E80300EB7086E80300FEF732
:107B2000C3FF96E803006368227884E803000549F0
:107B300018460A70FEBD00BF940600200C07002006
:107B400006070020780200202DE9F04F984B9BB0EB
:107B50001B781BB9974B93F865316BB1964B1B782B
:107B6000062B09D00A2B07D00F2B05D01F2B03D0D3
:107B7000904B002283F834218E4A92F83431591EFA
:107B8000C9B2012946D892F866018C498C4ACC6862
:107B90001278012B0CBF4FF0070C4FF0080C00239C
:107BA0000E948DF834C08DF835008DF83630CAB992
:107BB000844B8E681D7819795C7893F807C09879A2
:107BC0005B798DF83C608DF83D508DF83E408DF826
:107BD0003FC08DF840008DF841308DF842108DF88F
:107BE00043200AE0012A08D1774A0133995C1AA898
:107BF000C218082B02F82D1CF6D1744B1B78002BF1
:107C000040F0C2800DA801F02DF8002840F0BC80A3
:107C100000F00FBC032B25D192F8D040002C40F08F
:107C20008680674B1B7893B9644D664CA8786E7854
:107C3000227863788619B618E279F618A379B6180F
:107C40006279F6182379B618F618F6B219E0012B06
:107C500040F09A805C4BE05C013400F09FFE092C00
:107C6000F8D191E0042B27D1544D564CAB786E7867
:107C700018469E1901360023012222706360F6B275
:107C8000637000F08BFE687800F088FE207800F0CA
:107C900085FE607800F082FEE07900F07FFEA0793A
:107CA00000F07CFE607900F079FE207900F076FE2D
:107CB000304600F073FE67E0072B3CD192F8D030DD
:107CC000002B34D13E4A127822BB3C4A3D4B5578BA
:107CD00096781C7893F801C0AF19D879E71999798B
:107CE00067445A79C7191B79CF19D719DF198DF84D
:107CF00058708DF850608DF851508DF852408DF8C5
:107D000053C08DF854008DF855108DF856208DF81D
:107D1000573008E0012A06D12B4A995C14AAD154A5
:107D20000133092BF8D1294B1B786BB328E0254888
:107D300004F00AFA28E0082B26D1204B00225978BB
:107D40009878224B45181C781E4B4FF0010C0135DA
:107D50005A608DF852C08DF8532016468DF8542085
:107D60008DF855208DF856208DF857208DF85850F5
:107D70005A7083F800C08DF850008DF851101CB176
:107D800014A8092101F0AAFD114B1B78002B00F06B
:107D90009980104A0D4B12780F4C013A062A00F2D6
:107DA0008C80DFE802F01B1B418A8A8A650000BFD5
:107DB000050700207802002094060020080000201B
:107DC000F80600200C070020FC060020200B0020F5
:107DD0006C0C0020260C0020440B0020AB4A94F8C9
:107DE00000C0D068926819788DF82C206FF07F025F
:107DF0008DF82D200A3200238DF82E207D328DF84B
:107E000032C08DF824208DF826300A908DF82F305E
:107E10008DF830308DF831308DF8253000294CD177
:107E200009A800F01FFF48E0984D2278AB786E78E3
:107E300018469E190A36B61800F0B0FD687800F0B2
:107E4000ADFD802000F0AAFD8A2000F0A7FD0020F3
:107E500000F0A4FD002000F0A1FD002000F09EFD38
:107E6000F6B2207800F09AFD304600F097FD24E04D
:107E700086482278417880786FF07F0500EB010C0E
:107E80001C780CF10A0C002394448DF846500A35F6
:107E90008DF847508DF84A308DF84CC08DF844006D
:107EA0008DF845108DF848308DF849308DF84B200D
:107EB0001CB111A8092101F011FD754A00231370AE
:107EC000744A1370744B754893F864110022027061
:107ED00083F8652183F8342111B10120FCF7DAFD24
:107EE0006D4B93F8352152B193F8D0200021D2F197
:107EF000010238BF002283F8351183F8D020684B87
:107F00001B78002B46D10DA800F08AFE002841D036
:107F10009DF83430062B3DD9624B5C4A9DF83C708D
:107F20009DF83D609DF83E509DF83F409DF840E033
:107F30009DF841C09DF84280116983F803801F704D
:107F40005E709D709C7183F805E083F804C00E9B01
:107F5000514A9DF835008B4282F8660102D1012317
:107F600082F8653101F046FA9DF834304FF0000296
:107F7000072B4D4B484C18604C4B1A7001D1012314
:107F800000E0022384F83431434B93F8D1305A1E79
:107F9000D2B2E8E0404C94F8D050002D40F08C80F4
:107FA0000DF1670000F0C8FC002800F0858000F0AB
:107FB000DFFC08B184F86751374B9DF8670093F8F0
:107FC00067114A1CD2B2C918092A81F8680183F8DE
:107FD000672140F0F1802D4993F8682148784FF0EF
:107FE000000C904283F867C107D091F82730002B2E
:107FF00000F0E2809A4240F0DF80244B93F8273073
:10800000934203D1244B012283F8652100231A46B1
:10801000214C04F5B471C95C01335218082BD2B25B
:10802000F6D194F8703193422DD11E4B94F86D1116
:1080300094F86E2194F86F5194F8696194F86AE1AC
:1080400094F86BC194F86C01DD7059711A711E704F
:1080500083F801E083F802C0987101F0CBF9144D68
:1080600094F8D1302860591E12480022C9B202701B
:108070000320012984F8340184F8672177D9052B7E
:1080800075D0013291E0042373E000BF08000020A6
:108090006C0C0020440B002078020020F806002021
:1080A000200B002094060020180C0020210B00203B
:1080B000200C0020250C00209B4C94F8D03083B17C
:1080C0009A4804F087F860B101F094F9984994F85F
:1080D000D130086097495A1E00200870D2B203219F
:1080E0003FE0914B93F8D040002C45D1924B1B7848
:1080F000002B41D017A801F0DBFB00283CD0234621
:10810000224617A9C95C01335218082BD2B2F8D104
:108110009DF86410844C91422BD1844B9DF86110E2
:108120009DF862209DF85D609DF85EE09DF85FC05F
:108130009DF860009DF8635059711A711E70DD70D2
:1081400083F801E083F802C0987101F053F978498F
:1081500094F8D130086077495A1E00200870D2B2D6
:10816000072184F83411012A01D9052B1CD10022E2
:108170001BE084F834311FE06B4C94F8D130013BA4
:10818000DBB2012B18D8A368B3F5006F10D2FCF74F
:108190001FFA68B1A368654918460133A36000F06F
:1081A00011FB092384F834310122644B1A7003E077
:1081B0005D4B002283F8D1205B4C94F8D130042B26
:1081C00005D15A4E327812F0800F00F00581564BDF
:1081D00093F834313BB1042B05D0082B03D0062B88
:1081E00001D0FEF761FC504C94F83431092B40F07B
:1081F000CA8001F0FFF8D4F8DC30514AC31A002BD2
:108200001268B8BF5B4293420AD94E4B1A78012AD2
:1082100001D101321A7001F0EDF8434BC3F8DC00D4
:1082200001F0E8F8404BD3F8E020454B821A002AD1
:108230005B68B8BF52429A420AD9424B5A78012A27
:1082400001D101325A7001F0D5F8374BC3F8E00084
:1082500001F0D0F8344BD3F8E420394B821A002ACD
:108260009B68B8BF52429A420AD9364B9A78012A83
:1082700001D101329A7001F0BDF82B4BC3F8E40034
:10828000294A537C002B7ED0937C002B7BD19C46CB
:108290002D4BD2F8EC001B68D2F8E81007932B4B5B
:1082A00004901B68D2F810810693294BD2F8147100
:1082B0001B68D2F81841059392F82C31D2F81C6152
:1082C0000293107C9368D2F82051D2F824B1D2F8EE
:1082D0002821039101926246DFF86890194619F847
:1082E00002A0BAF1020F18D11A4951F82210B1F1C7
:1082F000FF3F0ED00546D0B202900398DDF810B0D3
:108300000190059E069FDDF81C804FF0010C0020B7
:1083100004E0002109F802101946234601322F2AF1
:108320001AD01C460B46D7E778020020940600209E
:10833000200C0020250C0020200B00200607002028
:10834000E80B0020380C0020F40600201407002061
:108350009C0600208C020020374A9160C2F8183138
:108360000199029B82F812C0C2F81081C2F8147100
:10837000C2F81C611074C2F82051C2F824B1C2F8CE
:10838000281182F82C312C4B93F83421092A06D17C
:1083900093F8D110022902D1033183F8D110264B72
:1083A000D3F83811002944D0092A42D193F8D120BA
:1083B000012A3ED19868002308E054F82340013395
:1083C000A04203D1052382F8D13032E01A4A8B4211
:1083D00002F59E74F1D32CE094F834314BB3042BA6
:1083E00027D0082B25D0062B23D0F3787168D4F83A
:1083F0003001124D43EA0123B0F5006F6A706B60E3
:1084000012D2314600F00EF93146D4F8300100F0B6
:1084100031F930B1D4F830310133C4F8303165234B
:1084200000E007232B7004E007232B70002384F85F
:10843000D1301BB0BDE8F08F780200200C0700207F
:1084400070B5044600200E46154603210246FCF78F
:108450003FFC0020C4F307210246FCF739FC002052
:10846000E1B20246FCF734FC002407E0944214BF5A
:1084700000220122FCF72CFC3055013400206A1E3A
:10848000AC420146F2D370BD10B504460020032172
:108490000246FCF71DFC0020C4F307210246FCF74E
:1084A00017FC0020E1B20246FCF712FC0020014656
:1084B0000122FCF70DFC10BD2DE9F04104460F46EA
:1084C0001646002006210122FCF702FC00200521AF
:1084D0000246FCF7FDFB002001220146FCF7F8FBF9
:1084E00010F0020FF2D0002002210246FCF7F0FB50
:1084F0000020C4F307210246FCF7EAFB0020E1B2AA
:108500000246FCF7E5FB002543E0013414F03F0888
:10851000795D01D1012204E0721E954214BF002250
:1085200001220020FCF7D4FBB8F1000F30D1731EFC
:108530009D422DD2002005210246FCF7C9FB0020F8
:1085400001220146FCF7C4FB10F00100F2D1062124
:108550000122FCF7BDFB002005210246FCF7B8FB19
:10856000002001220146FCF7B3FB10F0020FF2D00D
:10857000002002210246FCF7ABFB0020C4F30721D8
:108580000246FCF7A5FB0020E1B20246FCF7A0FB87
:108590000135B542B9D3002005210246FCF798FB0E
:1085A000002001220146FCF793FB10F0010FF2D1ED
:1085B000BDE8F08138B5012204460D4600200621B1
:1085C000FCF786FB002005210246FCF781FB00201A
:1085D00001220146FCF77CFB10F0020FF2D00020D4
:1085E00002210246FCF774FB0020C4F30721024677
:1085F000FCF76EFB0020E1B20246FCF769FB29465E
:1086000000200122FCF764FB002005210246FCF754
:108610005FFB002001220146FCF75AFB10F0010F1E
:10862000F2D138BD38B50725454305F500650C4640
:10863000284609780135FFF7BDFF284661780135E6
:10864000FFF7B8FF2846A1780135FFF7B3FF2846AA
:10865000E1780135FFF7AEFF284621790135FFF7B4
:10866000A9FF28466179FFF7A5FF681CA179FFF7EC
:10867000A1FF38BD2DE9F3470725454300200C46EF
:1086800002460321FCF724FB05F500650020C5F335
:1086900007210246FCF71CFB0020E9B20246FCF76A
:1086A00017FB002001460246FCF712FB8246002021
:1086B00001460246FCF70CFB8046002001460246BC
:1086C000FCF706FB0746002001460246FCF700FBCC
:1086D0008146002001460246FCF7FAFA06460020D1
:1086E00001460246FCF7F4FA054600200122014645
:1086F000FCF7EEFA237853451DD1637843451AD130
:10870000A378BB4217D1E37821798DF804608DF806
:1087100005508DF80600627943EA012343EA0243DB
:10872000A079019A43EA006049EA0229814514BF11
:108730000020012000E00020BDE8FC8738B54FF4A0
:108740000064002006210122FCF7C2FA0020052166
:108750000246FCF7BDFA002001220146FCF7B8FAF8
:1087600010F0020FF2D0002002210246FCF7B0FA0E
:108770000020C4F307210246FCF7AAFA0020E1B268
:108780000246FCF7A5FA002500203F2D14BF002269
:10879000012201460135FCF79BFA402DF4D100205F
:1087A00005210246FCF794FA002001220146FCF75D
:1087B0008FFA10F0010FF2D14034B4F5804FC0D1E0
:1087C00038BD00BF38B50725454300200C4602469A
:1087D0000321FCF77DFA05F500650020C5F30721AC
:1087E0000246FCF775FA0020E9B20246FCF770FA7F
:1087F000002001460246FCF76BFA2070002001467B
:108800000246FCF765FA6070002001460246FCF75C
:108810005FFAA070002001460246FCF759FAE070AA
:10882000002001460246FCF753FA20710020014661
:108830000246FCF74DFA6071002001460122FCF768
:1088400047FAA07138BD00BF37B5002005210246A8
:10885000FCF73EFA002001220146FCF739FA10F03D
:108860007104F2D100F0C6FD054605E0FFF70CFEED
:10887000422814BF0024012400F0BCFD431B002B40
:10888000B8BF5B42B3F5FA6F40F2FF7002DA002C1A
:10889000ECD000E01CB1234B1B78002B36D040F20B
:1088A000FF700021FFF786FEFFF748FF00201E49FA
:1088B0004022FFF701FE4FF480701C49B422FFF7FD
:1088C000FBFD40201A492022FFF7F6FD002301930B
:1088D0004FF4C36401AD2046042204342946FFF757
:1088E000EBFDB4F5FF6FF5D100230193A4F53074CF
:1088F0002046042204342946FFF7DEFDB4F5C36F99
:10890000F6D140F2FF704221FFF754FE00204022D2
:108910000549FFF795FD402006492022FFF790FD0D
:108920003EBD00BF5C0B0020080000204826010867
:1089300078260108C00B0020094B19685A6891423B
:1089400001D100200BE01A68D118097A01320170B8
:108950001A601A68202A01D100221A60012070478B
:10896000EC030020014B9862704700BFEC0300202D
:10897000034B1A78104612B100221A70012070477A
:10898000780C002008B5FBF787FD034B00221A6026
:108990005A60FBF77FFD08BDEC03002038B50B4B98
:1089A0008446DC6A1A6B0134202C08BF00249442F0
:1089B0000AD0DD6A0648ED1885F834C040F2277108
:1089C0000122DC6206F018FB38BD00BFEC0300207A
:1089D0000044004038B50546002401E0FFF7DEFF03
:1089E0002B5D01341846002BF8D138BD2A4910B54B
:1089F0000B8813F0200F1CD0284BDB6813F0020FFC
:108A000001D08B8815E0264B5A6818680132202A5D
:108A100008BF0022824205D05C688888E118C0B295
:108A200008725A601F4B0A221A601D4B9A6A1E4B2D
:108A30001A601948038813F0800F1BD01A4B1A686C
:108A4000C2B9174BDC6A196B8C420FD01349022450
:108A50000C61196BCC1894F834C00131A0F804C033
:108A60001963196B202905D11A6303E040F22771BD
:108A700006F0C2FA0848038813F0400F0BD040F20A
:108A8000266106F0B1FB064B1A6BDB6A9A4202D1F3
:108A9000024B02225A6110BD004400400008014010
:108AA000EC030020740C0020700C002030B505464B
:108AB00087B0564806F0E8FB4FF40030012105F07E
:108AC00031FA0420012105F01FFA0420002105F0ED
:108AD00037FA0820002104F09FFE06AC4FF0040393
:108AE00024F8083D03234A4821468DF812301533F7
:108AF0008DF8133004F000FE482345488DF81330FC
:108B000021464FF00803ADF8103004F0F5FD68463B
:108B100006F03CFA0B2D25D8DFE805F02406090CF9
:108B20000F1215181B1E20224FF461531CE04FF446
:108B3000964319E04FF4E14316E04FF4164313E077
:108B40004FF4614310E04FF496330DE04FF4E133FE
:108B50000AE04FF4613307E02E4B05E02E4B03E0B3
:108B60002E4B01E04FF416530093009B06A95B08BF
:108B700041F8183D2548694606F03EFB26230024AF
:108B8000012505A88DF8143007238DF815308DF8D0
:108B900016408DF8175004F01FFF1C4840F2FF31BB
:108BA00006F0FEFA28212246184806F025FA2A4641
:108BB000164840F2277106F01FFA2A46134840F281
:108BC000266106F019FA2A46104840F2255106F0AF
:108BD00013FA22460D4840F2244106F00DFA2246CF
:108BE0000A4840F6460106F007FA2246074840F6D2
:108BF0006A1106F001FA60212246044806F0FCF9E9
:108C00002946024806F0EAF907B030BD00440040AA
:108C10000008014090D0030020A1070040420F004F
:108C200030B50C4B0C4C844622681B689A4201D12B
:108C300000200EE02368094A5D1C02EB03130FCBF2
:108C40008CE80F0025602368082B01D100232360E6
:108C5000012030BD080D00207C0C0020880C002075
:108C6000704700BFF0B5437887B00646426833B11D
:108C700004238DF80C3000230292019303E001924B
:108C800002938DF80C30B37803B102238DF80D30C8
:108C9000327800238DF80E20F21801A8117AC2183C
:108CA0000133082BD172F7D103F068FF042818D1E3
:108CB0000D4D0E4B2C681B680134082C08BF002496
:108CC0009C4201D100200DE096E80F002F68084E6D
:108CD00006EB071C8CE80F00012001462C6003F016
:108CE0003FFF012007B0F0BD800C0020840C002065
:108CF0000C0D00207FB52B4B2B4A1968126891424E
:108D000004D10120002103F02BFF48E01968274A15
:108D100002EB0111487850B11B6802EB0312536853
:108D200004228DF80C2000220192029307E01B68B8
:108D3000029002EB031253688DF80C000193194B5B
:108D40001A681A4B03EB02139B781BB102238DF8B0
:108D50000D3001E08DF80D30124B00221968134BD5
:108D60000901CB5C8DF80E300E4B0DF1180C186814
:108D70000CEB020102EB001C0C4801326044007A4B
:108D8000082A01F8090CEFD11A6801321A601A6832
:108D9000082A01D100221A6001A803F0EFFE07B0F3
:108DA00000BD00BF840C0020800C00200C0D0020B2
:108DB00073B50220002103F0D3FE1020002103F040
:108DC000CFFE01AC0021012003F0CAFE00250726DA
:108DD000142320468DF804308DF805608DF8065078
:108DE0008DF8075004F0F8FD152320468DF8043067
:108DF0008DF805608DF806508DF8075004F0ECFDF5
:108E0000204613238DF804308DF805608DF8065048
:108E10008DF8075004F0E0FD04F0ACF829464FF05F
:108E2000007005F07FF87CBD2DE9F04101388AB073
:108E30000C46154607285BD8DFE800F04C40342884
:108E40001C5A10040C238DF81C3003238DF81D30A0
:108E500000238DF81B304FF0020354E00C238DF8F3
:108E60001C3003238DF81D3000238DF81B304FF08C
:108E700004023AE00C238DF81C3003238DF81D30DA
:108E800000238DF81B304FF010022EE00C238DF8DC
:108E90001C3003238DF81D3000238DF81B304FF05C
:108EA000140330E00C238DF81C3003238DF81D30A3
:108EB00000238DF81B304FF0280216E00C238DF8AC
:108EC0001C3003238DF81D3000238DF81B304FF02C
:108ED000640318E00C238DF81C3003238DF81D303B
:108EE00000238DF81B304FF0C802ADF81E200CE0B7
:108EF0000C238DF81C3003238DF81D3000238DF8D2
:108F00001B304FF00803ADF81E3004F033F8012198
:108F10004FF0007005F006F80120014604F0F4FF60
:108F20000820012104F0F0FF0820002105F008F8D6
:108F300001214FF4EA1004F06FFC0AAE4FF4007206
:108F400026F8042D032331468A488DF82630153340
:108F50008DF8273004F0D0FB0423314685488DF886
:108F600027304FF4807300260127ADF8243004F039
:108F7000C3FB05A88DF81A608DF814608DF8157084
:108F80008DF816608DF817608DF818708DF81970CF
:108F900003F0E4FCB4F5006F01A815DA4FF0FF32DE
:108FA0006301ADF80830ADF810608DF812708DF8DF
:108FB00004608DF805608DF80670ADF80A60ADF8B4
:108FC0000C20ADF80E2013E04FF0FF338DF8067043
:108FD000ADF810608DF812608DF804608DF80560B2
:108FE000ADF80860ADF80A60ADF80C30ADF80E30A1
:108FF00003F026FDDDB1B5F5006F18DA002201237C
:109000006901ADF80A208DF805204FF0FF3201A864
:10901000ADF808108DF812308DF804308DF8063058
:10902000ADF80C20ADF80E20ADF8103016E000239E
:109030000122ADF80A308DF812308DF80530ADF808
:1090400008304FF0FF3301A8ADF810208DF8042050
:109050008DF80620ADF80C30ADF80E3003F0F0FCC2
:10906000E30043F004030DF1040800270126022267
:109070006413ADF80A3040464FF0FF338DF80420FA
:10908000ADF808408DF805708DF80660ADF80C302D
:10909000ADF80E30ADF810708DF8126003F0D0FC12
:1090A000BD421ADDEB0043F004036D130322ADF85B
:1090B0000A304FF0FF3340468DF804208DF80570DC
:1090C000ADF808508DF812608DF80660ADF80C30E0
:1090D000ADF80E30ADF8106017E003238DF80430C2
:1090E0004FF004024FF0FF334046ADF80870ADF882
:1090F00010608DF812708DF805708DF80660ADF86F
:109100000A20ADF80C30ADF80E3008AF03F098FC33
:10911000012407260025142338468DF820308DF8C9
:1091200021608DF822508DF8234004F055FC152362
:1091300038468DF820308DF821608DF822508DF85A
:10914000234004F049FC132338468DF820308DF875
:1091500021608DF822508DF8234004F03DFC022060
:10916000214603F0FDFC2146102003F0F9FC0AB073
:10917000BDE8F081000C014030B52A4D2A4B2C6827
:109180001B680134082C08BF00249C4287B044D0DF
:10919000012001A903F0CEFD9DF80C20234B042AE9
:1091A00009D12A68012103EB021251702A6803EBEE
:1091B0000213029A08E02A68002103EB02125170A0
:1091C0002A6803EB0213019A5A609DF80D30154A84
:1091D000022B164B04D1126803EB0213012203E0A9
:1091E000126803EB021300229A700E4B9DF80E10CA
:1091F0001A680E4B1201D15400230A4A06A9C81856
:1092000011680A4D03EB011110F8090C01334919DB
:10921000082B0872F1D1146002E0012003F06EFD0A
:1092200007B030BD080D00207C0C0020880C002009
:1092300030B52A4D2A4B2C681B680134082C08BF16
:1092400000249C4287B044D0002001A903F072FDA5
:109250009DF80C20234B042A09D12A68012103EB35
:10926000021251702A6803EB0213029A08E02A687E
:10927000002103EB021251702A6803EB0213019ADA
:109280005A609DF80D30154A022B164B04D1126816
:1092900003EB0213012203E0126803EB0213002226
:1092A0009A700E4B9DF80E101A680E4B1201D15495
:1092B00000230A4A06A9C81811680A4D03EB0111D8
:1092C00010F8090C01334919082B0872F1D1146008
:1092D00002E0002003F012FD07B030BD080D0020B1
:1092E0007C0C0020880C0020F0B5384B1A787AB13D
:1092F0005968374A013159601168364B01311160A4
:109300001A6812B11A68013A1A6000222F4B00E065
:1093100001221A70304B1A683AB11A68013A1A6081
:109320001B6813B92D4B01221A702D4B2D4A9B8CB3
:109330002D499BB2136010680B68984218DD1468C1
:1093400008682A4B201AB0F5004F294806DAD3E9FD
:109350000045166809680268701A29E0D3E90045DB
:109360000E68116806F5803C0268C1EB0C0011E044
:1093700010680B68984223DA0C6810681B4B201A9F
:10938000B0F5004F1A480ADAD3E900450E681168B3
:109390000268701A5043261A65EBE0770CE0D3E9B7
:1093A00000451268096802F5803C0268C1EB0C00B8
:1093B0005043261845EBE07730463946C3E90001B3
:1093C000084B1A68084B1A60F0BD00BF400400202B
:1093D00008070020700C0020740C0020780C00207E
:1093E00000080040680C0020400B0020600B0020AB
:1093F000680B0020014B5868704700BF40040020F4
:1094000008B5042004F0B0FF48F6A04004F0BCFF0B
:10941000012004F0BFFF04480321002204F0AAFB4E
:10942000012004F0CDFF08BD9AC302000000000037
:109430000828F8B508D009280ED008B100205AE055
:109440003B4B188880B256E0394B588840F21323C2
:1094500080B2584300134EE0354B988880B208F034
:109460003DFB07F01FFF0022324B07F06FFF22A3E6
:10947000D3E9002306460F4607F068FF20A3D3E98F
:10948000002307F0B1FD1EA3D3E9002304460D46D7
:109490003046394607F05AFF1BA3D3E9002308F0F2
:1094A0007FF802460B462046294608F079F808F076
:1094B0000FFA07F0F7FE00221F4B08F071F807F0D3
:1094C00099F913A3D3E9002307F040FF12A3D3E9CE
:1094D000002307F089FD02460B4611A1D1E90001E6
:1094E00008F05EF810A3D3E9002307F07BFD08F035
:1094F000EFF908F011FDF8BD6666666666660AC09B
:109500006666666666660A409A99999999990140D5
:10951000C3F5285C8FA272400000000000FEAA4044
:109520009A999999FD6F2F41C3F5285C8F1271406C
:10953000480400200000303F00002440F0B593B004
:1095400011AF01240025032641483946ADF84440B7
:109550008DF846608DF8475004F0CEF84FF01103B7
:1095600039463C48ADF844308DF846608DF8475098
:1095700004F0C2F82046214604F0B8FC21464FF41E
:10958000007004F0C1FC344803F000FD334B324856
:109590000193334B01A9029380230693DB180793B1
:1095A00003F540730893A3F57873099303F5FF530C
:1095B0000A930395049605950B9503F057FD2648ED
:1095C000214603F083FD4FF4602326480CA90E9337
:1095D0008DF834400C958DF835400F958DF840602E
:1095E00002F0F0FF1F4808212246334603F06CF8D2
:1095F0001C4804210222334603F066F83346324603
:109600001848294603F060F82A4616484FF4FC61D2
:1096100003F01CF81348214603F00EF811482146C8
:1096200003F000F80F4803F01BF80E4803F01EF893
:109630000028FAD10B4803F01DF80A4803F020F87F
:109640000028FAD10748012103F01EF813B0F0BD3D
:10965000000C014000080140080002404C24014079
:109660004804002000240140014B03221A60704787
:1096700050040020044A054B927A0AB1052200E00A
:1096800001221A60704700BF980D0020500400208E
:10969000704700BF014B00225A6070475004002001
:1096A00008B5074B1A6892B242F008021A601A68AD
:1096B00092B242F004021A60FFF7D6FF08BD00BF65
:1096C000405C004010B5064C4FF6FB73226802EA7E
:1096D00003032360FFF7CEFF4FF40643236010BD62
:1096E000405C0040072818BF1F4B10B51E4C18BF28
:1096F00018702378052B33D8DFE803F003060A0E31
:109700001621FFF7DFFF2BE0FFF7DCFF042328E043
:1097100002236370013324E06378013BDBB26370A2
:109720006378FBB9042218E0104B1A6892B242F039
:1097300010021A6005232370DB18637012E063784F
:10974000013BDBB26370637863B9084A4FF6EF738D
:10975000116801EA030313600622034B1A7001E04B
:109760000623237010BD00BFFC0D0020405C0040AC
:10977000034B9B7A13B1034B05221A60704700BF5D
:10978000980D002050040020014B04221A607047FD
:1097900050040020034B1A7A202A01D100221A72A9
:1097A000704700BF50040020704700BF212808B553
:1097B00008D1124B1B681B7803F07F03212B1AD1B1
:1097C0000F4B0EE0202816D10C4B0E4A1B681B785D
:1097D00010720D4A03F07F03212B0CBF13460023A8
:1097E0004BB1064A4FF0000112680020518293618C
:1097F0009847002000E0022008BD00BFF80D0020BF
:1098000041980008500400205D980008074B1B6831
:109810001B7803F07F03212B05D1022801D02228D9
:1098200001D1002000E00220704700BFF80D0020A9
:1098300019B9012801D8084600E00220704700BF8E
:1098400028B9044B4FF008021B681A8200E0024856
:10985000704700BFF80D00204800002028B9044BD5
:109860004FF008021B681A8200E00248704700BFF0
:10987000F80D0020480000200B4B10B5DA6882B1CB
:109880001B68052B01D000220BE0002303E00749F1
:10989000595CC15401330449CC68A342F7D3002377
:1098A000CB60104610BD00BF50040020000E002009
:1098B000084BDB68082B01D800200AE00023064A89
:1098C0009A5CC2540133092BF9D1024B0022DA60B1
:1098D0000120704750040020000E002010B5074CF6
:1098E0000B468AB2C021636006F0AAFA0120A18863
:1098F00006F0B4FC012006F07FFB10BD50040020F0
:1099000007B5142200238DF8042001A801228DF848
:1099100006308DF807208DF8053004F05DF80EBD97
:1099200007B5142200238DF8042001A801228DF828
:1099300006308DF807208DF8053004F04DF80EBD87
:1099400008B5064B1B68DB78042B01D9002004E026
:10995000034901EBC30105F01BFE08BDF80D002013
:109960005000002008B5024905F012FE08BD00BFF6
:109970007000002008B5024905F00AFE08BD00BFCE
:1099800078000020334B10B51B686FF03F020024B5
:109990005A72DC729C72204606F0A6FA20464FF4FA
:1099A000007106F0BFFA1021204606F0D1FA4021DE
:1099B000204606F027FC8021204606F013FC2046B6
:1099C00006F050FB244B204693F8641006F068FC28
:1099D000204606F01FFB0120214606F0A3FA0120D5
:1099E000C02106F0FFFB0120202106F0B1FA012082
:1099F000214606F0C5FA02204FF4C06106F092FA43
:109A000002204FF4807106F0EDFB0220214606F0A3
:109A1000B7FA0220202106F09BFA0320214606F027
:109A200081FA03204FF4887106F0ECFB03204021FB
:109A300006F036FC03204FF4405106F0A1FA21460F
:109A4000032006F085FA204605F0B0FD034B012205
:109A50001A6010BDF80D00204800002050040020BE
:109A600008B5174B174A196889B211801649128830
:109A7000098801EA020212F4806F05D04FF6FF3226
:109A80001A60124BDB6B98470E4B1A880E4B1B88E3
:109A900003EA020212F4007F08D009490C4A4FF68B
:109AA000FF500860117C0131C9B21174054A128857
:109AB000134013F4004F01D006F0FEF808BD00BFBC
:109AC000445C00408E0D0020400E00204800002025
:109AD0005004002010B5032006F012FC064C03468B
:109AE00002464FF488710548E36006F0C1F903208F
:109AF00006F090FA10BD00BF50040020000E0020B8
:109B000008B500B10120FAF785FF08BD38B5064D4C
:109B100001232B60054B002420461C60FFF7F0FF5B
:109B200003232B60204638BD405C0040445C00406D
:109B300008B5FFF7EBFF08BD08B50120FFF7E0FF10
:109B4000064B0121196006494FF4E0520A8005498D
:109B50000020186008601A6008BD00BF405C00402B
:109B6000400E0020445C0040084B10B51B680024E8
:109B70009C72FFF7E1FF064A4FF406431460043A73
:109B80001360044A1460044A138010BDF80D0020CD
:109B9000445C004050040020400E0020002008B526
:109BA00004F028F94FF40000012104F0BBF908BDCE
:109BB00008B5FFF7F3FFFFF7B3FE06F01FF808BD87
:109BC000704700BF704700BF704700BF704700BFBD
:109BD000704700BF704700BF704700BF704700BFAD
:109BE00008B5FAF75BFD052805D9FAF757FD40F2ED
:109BF000F933984201D9012200E00022094B5A6052
:109C0000094B1B786BB1074B08495A68084B0A602F
:109C10001AB91A6842F0080202E01A6822F0080233
:109C20001A6008BD0C07002006070020F40600207B
:109C30009C06002010B5FFF7DDFB074C2368C31A14
:109C4000B3F5FA7F07D9054BDA6882F00402DA60CF
:109C5000FFF7D0FB206010BD440E0020000C014037
:109C6000024B03EBC003D879704700BF64040020A7
:109C7000024B03EBC0035879704700BF6404002017
:109C8000024B03EBC0039879704700BF64040020C7
:109C9000024B0B2202FB0033187A70476404002049
:109CA000024B0B2202FB0033587A704764040020F9
:109CB000024B0B2202FB0033D87A70476404002069
:109CC000024B0B2202FB0033987A70476404002099
:109CD000024B0B2202FB0033187B70476404002008
:109CE000024B0B2202FB0033587B704764040020B8
:109CF000024B0B2202FB0033987B70476404002068
:109D0000024B0B2202FB0033187C704764040020D6
:109D1000024B0B2202FB0033587C70476404002086
:109D2000024B0B2202FB0033987C70476404002036
:109D3000024B052202FB0033187D704764040020AB
:109D4000024B052202FB0033587D7047640400205B
:109D5000024B052202FB0033987D7047640400200B
:109D6000024B052202FB0033D87D704764040020BB
:109D7000024B052202FB0033187E7047640400206A
:109D8000024B032202FB0033187F7047640400205B
:109D9000034B032202FB003393F91D00704700BF01
:109DA00064040020024B032202FB0033987F7047BB
:109DB00064040020024B03EBC00393F820007047BB
:109DC00064040020024B03EBC00393F821007047AA
:109DD00064040020024B03EBC00393F82200704799
:109DE00064040020024B03EBC00393F82300704788
:109DF00064040020024B03EBC00393F82400704777
:109E000064040020024B03EBC00393F82500704765
:109E100064040020024B03EBC00393F82600704754
:109E200064040020024B03EBC00393F82700704743
:109E30006404002006281AD8DFE800F004070A0DA1
:109E4000101316000A4B9B6A10E0094BDB6A0DE009
:109E5000074B1B6B0AE0064B5B6B07E0044B9B6BED
:109E600004E0034BDB6B01E0014BDB7B0B607047D5
:109E70006404002070B5C0F30741054600220120AC
:109E8000FAF726FF0A4C0602C5F30721002201203B
:109E9000A662FAF71DFF064301203602E9B2024628
:109EA000A662FAF715FF06433609A66270BD00BF29
:109EB000640400202D4B032202FB003310B51C3339
:109EC00093F901203F2A01DD3F225A70274B0322DC
:109ED00002FB00331C3393F9012012F13F0FBCBF8A
:109EE0006FF03E025A70214B032202FB00331C33F9
:109EF0009A781F2A01D91F229A701C4B032202FB59
:109F000000324FF440211964127F012A04BF4FF43C
:109F100050221A64154B03EBC00292F827203AB97D
:109F2000033202FB0032527F196C02F07F020BE019
:109F3000032101FB003191F81DC002F003020CF077
:109F40007C0C196C4CEA0202084C41EA02221A64A9
:109F5000032303FB0040236C827F42EA030318467D
:109F60002364FFF787FF236CA36310BD6404002004
:109F700008B5044B032202FB00339977FFF79AFFE1
:109F800008BD00BF6404002008B5044B032202FB97
:109F900000335977FFF78EFF08BD00BF640400202F
:109FA00008B5044B032202FB00331977FFF782FF49
:109FB00008BD00BF64040020264B052210B502FB3B
:109FC00000331A7D012A01D901221A75214B05227D
:109FD00002FB003314335A78032A01D903225A7042
:109FE0001C4B052202FB003314339A780F2A01D947
:109FF0000F229A70174B052202FB00331433DA78D4
:10A00000032A01D90322DA70124B052202FB003326
:10A0100014331A790F2A01D90F221A710D4C052316
:10A0200003FB004000F114021379017D43F4202367
:10A03000507843EAC133917843EA4033D27843EA17
:10A04000012343EA421318462364FFF713FF236CEE
:10A05000636310BD6404002008B5044B052202FBB5
:10A0600000331976FFF7A8FF08BD00BF6404002085
:10A0700008B5044B052202FB0033D975FFF79CFF9E
:10A0800008BD00BF6404002008B5044B052202FB94
:10A0900000339975FFF790FF08BD00BF64040020EE
:10A0A00008B5044B052202FB00335975FFF784FF06
:10A0B00008BD00BF6404002008B5044B052202FB64
:10A0C00000331975FFF778FF08BD00BF6404002056
:10A0D000514B0B2210B502FB00331A7A032A01D927
:10A0E00003221A724C4B0B2202FB003308339A787E
:10A0F000032A01D903229A70474B0B2202FB00333B
:10A1000008331A790F2A01D90F221A71424B0B22F8
:10A1100002FB003308335A79072A01D907225A7102
:10A120003D4B0B2202FB003308339A790F2A01D9E9
:10A130000F229A71384B0B2202FB003310335A78EE
:10A140000F2A01D90F225A70334B0B2202FB003326
:10A1500010339A780F2A01D90F229A702E4B0B22B6
:10A1600002FB0032117AC90341F400241C64527AC4
:10A1700012B141F404211964274B0B2101FB00317A
:10A18000C97A19B1196C41F400511964224B8AB98A
:10A190000B3202FB0032083292F804C091784FEA89
:10A1A000CC1C1C6C4CEAC12C51794CEA040242EAEA
:10A1B00001121DE00B2202FB0032127C1AB11A6C54
:10A1C00042F480521A64144B0B2101FB0031103110
:10A1D00091F801E01A6C897842EACE1201F0070C7E
:10A1E00042EA0C1211F0080F1A6402D042F4006225
:10A1F0001A64094B0B2202FB00300830C27922B9E5
:10A2000081791A6C41EA02021A64034C206CFFF750
:10A2100031FE236C236310BD6404002008B5064B97
:10A220000B2202FB00330833DA791AB10022DA710B
:10A23000FFF74EFF08BD00BF6404002008B5064BC1
:10A240000B2202FB00330833DA791AB90132DA71D2
:10A25000FFF73EFF08BD00BF6404002008B5044BB3
:10A260000B2202FB00339974FFF732FF08BD00BFD9
:10A270006404002008B5044B0B2202FB0033597420
:10A28000FFF726FF08BD00BF6404002008B5044B9B
:10A290000B2202FB00331974FFF71AFF08BD00BF41
:10A2A0006404002008B5044B0B2202FB00339973B1
:10A2B000FFF70EFF08BD00BF6404002008B5044B83
:10A2C0000B2202FB00335973FFF702FF08BD00BFEA
:10A2D0006404002008B5044B0B2202FB0033197301
:10A2E000FFF7F6FE08BD00BF6404002008B5044B6C
:10A2F0000B2202FB00339972FFF7EAFE08BD00BF94
:10A300006404002008B5044B0B2202FB0033D97211
:10A31000FFF7DEFE08BD00BF6404002008B5044B53
:10A320000B2202FB00335972FFF7D2FE08BD00BFBB
:10A330006404002008B5044B0B2202FB00331972A1
:10A34000FFF7C6FE08BD00BF6404002010B5254B12
:10A350004FF460221A6403EBC00292F8272012B176
:10A360004FF470221A641F4B03EBC00292F82110C5
:10A3700092F820C01C6C090341EA8C312143196416
:10A3800092F82220012A04BF41F480611964154B20
:10A3900003EBC00191F823C01A6C42EA0C221A6444
:10A3A00091F82410012904BF42F080021A640D4B79
:10A3B00003EBC00292F82520012A03D11A6C42F067
:10A3C00040021A64074C04EBC00090F82620236C6E
:10A3D00043EA021318462364FFF74CFD236CE36342
:10A3E00010BD00BF6404002008B5044B03EBC0039C
:10A3F00083F82610FFF7AAFF08BD00BF6404002001
:10A4000070B50F4B064603EBC00393F82650032D9F
:10A4100002D00321FFF7E8FF3046FFF797FF084B14
:10A420009C6A14F4002F1CBF6FEA04346FEA1434E2
:10A43000032D03D030462946FFF7D6FF204670BDD6
:10A440006404002008B5044B03EBC00383F8251017
:10A45000FFF77CFF08BD00BF6404002008B5044B73
:10A4600003EBC00383F82410FFF770FF08BD00BFA3
:10A470006404002008B5044B03EBC00383F82310E9
:10A48000FFF764FF08BD00BF6404002008B5044B5B
:10A4900003EBC00383F82210FFF758FF08BD00BF8D
:10A4A0006404002008B5044B03EBC00383F82110BB
:10A4B000FFF74CFF08BD00BF6404002008B5044B43
:10A4C00003EBC00383F82010FFF740FF08BD00BF77
:10A4D00064040020064B10B503EBC003044683F868
:10A4E0002710FFF733FF2046FFF7E4FC10BD00BF45
:10A4F0006404002010B5144B00221A6403EBC00260
:10A50000527912B14FF400721A640F4B03EBC00280
:10A5100092791AB11A6C42F480721A640A4B03EBF6
:10A52000C003DA790F2A01D90F22DA71064C04EB45
:10A53000C000C279236C42EA030318462364FFF784
:10A5400099FC236CE36210BD6404002070B5084DD3
:10A550009DF810E09DF8146005EBC0042671627050
:10A56000A37084F803E005F83010FFF7C3FF70BD57
:10A570006404002008B5034B03EBC0039971FFF797
:10A58000B9FF08BD6404002008B5054B03EBC00308
:10A59000597109B10422DA71FFF7ACFF08BD00BFA1
:10A5A0006404002008B5054B042903EBC003D971EE
:10A5B00001D000225A71FFF79DFF08BD64040020FE
:10A5C0002DE9F047344D0446401990F844000E46FA
:10A5D00017469846DDF82090DDF824A004281FD8FF
:10A5E000DFE800F003090F151B002046FFF770FDA0
:10A5F0006519012316E02046FFF7A8FE651902231E
:10A6000010E02046FFF7D8FC651903230AE0204636
:10A61000FFF750FC6519042304E02046FFF76AFFAA
:10A620006519002385F844301B4B03EBC40494F8F0
:10A630002620012A0DD002D3022A23D111E016B11F
:10A640009B6A9B0C3370EFB1134B9B6A9B0A3B7068
:10A6500018E0B8F1000F15D09B6A9B0AC8F80030CB
:10A6600010E0B8F1000F04D09B6ADB0B5B01C8F867
:10A670000030B9F1000F05D0074B9B6AC3F3842368
:10A6800089F80030BAF1000F03D0034B9B6A8AF8B7
:10A690000030BDE8F08700BF64040020214B10B5F6
:10A6A000032200244FF0050C02214FF0010E83F825
:10A6B00025E0197383F80EC09A745C7483F81CE06B
:10A6C00083F81DC083F81EC083F8202083F8212062
:10A6D00083F8224083F8234083F8244083F826102F
:10A6E00083F827401C755C759C75DC751C765C7165
:10A6F0009C71DC7119725C72DC729C725A73DC732F
:10A700001C742046FFF758FC2046FFF7D3FB204679
:10A71000FFF71CFE2046FFF7EDFE2046FFF7D8FCB2
:10A7200010BD00BF6404002008B5044A0023917ADC
:10A73000034A18461370FAF7B5F908BDC00B00209C
:10A74000280C00202DE9FF417E4B1A7822B90132F6
:10A750001A706FF000425A607A4B1C7A5CB9E0B212
:10A76000F9F764FF774B03F10C0210550134082C04
:10A77000F5D101221A7227240025E8B2F9F756FF15
:10A78000714A535D834219D0704B291D53F8213013
:10A790005055022B05D0032B0AD0012B0ED168B1E6
:10A7A00006E058B96A4A115D012907D1135505E041
:10A7B000674B1A5D012A01D101321A550135013466
:10A7C000082DDAD1634EF36993B1634C25787DB9D6
:10A7D000FEF710FE614AF3691268821A002AB8BFB8
:10A7E00052429A4204D9284601F092FA012323707A
:10A7F000584E336A93B15A4C25787DB9FEF7FAFD6D
:10A80000584A336A1268821A002AB8BF52429A42E2
:10A8100004D9284601F07CFA01232370494C524D9B
:10A82000207D830005EBC302127B002A00F0298102
:10A830004E4A4F4F4F4E0021D3183F1836180A4644
:10A8400000970196FFF7BCFE237D05EB43152A7B9D
:10A85000013A042A00F20481DFE812F005004E00FC
:10A86000D2004E00D200444A364D926812F4004F96
:10A870001BD05D192A7E022A04D1404AD25C002AEC
:10A8800000F0EE80384A2F4C02EB43121846517A02
:10A89000FAF708F9207DFFF7C1FC237D374A002134
:10A8A000E418D15402232376DAE05D192A7E012AC6
:10A8B00004D1324AD25C002A00F0D2802A4C1846D9
:10A8C00004EB4313997AFAF7EDF81E4B187D04EB6D
:10A8D0004014A37A13B9FFF7B1FC04E0274B1B5CCB
:10A8E0000BB1FFF79BFC174A2449137D0020D218B7
:10A8F000C85401231376B3E01E4A124DD256002AE3
:10A900003EDB5D192A7E022A02D11C4AD25C8AB142
:10A91000154A0C4C02EB43121846517AFAF7C2F86A
:10A92000207DFFF77BFC237D144A0021E418D154DD
:10A9300002232376034C257DFEF75CFD04EB8504A2
:10A94000606055E0AC040020B8040020E80B002053
:10A95000380C002008000020250C0020200C0020CE
:10A96000210B0020180C0020C00B0020580B0020E9
:10A970002C0B0020B80B002000080140240C002004
:10A980005B191B7E012B11D0FEF734FD2B7D8E4A07
:10A9900005EB830502EB43139B8B0A2253436A6842
:10A9A000821A002AB8BF52429A4204DC874B884A76
:10A9B0001B7DD35CE3B1854D834C287D04EB4013B4
:10A9C000997AFAF76FF8287D04EB4014A37A13B94B
:10A9D000FFF734FC04E07E4B1B5C0BB1FFF71EFC61
:10A9E0007A4A7B49137D0020D218C854012313767C
:10A9F000764B1A7D744B03EB42131B7B042B20E038
:10AA0000724A9A18127E022A02D1714AD25C8AB125
:10AA10006D4A6E4C02EB43121846517AFAF742F82F
:10AA2000207DFFF7FBFB237D694A0021E418D15408
:10AA300002232376654B1A7D634B03EB42131B7B8A
:10AA4000052B0DD1634B9B6813F4004F04D0624B70
:10AA50004FF400425A6103E05F4B4FF400421A6129
:10AA6000FEF7C8FC594CE369C31A002BB8BF5B4220
:10AA70000A2B40F37083F9F783FEFEF7BBFCE0611D
:10AA800069E3F9F77DFEFEF7B5FCE369C31A002B15
:10AA9000B8BF5B420A2B05DC4E4B9B6813F4806FFA
:10AAA00040F05983494D0020297D490141F00A01B8
:10AAB00001F0EA0100F0EEFF0446287D01F04CF9B8
:10AAC0002B7D0C20584345494218157A0DB1455845
:10AAD00000E05568424AD25C032A00F2E780DFE8D2
:10AAE00002F002831C4B002C00F0E080364A374D08
:10AAF00002EB4311C97F3A4E29B11846F9F7D2FF4C
:10AB00002B7D032207E002EB43121846517AF9F736
:10AB1000C9FF2B7D0222F254C8E04CB95B0143F01F
:10AB2000080101F0E801204600F0B4FF002865D0DC
:10AB3000264E254B307D03EB4013D97F002900F0D2
:10AB4000AE80002D84EAE472B8BF6D42A2EBE472DD
:10AB5000AA4202D0002C40F09C80224B53F83010C7
:10AB60008A4280F09C8003EBC0031979F9F79AFFC1
:10AB7000164B01211B7D90E0002D84EAE471B8BFE3
:10AB80006D42A1EBE471A94202D0002C40F0878015
:10AB9000144A0E4D52F83300114E814208D202EB96
:10ABA000C30218461179F9F77DFF2B7D012208E0D9
:10ABB000054A184602EB4313597AF9F773FF2B7DC8
:10ABC0000222F2546BE000BFC00B0020AC04002056
:10ABD000240C002000080140001001406C0B0020F4
:10ABE000280C0020300B002044BB5B0143F008011F
:10ABF00001F0E801204600F04DFFF8B9FEF7FAFB3E
:10AC00001F4D204A2B7D4FF00A0E02EB4311B1F885
:10AC10001CC099004E1976680EFB0CFC861B002E9A
:10AC2000B8BF7642664541DD02EBC1021846917A13
:10AC3000F9F738FF2B7D144AD45437E0104E114AEF
:10AC4000337D02EB4312D17F49B3002D84EAE472D5
:10AC5000B8BF6D42A2EBE472AA4200D0C4B90B495E
:10AC600051F833108A421AD3064A184602EB4313AE
:10AC7000597AF9F717FF024B02211B7D0DE000BF47
:10AC8000AC040020C00B0020280C0020300B00205A
:10AC90001846F9F707FF337D0321A34AD154A34D8A
:10ACA0002E7DFEF7A7FB05EB860568609F4DA04F44
:10ACB0002B7DA04E1846F618FF189F4B002103EB82
:10ACC00080030A46019600979C4EFFF779FC287D89
:10ACD00006EB40139B6943B3F9F7D2FB28B3287DF9
:10ACE00084EAE47206EB40139B69A2EBE4729A4299
:10ACF0001BD901F00DF82A7D914906EB42139B7F89
:10AD00000120885443B1B27F9A4205D1013800F046
:10AD1000FFFF002000F03AFA844B8A4A1B7D0F3374
:10AD2000D15C012901D10131D154804D2B7D022B01
:10AD300025D8002000F08AFD95F8203010F0010F92
:10AD400003F0F80385F820301CBF43F0010385F8B9
:10AD5000203010F0040F8DF80C0006D0734B93F8E0
:10AD6000202042F0020283F8202010F0100F06D0BD
:10AD70006E4B93F8202042F0040283F82020724AA0
:10AD8000137853B1694991F820100B4205D16F49EE
:10AD90006F480978037001B911706D4B1B784BB186
:10ADA000624A92F8202003EA02029A4202D1694BD9
:10ADB00001221A705D4B93F8202012F0010F0AD087
:10ADC00093F8213013F0010F05D15E4BDA78012A98
:10ADD00001D10132DA70554B93F8202012F0020FA6
:10ADE0000AD093F8213013F0020F05D1554B1A7990
:10ADF000012A01D101321A714C4B93F8202012F034
:10AE0000040F0AD093F8213013F0040F05D14D4BF5
:10AE10005A79012A01D101325A71444D03222B7D06
:10AE200004A8B3FBF2F2821812F9042C95F8201052
:10AE3000002A85F821104ADA5B0143F01601002050
:10AE400001F0F60102AA00F03DFE9DF80A3013F071
:10AE5000400F08D02A7D3B4952001B32885C0128F4
:10AE600001D10130885413F0800F0AD02F49354AA0
:10AE7000097D0E3112F81100012802D1013002F8CB
:10AE8000110013F0100F09D0284A2E49127D5200EC
:10AE90001B32885C012801D10130885413F0200F47
:10AEA0000AD0224A274B127D0E3213F812100129C4
:10AEB00002D1013103F812101C4B0020197D02AAA7
:10AEC000490141F0160101F0F60100F097FF174F1C
:10AED0001A4E3B7D06EB43125269002A00F0818036
:10AEE0001D4AD55C002D7CD1002C7AD05B0143F04B
:10AEF000020101F0E201284600F092FD8046387D13
:10AF0000F9F736FD397DC0EB080806EB41135B69A4
:10AF1000B8F1000F83EAE372B8BFC8F10008A2EBF2
:10AF2000E37290455DDD19E0280C0020AC040020A0
:10AF30002C0B0020B80B0020580B0020C00B002069
:10AF4000B40B0020380C0020540B0020280B0020EC
:10AF5000440B00206C0C00203C0B0020002B0EDD6D
:10AF6000084600F0D5FE3B7D06EB43139B7F3BB3C9
:10AF7000B27F9A4224D1284600F0CAFE1DE028463E
:10AF8000022200F027FD397D2846490141F00801E1
:10AF900001F0E80100F09EFE3B7D06EB43139B7F32
:10AFA00073B1B27F9A420BD129462846022200F0A3
:10AFB00011FD2846082100F08DFE284600F0E6F835
:10AFC000664B674A1B7D1533D15C012901D10131E4
:10AFD000D154624B634A1B7D01211846D15400F0C5
:10AFE000D5F8614F3B68002B47D05C4E5D4A337DFE
:10AFF000D55C002D41D1002C40D05B0143F0020113
:10B0000001F0E201284600F00BFD8046307DF9F7A3
:10B0100055FA3B68C0EB0808B8F1000F83EAE37209
:10B02000B8BFC8F10008A2EBE372904531DD002BF8
:10B03000317D03DD084600F06BFE0CE0284602225D
:10B0400000F0C8FC317D2846490141F0080101F0BB
:10B05000E80100F03FFE414B414A1B7D1533D15CB6
:10B06000012901D10131D1543C4B3E4A1B7D0121C4
:10B070001846D15400F08AF80BE054B9374B002041
:10B08000197D490141F0080101F0E80100F002FDDD
:10B0900020B1324D354B2E7D9B5D43B32F4B344A4F
:10B0A0001B7D02EB4312D28912B9304AD35C1BB329
:10B0B000FEF7A0F9294D2E492B7D4FF00A0C9A007E
:10B0C00001EBC201C9895219526A0CFB01F1821AC3
:10B0D000002AB8BF52428A420EDD264EF25C5AB9AF
:10B0E0001846FFF7ABF82B7D0122F25404E0FEF77F
:10B0F00081F905EB86056862184E1F4D307D002CE6
:10B1000055F83030B8BF64429C420AD2FEF730FE98
:10B11000337D05EBC3056A7982420DD118460021C3
:10B1200008E0FEF725FE337D05EBC305697988420B
:10B1300002D01846FEF790FF084C207D00F034F84E
:10B14000237D0133DBB223750BB100232375FEF79A
:10B1500051F9024BD861BDE8FF8100BFAC0400206B
:10B16000380C00203C0B00204C0B0020300C002041
:10B17000C00B0020340C0020300B0020024B1A5C66
:10B180000AB901321A547047D4040020024B1A5CE9
:10B190000AB10F221A547047D4040020014B185CE6
:10B1A000704700BFD40400202DE9F3474601F5B2F3
:10B1B000044645F07C01002001AA00F083FCB74A58
:10B1C000610002EB4413187A06EB020710F0400FFF
:10B1D0009DF8063012D04FF001084FF0020C08FA2B
:10B1E00001F80CFA01FCB1587E680CEA030208EA87
:10B1F0000307C1F10009C6F1000A0FE04FF0010C8E
:10B200004FF002080CFA01FC08FA01F156F802901E
:10B21000D7F804A00CEA030201EA030710F0800F3C
:10B2200000F03F0606D09E4B9B6883F40048C8F3AD
:10B23000C03803E09A4B9B68C3F3C038731E072BDA
:10B2400000F2D182DFE813F00800080008000800CF
:10B250006E016E016E016E01924B1B5D013B0E2B68
:10B2600000F2C182DFE813F00F003D0053006200DE
:10B270007A0082008E00A000D10014012401BF02D8
:10B2800043014E01A60201AA45F014010020854F9A
:10B2900000F018FC9DF8053045F0060507EB840822
:10B2A000C8F804302946002000F0F4FB0222C8F858
:10B2B00008002146002000F08DFB023E00202946B8
:10B2C00040F2FF7200F0F2FCF6B2002003222146A9
:10B2D00000F05AFB012E01D8022300E004233B5565
:10B2E00081E2704E002006EB84035A68214602F08A
:10B2F0000402824214BF0522012200F045FB45F002
:10B3000008014A46002000F0D1FC032324E0002A73
:10B3100000F0698245F00201002000F081FB614BE2
:10B3200004221A55604B43F824005CE25D4E002075
:10B3300006EB84035A68214602F00402824214BFDD
:10B340000622022200F020FB45F00801C9F10002AC
:10B35000002000F0ABFC0523335544E2002F00F041
:10B360004282204600F0D4FC06222FE20020214633
:10B37000032200F009FB45F008015246002000F0CE
:10B3800095FC68E1002F40F02E8245F008053A4612
:10B390003846294600F08AFCCAF1000238462946A0
:10B3A00000F084FC082211E2002F00F01C8245F01E
:10B3B0000201002000F034FB06460020024645F062
:10B3C000080100F073FC384B002053F8247021462C
:10B3D000BF1B43F82470032200F0D6FA8AEAEA720F
:10B3E00045F00601A2EBEA72002000F05FFC61016B
:10B3F00001F0E0013246002000F0C4FB00200246CC
:10B40000214600F0E7FA0922E0E1002000F01EFAF0
:10B41000630050FA03F313F0010F00F0E48145F0EC
:10B4200002073946002000F0FBFA204B45F00805E2
:10B4300043F8240000200246294600F037FC002093
:10B440000222214600F0C6FA00200246394600F0EA
:10B4500099FB00206101024601F0E001033E00F08B
:10B4600091FBF6B200212046F9F758FA012E0D4E55
:10B470000CD800202146022200F0ACFA2946CAF17D
:10B480000002002000F012FC0A2365E70E2363E7A8
:10B49000002F00F0A8810B2298E100BFC00B002014
:10B4A00000080140D4040020240B0020E40B0020FD
:10B4B000002F40F0988145F00201384600F0B0FAC4
:10B4C00045F0080106463A46384600F0EFFB6101B8
:10B4D000022296FBF2F201F0E001384600F052FB46
:10B4E0003A463846214600F075FA0D226EE10020FA
:10B4F00000F0ACF9630050FA03F313F0010F00F011
:10B50000728162E1A84E45F0060106EB8405002039
:10B51000AA6800F0CBFB2A790020214600F034FA1B
:10B52000002319E7A04B1B5D013B0E2B00F25B8152
:10B53000DFE813F00F00340052006200810059016F
:10B54000930059015901CC00DC00AD0008014F0106
:10B55000400145F0140101AA0020934F00F0B2FA17
:10B560009DF805C007EB840300200222C3F804C045
:10B57000214600F02FFA002045F0060140F2FF724C
:10B5800000F094FB00200322214600F0FDF9062E76
:10B5900002D0082E7FF4A2AE022217E1062E0CD1B3
:10B5A000814B002003EB84035A68214602F0040219
:10B5B000824214BF0522012204E0082E04D100209B
:10B5C0002146032200F0E0F94A4645F00801002038
:10B5D00000F06CFB0322F9E0731FDBB2012B05D8EE
:10B5E00022B1062E704E30D10423B5E6B8F1000F1B
:10B5F00000F0F9800C22E9E0052E0CD16A4B002006
:10B6000003EB84035A68214602F00402824214BF0D
:10B610000622022204E0072E04D100202146032244
:10B6200000F0B2F9C9F1000245F00801002000F075
:10B630003DFB0522CAE0731FDBB2012B07D837B1EF
:10B64000052E594E01D1022386E60F2384E6B8F178
:10B65000000F00F0C8800722B8E0B8F1000F40F0FA
:10B66000C280073EF6B2012E0DD94F4B404603EB88
:10B6700084035A68214602F00402002A14BF0522FE
:10B68000012200F081F945F00801524619E0B8F1B5
:10B69000000F40F0A880073EF6B2012E0DD9424BB4
:10B6A000404603EB84035A68214602F00402002A54
:10B6B00014BF0622022200F067F945F00801CAF122
:10B6C0000002002000F0F2FA0A227FE0B8F1000F39
:10B6D00000F0898045F00201002000F0A1F9324B12
:10B6E0000B2103EB84021955D0607CE0B8F1000F08
:10B6F00079D145F00201404600F092F92B4BA700AA
:10B70000294E03EBC7038AEAEA72814645F0060137
:10B71000A2EBEA72404683F80D80BF1900F032FABE
:10B72000FB6861019944022399FBF3F201F0E00107
:10B73000404600F027FA40462146424600F04AF9CA
:10B740000D2309E6002000F081F8630050FA03F3AE
:10B7500013F0010F47D0144B0E2245F002061A5584
:10B760003146002000F05CF9114B45F0080143F828
:10B7700024000020024600F099FA2146002002220F
:10B7800000F028F900203146024600F0FBF90020C5
:10B790006101024601F0E00100F0F4F920460021C9
:10B7A000F9F7BCF81FE000BFD4040020C00B002054
:10B7B000E40B002000202146022200F00BF90020BB
:10B7C00045F00801024600F071FA0E22074B1A55A7
:10B7D00009E0064D002005EB84031A79214600F0AC
:10B7E000D3F800232B55BDE8FC8700BFD40400200C
:10B7F000154B10B503EB0012926891420EDD8A1AC8
:10B80000C2F18074A2424FEA001C03DC63445C680E
:10B8100012190EE063445A68141B0FE00FDA521A33
:10B82000C2F18074A2424FEA001C04DC63445C68ED
:10B83000A21A5A6003E063445A68A4185C60024B81
:10B8400003EB0010816010BD480E0020012108B5F7
:10B8500002200A46F9F73CFA08BD00BFF8B5137894
:10B86000144613F0600F06460D4627D1414A127B5D
:10B8700022BB13F0010F21D15F2B1FD83E4A127853
:10B88000E2B913F09F0301D0082B17D13B4F387852
:10B8900060B9384BD97F19B1F9F704F9032304E0F3
:10B8A0000846597AF9F7FEF802233B70344F3B788B
:10B8B00023B10020FEF7B2FC00233B700022217868
:10B8C0000220F9F705FA2870002261780220F9F7C2
:10B8D000FFF968700022A1780220F9F7F9F9A87041
:10B8E00001220220E178F9F7F3F9E870237813F0E8
:10B8F000010F3ED15F2B3CD803F01E02082A04D072
:10B90000142A2CD0062A34D11BE0242171435B0970
:10B910000C2000FB0313A57894F803C0194A4CEAE5
:10B9200005259D50A37813F0080F22D026787609BC
:10B9300000FB0616B3586FEA03536FEA1353B35074
:10B9400017E0242256435B090C22A17802FB036313
:10B95000E27842EA01220B495B185A6009E024228E
:10B9600056435B090C2202FB03630649E2785B182D
:10B970001A72F8BDC00B0020300C0020280C0020EB
:10B98000340C00206C0B00202DE9F3414901CEB2AC
:10B9900001AC46F015031746694622468DF804307F
:10B9A0008046FFF75BFF9DF801C09DF8033046F02D
:10B9B00014064046694622466D468DF804608DF8AF
:10B9C00005C08DF806708DF80730FFF747FFBDE81A
:10B9D000FC8100BF2DE9F3414901CEB201AC46F034
:10B9E00015031746694622468DF804308046FFF756
:10B9F00035FF9DF801C09DF8023046F01406404620
:10BA0000694622466D468DF804608DF805C08DF8B4
:10BA100006308DF80770FFF721FFBDE8FC8100BFFD
:10BA200037B541F001030C466A4601A98DF8003094
:10BA30000546FFF713FF9DF806009DF8052000025C
:10BA40009DF8073040EA0240184310F4000F18BF79
:10BA500040F07F405F2C1AD8C4F3411314F01E0449
:10BA600002D0022C13D106E0032202FB0535084A5E
:10BA70002D01A8580BE0032202FB053520F07F4181
:10BA8000E8B2FFF7B5FE024B03EB051568683EBD53
:10BA9000480E002007B541F001036A4601A98DF860
:10BAA0000030FFF7DBFE9DF806009DF8073043EA03
:10BAB000002010F4006F1CBF6FEA00506FEA1050B6
:10BAC0000EBD00BF13B541F00103144601A96A463B
:10BAD0008DF80030FFF7C2FE9DF805109DF8063086
:10BAE0009DF807202170A27063709DF804001CBDB2
:10BAF00007B5410141F0160101F0F601002001AA4D
:10BB0000FFF7E0FF9DF80530D80913F0200F18BFAC
:10BB100040F002000EBD00BF07B5410141F0160123
:10BB200001F0F601002001AAFFF7CCFF9DF80530D7
:10BB3000C3F3801013F0100F18BF40F002000EBDC9
:10BB400037B50C4641EA401101AA0546C9B20020AA
:10BB5000FFF7B8FFB4235D436408032305F5807540
:10BB600003FB04549DF804102046FCF723FD601CE1
:10BB70009DF80510FCF71EFDA01C9DF80610FCF7B3
:10BB800019FD3EBD5F292DE9F3410D4606461446D9
:10BB900062D8C1F3411811F01E0102D002295BD115
:10BBA0001EE0032202FB0088344A4FEA0810831883
:10BBB0005B688450E01A0028B8BF4042B0F5000F1F
:10BBC0000ADB9C42CCBF2E4C2E4C2C4A1C1902EB9B
:10BBD0000812012313733FE002EB081211733BE0DC
:10BBE000032707FB0087254B3801C1587A00C4EBB7
:10BBF000010C0132BCF1000FB8BFCCF1000C00EB1E
:10BC0000030EBCF5000F24F07F40CEF8044043F84B
:10BC100032001DDBA142CCBF194B1A4B4FEA48182A
:10BC2000E3184FEA234E4FEA232C3046694601AA17
:10BC30008DF807308DF804808DF805E08DF806C08A
:10BC4000FFF70CFE0D4B03EB071701233B7303E0DB
:10BC500003EBC20300221A714FEA244C2312304630
:10BC6000694601AA8DF804508DF805C08DF806309C
:10BC70008DF80740FFF7F2FDBDE8FC81480E00207B
:10BC8000FFFF7F00010080FF38B50D4668210446A4
:10BC9000FFF7C6FE15B140F0010201E020F00102FD
:10BCA00020466821FFF76EFF38BD00BF07B5134679
:10BCB0004FEA222C8DF804104FF0000E694601AABD
:10BCC0008DF805E08DF806C08DF80730FFF7C6FD4A
:10BCD0000EBD00BF07B50B4611F01E01024601D094
:10BCE000022905D1104619460022FFF74BFF0DE04F
:10BCF0004FF0000C694601AA8DF804308DF807C09A
:10BD00008DF805C08DF806C0FFF7A8FD0EBD00BF79
:10BD100010B5C4B22146640100200222E4B2FFF74C
:10BD200059FE002044F00801FFF7D4FF44F00A0157
:10BD30000020FFF7CFFF10BD07B59DF810C08DF8AC
:10BD400004108DF80520694601AA8DF806308DF89B
:10BD500007C0FFF783FD0EBD30B5430185B0044633
:10BD600043F00303002003A902AA8DF80830FFF76F
:10BD700075FD9DF80E109DF80D209DF80F300902FD
:10BD800041EA024119432046FFF732FD174B03EB0E
:10BD9000041108310A7932B3154A0C2000FB042241
:10BDA000107A00BB2201D518D2586B68C3EB020C85
:10BDB000BCF1000FB8BFCCF1000CBCF5000F05DBE7
:10BDC0009A42CCBF0B4A0C4A9A1800E008716101F4
:10BDD000C2F30723D4B201F0E0010020C2F307420E
:10BDE0000094FFF7A9FF05B030BD00BF480E00204A
:10BDF0006C0B0020FFFF7F00010080FF07B59378E8
:10BE000092F800E092F801C08DF8041001AA69468A
:10BE10008DF805E08DF806C08DF80730FFF71EFDA0
:10BE20000EBD00BF37B5440144F01604E4B20D4620
:10BE300001AA21460020FFF745FE9DF8053015F0C8
:10BE4000010F1ABF6FEA43636FEA536303F07F0386
:10BE50008DF805309DF8053015F0020F14BF43F042
:10BE6000200323F020038DF80530002318462146D7
:10BE700001AA8DF80630FFF7C1FF3EBD37B544017A
:10BE800044F01604E4B20D4601AA21460020FFF753
:10BE900019FE9DF8053015F0010F14BF43F0400363
:10BEA00023F040038DF805309DF8053015F0020FA2
:10BEB00014BF43F0100323F010038DF80530002366
:10BEC0001846214601AA8DF80630FFF797FF3EBDC0
:10BED00073B5B42545434B08032205F5807502FB75
:10BEE0000355044628460E46FCF7CEFA8DF80400AA
:10BEF000681CFCF7C9FA8DF80500A81CFCF7C4FA09
:10BF000046EA44148DF80600E1B2002001AAFFF7CA
:10BF100075FF7CBD2DE9F74F4001C7B24C050020ED
:10BF200047F0180101AAFFF7CDFD9DF80560640DEB
:10BF300006F00F053609B5420EDB204605F090F9F4
:10BF4000AD1B80460120A840894605F099F90022E2
:10BF5000334B05F0FBF90FE0204605F081F9751B26
:10BF600080460120A840894605F08AF902460B4622
:10BF700000202B4905F014FB02460B46404649467B
:10BF800005F00EFB05F0A4FC05F08CF922A3D3E923
:10BF9000002305F0DBF905F09BFC05F083F9002296
:10BFA000204B05F0D3F94FF0FF36B046002582460E
:10BFB0008B460120A84005F063F902460B46504627
:10BFC000594605F0C3F905F05BFCA0F180027F2A19
:10BFD00098BF2E46034605F1010588BF43460E2D46
:10BFE00001D09846E5E7002547F0120101AA28464E
:10BFF0008DF805308DF806608DF80450FFF7FEFED1
:10C00000284647F00C012246FFF750FE2846BDE8BF
:10C01000FE8F00BFAFF3008004560E2DB29DEF3FA0
:10C02000000060400000204013B5154B587E10F012
:10C03000010003D000206821212201E06821202294
:10C040000024FFF79FFD20467E21202223460094F6
:10C05000FFF772FEE1B200200134FFF739FF1D2C1B
:10C06000F8D10C210020FFF7DBFC01460020FFF790
:10C0700051FF0020162143F2FF12FFF717FE1CBDEF
:10C0800008000020AFF30080084B1868034605E065
:10C090002C2A02D100221A7003E001331A78002AF8
:10C0A000F6D1024A01331360704700BFE404002058
:10C0B00010B50E4B02461B78ABB10D4B1C7994B1F9
:10C0C0009C68601CE4180D2A2273986002D03F28F7
:10C0D00000D851B9064C014604F10C00FDF7FEFBF7
:10C0E0000023A36001E0FCF759FC10BD200B0020E9
:10C0F000E404002030B50121044687B02020FFF77A
:10C10000D7FF002C04DA2D200121FFF7D1FF644274
:10C1100000230A2194FBF1F201FB124101AD303101
:10C12000E954591C141E01DD0B46F2E7ED181C46BC
:10C130000121013C15F80109FFF7BAFFB4F1FF3FF7
:10C14000F6D107B030BD00BF38B50C4D0446A87815
:10C1500001214030C0B2FFF7ABFF687801214030C9
:10C16000C0B2FFF7A5FF2078FFF7C4FF6068FFF7B4
:10C17000C1FF0D200121FFF79BFF38BD0800002003
:10C1800070B5124B06461B78EBB1FCF7D5FB104C93
:10C19000054618B100232371012016E0E36C226DDF
:10C1A000934208D21A1992F85420013301203270B8
:10C1B000E364207109E004F15400FDF75DFBE564E0
:10C1C0002065284601E0FCF7B7FB70BD200B00207E
:10C1D000E40400202DE9F34104460DF10700FFF7C8
:10C1E000CFFF002800F0CB808B4B8C4A93F8941043
:10C1F00019BB51789DF80700403188420DD1D3F822
:10C200009810002940F0BB801179012231F0010122
:10C2100083F8942040F0B380AFE00D2801D01B28B4
:10C2200002D100227C4B05E0D3F898207E2A00F250
:10C23000A6800132C3F89820A1E0117931F0010104
:10C2400003D19DF80700FFF733FF9DF807301F2B40
:10C250000BD9714AD2F898107E297FD8481C8918CA
:10C2600081F89C30C2F8980078E0082B08D16A4B1E
:10C27000D3F89820002A71D0013AC3F898206DE0D5
:10C280000D2B6BD1644BD3F89830002B66D0634BE9
:10C290001A79112A15D1587801214030C0B2FFF720
:10C2A00007FF002503E0585DFFF702FF01355A4BF9
:10C2B0000121D3F898209C339542F4D30D20FFF749
:10C2C000F7FE554A00231568D2F8987019461A46A9
:10C2D00033E001290FD002D302292DD122E04E4EA6
:10C2E00006F19C00805C202826D09E1986F81C014F
:10C2F0000133012120E0484800F19C0C1CF802C0E9
:10C30000BCF1200F0AD1012B04D91818002180F8A4
:10C310001C110133424D0221ED180DE0181880F870
:10C320001CC108E03C4E06F19C00805C202803D034
:10C330009E1986F81C0101330132BA42C9D3364A2C
:10C340000021981880F81C110120C2F8981015607F
:10C3500082F8A001C2F89C3182F894109DF8073051
:10C360001B2B0CD12D4A2C4B12790021012A83F86A
:10C370009410C3F8981002D10D20FFF799FE264BB8
:10C3800093F8A001002878D00022164683F8A02157
:10C390001546DFF8A880072707FB058720483946A0
:10C3A000013504F03BF930B9BE797B7916F0010F05
:10C3B000237049D007E018F806300736002B5ED00E
:10C3C000FF2DE6D15BE0FFF75FFE23780546042BE7
:10C3D0000CD1144904F022F90346D8B12846124979
:10C3E00004F01CF970B1284610490FE00D2B28D13C
:10C3F0000F4904F013F9034660B128460D4904F0D3
:10C400000DF908B9012305E00B49284604F006F9A7
:10C41000B0B90223637017E0E40400200800002094
:10C4200000060020592901085D2901086129010839
:10C43000672901086D2901087229010850270108A0
:10C44000284604F0E5F8607016F0020F04D0FFF7FC
:10C450001BFE04F0DDF8A07016F0040F0CD0FFF7FF
:10C4600013FE04F0D5F8010EC0F30722C0F3074312
:10C47000A17122716371E0700120BDE8FC8100238D
:10C480002370F9E7704700BFFEE700BFFEE700BF7B
:10C49000FEE700BFFEE700BF704700BF704700BF68
:10C4A000704700BF704700BF704700BF704700BFB4
:10C4B000704700BF704700BF704700BF704700BFA4
:10C4C000704700BF704700BF704700BF704700BF94
:10C4D000704700BF704700BF704700BF704700BF84
:10C4E000704700BF704700BF704700BF704700BF74
:10C4F00008B5024B1B68984708BD00BF480B0020D9
:10C5000008B5024B1B68984708BD00BF2C0C0020E3
:10C5100008B5024B1B68984708BD00BFBC0B002044
:10C5200008B5024B1B68984708BD00BFE00B002010
:10C53000704700BF704700BF704700BF704700BF23
:10C54000704700BF704700BF704700BF704700BF13
:10C55000704700BF704700BF704700BF704700BF03
:10C56000704700BF704700BF704700BF704700BFF3
:10C57000704700BF704700BF704700BF704700BFE3
:10C58000704700BF704700BF704700BF704700BFD3
:10C59000704700BF704700BF704700BF704700BFC3
:10C5A000704700BF704700BF704700BF704700BFB3
:10C5B000704700BF704700BF704700BF704700BFA3
:10C5C000704700BF436830B523F470230C680A79C4
:10C5D00023F48073234343EA0223436082688D6817
:10C5E000CC680A4B45EA040C02EA03034A794CEA98
:10C5F000030343EA420383600B7CC26A013B22F4DB
:10C600007002DBB242EA0353C36230BDFDF7F1FFB3
:10C61000002301220274C3600360037143718360CD
:10C62000704700BF19B1836843F0010302E08368DB
:10C6300023F001038360704719B1836843F480736A
:10C6400002E0836823F4807383607047C9B212B13B
:10C650004368194302E0436823EA010141607047DF
:10C66000836843F008038360704700BF8068C0F3AD
:10C67000C0007047836843F004038360704700BFC5
:10C680008068C0F38000704719B1836843F4A00349
:10C6900002E0836823F4A003836070478068C0F3DE
:10C6A000805070474368013923F4604343EA4133C3
:10C6B0004360704719B1436843F4006302E0436884
:10C6C00023F4006343607047092930B511D94FF056
:10C6D000030C0CFB01FC0725ACF11E0C05FA0CF554
:10C6E00003FA0CFCC46824EA050343EA0C03C360A4
:10C6F0000EE04FF0030C0CFB01FC072505FA0CF5CE
:10C7000003FA0CFC046924EA050343EA0C03036101
:10C71000062A0DD80523013A5A434FF01F0C0CFA94
:10C7200002FC9140436B23EA0C020A4342631CE083
:10C730000C2A0DD805235A434FF01F0C233A0CFA4C
:10C7400002FC9140036B23EA0C020A4302630CE0F3
:10C7500005235A434FF01F0C413A0CFA02FC91405A
:10C76000C36A23EA0C020A43C26230BD19B183686E
:10C7700043F4801302E0836823F4801383607047DE
:10C78000C06C80B2704700BF014B1868704700BF93
:10C790004C24014019B1436843F4806302E04368CC
:10C7A00023F480634360704719B1436843F48053B6
:10C7B00002E0436823F4805343607047836823F4A6
:10C7C000E04341EA03038360704700BF19B1836807
:10C7D00043F4004302E0836823F40043836070471E
:10C7E00019B1836843F4021302E0836823F402134F
:10C7F000836070478068C0F340507047092930B5A6
:10C8000011D94FF0030C0CFB01FC0725ACF11E0CF9
:10C8100005FA0CF503FA0CFCC46824EA050343EAA4
:10C820000C03C3600EE04FF0030C0CFB01FC07256A
:10C8300005FA0CF503FA0CFC046924EA050343EA43
:10C840000C030361836BC3F3015CCCEB0202023285
:10C850004FF0050CD2B20CFB02F20CF11A0C0CFAE0
:10C8600002FC914023EA0C030B43836330BD00BFFD
:10C87000836B013923F4401343EA01538363704708
:10C880000A5070472830405880B27047436823F4FC
:10C89000400323F4007341EA03034360704700BF81
:10C8A00041628262704700BF436823F01F0341EA80
:10C8B00003034360704700BF20B1054B9A6842F400
:10C8C000000203E0024B9A6822F400029A6070476B
:10C8D00000240140036819420CBF0020012070476A
:10C8E000C9430160704700BF4368006810EA112027
:10C8F00004D0C9B219420CBF00200120704700BF0C
:10C900006FEA11210160704708B5134B98420FD0B0
:10C9100003F5A053984213D0A3F5C053984219D100
:10C920004FF40070012101F00BFB4FF400700EE09A
:10C930004FF48060012101F003FB4FF4806006E0BA
:10C940004FF40040012101F0FBFA4FF400400021B8
:10C9500001F0F6FA08BD00BF00280140374B012264
:10C960001A605A6812F0010201D1104664E00278A0
:10C97000012A0BBF1A681A6842F0800222F0800276
:10C980001A604378012B04D12C4B1A6842F0400204
:10C9900003E02A4B1A6822F040021A608378012BC8
:10C9A00004D1264B1A6842F0200203E0234B1A6898
:10C9B00022F020021A60C378012B04D11F4B1A68A1
:10C9C00042F0100203E01D4B1A6822F010021A60B8
:10C9D0000379012B04D1194B1A6842F0080203E0D5
:10C9E000164B1A6822F008021A604379012B04D111
:10C9F000124B1A6842F0040203E0104B1A6822F04E
:10CA000004021A608279C37990F808C0920742EA5A
:10CA100003624189437A42EA0C4242EA03520139F5
:10CA2000064B0A43DA611A6822F001021A6058685C
:10CA300080F0010000F00100704700BF006400407A
:10CA400090F800C0012202FA0CF23B4B2DE9F045B0
:10CA5000D3F8004292B244F00104C3F80042D3F884
:10CA60001C42D14301EA0404C3F81C428478A4B9EF
:10CA70000CF1480CD3F80C72B0F80AA0C688B0F8D4
:10CA8000088085884FEACC0404F1804446EA0A46CF
:10CA900045EA084501EA070715E0012C1AD10CF117
:10CAA000480CD3F80C72B0F804A0C688B0F808801F
:10CAB00045894FEACC0404F1804446EA0A4645EA37
:10CAC000084542EA070704F5C844C3F80C7243F866
:10CAD0003C60656043782BB9174BD3F8044201EAF8
:10CAE000040404E0144BD3F8044242EA0404C3F8FB
:10CAF0000442838923B9104BD3F81442214006E045
:10CB0000012B06D10C4BD3F8141242EA0101C3F8F1
:10CB10001412837B012B05D1074BD3F81C120A4357
:10CB2000C3F81C22044BD3F8002222F00102C3F800
:10CB30000022BDE8F08500BF0064004003220272BD
:10CB4000013A002342724FF00102C3714281037027
:10CB500043708370C370037143718371704700BF6A
:10CB600019B1054B5A69104303E0034B5A6922EA95
:10CB700000005861704700BF00640040364B70B53C
:10CB80009968024611F0806F01D000200CE099688E
:10CB900011F0006F01D0012006E09B6813F0805F68
:10CBA00001D1042056E002202B4B00F118010901AD
:10CBB000CC5804F00104CC50157A92F809C035B96C
:10CBC000146864051460CD584CEA050C07E05468FD
:10CBD00045EA0C0CE4005460CE584CEA060C4CEAD2
:10CBE0000404CC50947A00F1180C4FEA0C1C04F0A9
:10CBF0000F040CF18043947203F5C8435D68010192
:10CC000025F00F055D605D6801F180412C435C609B
:10CC1000537B947BD57A1B0443EA0463147B2B4338
:10CC200043EA042301F5C841C1F88831557C937C5F
:10CC3000D47B2D0445EA0365137C45EA040242EAED
:10CC40000322054BC1F88C215CF8032042F001025D
:10CC50004CF8032070BD00BF00640040012810D0D4
:10CC600002D302282CD11AE0164A91689368926880
:10CC700001F0010103F0020343EA8103C2F3806281
:10CC80001AE0104A9368916803F48073926801F483
:10CC900000719B0943EA1123C2F3C0620CE0094A08
:10CCA0009368916803F48033926801F400319B0B20
:10CCB00043EA1143C2F300721343034AD05C704746
:10CCC0000023FAE70064004030280108012808D05A
:10CCD00002D302280FD109E0074B9A6842F0800284
:10CCE00008E0054B9A6842F4004203E0024B9A6860
:10CCF00042F400029A6070470064004018B9044B87
:10CD00002022DA6002E0024B20221A61704700BF45
:10CD10000064004010B9064BD86805E0012801D036
:10CD2000002003E0024B186900F00300704700BFC9
:10CD300000640040254B00F11B02120110B5D458CD
:10CD400004F004040C721CB9D3585B0D0B6002E0B4
:10CD5000D358DB084B6000F11B021C4B1201D35867
:10CD600002F1804203F002034B7202F5C84254689C
:10CD7000030104F00F0C81F80AC0526803F18043EC
:10CD8000120ACA7403F5C843D3F8B821CA72D3F89B
:10CD9000B821120A0A73D3F8B821120C4A73D3F8D7
:10CDA000B821120E8A73D3F8BC21CA73D3F8BC2100
:10CDB000120A0A74D3F8BC21120C4A74D3F8BC319D
:10CDC0001B0E8B74FFF79AFF10BD00BF006400407C
:10CDD000044B1A6842F002021A601868C0F340005F
:10CDE000704700BF00640040054B1A6822F0020241
:10CDF0001A60186880F00200C0F34000704700BF5E
:10CE000000640040034B9B6918420CBF00200120C6
:10CE1000704700BF00640040024B9A6922EA00029A
:10CE20009A61704700640040202831D00CD8062851
:10CE300020D004D8042825D0052844D118E007289C
:10CE40001DD008283FD11FE0B0F5007F2BD005D8BA
:10CE500040281FD0B0F5807F35D11FE0B0F5803F6E
:10CE60002CD0B0F5003F2BD0B0F5806F2BD11FE058
:10CE7000012201E04FF48072134B9A6023E04FF4DB
:10CE80008032F9E7082200E010220F4BDA601AE046
:10CE9000082200E010220C4B1A6114E00A4B9A6938
:10CEA00022F0010208E0084B9A6922F0020203E036
:10CEB000054B9A6922F004029A6104E0082200E01E
:10CEC0001022014B5A6070470064004001420CBFC1
:10CED00000200120704700BF202808B532D00CD8B0
:10CEE000062821D004D8042826D0052818D119E016
:10CEF00007281ED0082813D120E0B0F5007F29D0E4
:10CF000005D8402820D0B0F5807F09D120E0B0F5C9
:10CF1000803F27D0B0F5003F22D0B0F5806F1BD006
:10CF2000002024E0012101E04FF48071104B98684B
:10CF30001BE04FF48031F9E7082100E010210C4B91
:10CF4000D86812E0082100E01021094B18690CE0B4
:10CF5000012102E0022100E00421054B986904E070
:10CF6000102100E00821024B5868FFF7AFFF08BD11
:10CF700000640040012108B54FF0007000F0EEFFA2
:10CF80004FF00070002100F0E9FF08BD02680023A7
:10CF900022F001020260036043608360C3602D4B96
:10CFA000984233D011D83C3B984229D006D8283B30
:10CFB000984221D0143398424BD11FE0264B98421F
:10CFC00020D01433984244D11EE0244B98422CD0F8
:10CFD00008D8A3F5677398421DD003F56273984291
:10CFE00037D11DE01E4B984229D0143398422BD0E4
:10CFF000283B98422DD11DE01A4B12E0194B15E049
:10D00000184B18E0174B1BE0164B1EE0154B5A68E7
:10D0100042F470021CE0134B5A6842F0706217E051
:10D02000114B5A6842F00F0212E00F4B5A6842F05F
:10D03000F0020DE00C4B5A6842F4706208E00A4BB3
:10D040005A6842F4704203E0074B5A6842F4702277
:10D050005A6070476C000240440002401C040240C9
:10D060004404024000000240000402408A6870B597
:10D070000C6A0B6944EA02024C691A438B69224329
:10D08000CC6905684E6A42EA030323438C6A334342
:10D0900025F4FE4C23432CF0F00C43EA0C03036010
:10D0A000CB6843600B6883604B68C36070BD00BF92
:10D0B00000238362036043608360C3600361436154
:10D0C0008361C36103624362704700BF19B10368A3
:10D0D00043F0010302E0036823F00103036070479B
:10D0E00012B10368194302E0036823EA01010160F9
:10D0F000704700BF406880B2704700BF10F0805F8B
:10D1000014BF044B044B1B6803420CBF00200120DA
:10D11000704700BF000402400000024010F0805F32
:10D1200014BF024B024B5860704700BF000402401E
:10D130000000024010F0805F14BF044B044B1B68DA
:10D1400003420CBF00200120704700BF00040240D2
:10D150000000024010F0805F14BF024B024B586089
:10D16000704700BF0004024000000240044B002250
:10D170001A605A609A60DA60024A5A61704700BFCA
:10D1800000040140FFFF0700837930B50168027990
:10D190004BB3184BCC431D6890F805C004EA050555
:10D1A0001D605D682C405C60D45844EA0101D15098
:10D1B00002689868D14301EA00009860D86801408D
:10D1C000BCF1100FD96007D1996811439960D968F3
:10D1D00041EA0202DA600BE05CF8031041EA020265
:10D1E0004CF8032004E0034BD05820EA0101D15051
:10D1F00030BD00BF0004014000230C228371427146
:10D2000003600371704700BF024B1A6940EA0202D3
:10D210001A61704700040140034B5B6918420CBF60
:10D2200000200120704700BF00040140014B5861FD
:10D23000704700BF00040140054B1A685B6903405A
:10D2400001D1184603E010420CBF002001207047B6
:10D2500000040140014B5861704700BF00040140C9
:10D26000044B1A6802F038021A601A6840EA020297
:10D270001A60704700200240044B1A6822F008022E
:10D280001A601A6840EA02021A60704700200240E1
:10D29000044B1A6822F010021A601A6840EA02026F
:10D2A0001A60704700200240034B044A5A6002F1A2
:10D2B00088325A60704700BF002002402301674552
:10D2C000024B1A6942F080021A6170470020024046
:10D2D000014BD8698008704700200240014B186A52
:10D2E000704700BF00200240024BD869C0F34000E5
:10D2F000704700BF00200240024B1868C0F3401086
:10D30000704700BF0020024019B1054B1A69104355
:10D3100003E0034B1A6922EA00001861704700BF5E
:10D3200000200240012804D1054BD86900F001001B
:10D3300005E0034BDB6818420CBF0020012070475A
:10D3400000200240014BD860704700BF002002401F
:10D35000094BDA6812F0010F01D001200BE0DA6806
:10D3600012F0040F01D0022005E0DB6813F0100F6B
:10D3700014BF0320042070470020024013B5044668
:10D380000AE000230193FF3301E0019B013B01937D
:10D39000019B002BF9D1013CFFF7DAFF012802D1F4
:10D3A000002CEED100E004B905201CBDF8B5124CEC
:10D3B000124B0546A36003F188330F20A3600E468D
:10D3C0001746FFF7DBFF042814D1236945F0F80561
:10D3D00043F0100323612E43094B37430B305F802A
:10D3E000FFF7CCFF012805D0226941F6EF7302EA6E
:10D3F00003032361F8BD00BF0020024023016745FD
:10D4000000F8FF1F38B5054640F6FF70FFF7B6FF7E
:10D4100004283CD11E4C1F4B40F6FF70A36003F163
:10D420008833A360236943F020032361236943F019
:10D4300040032361FFF7A2FF042820D1226941F6AF
:10D44000DF7302EA03032361236943F010032361BE
:10D450001DB1114B4FF0000202E00F4B4FF0A5023F
:10D460001A8040F6FF70FFF789FF01280FD0084AA5
:10D4700041F6EF73116901EA0303136107E0012824
:10D4800005D0226941F6DF7302EA0303236138BD48
:10D49000002002402301674500F8FF1F10B5044635
:10D4A0000F20FFF76BFF04283DD11F4A1F4BE443B9
:10D4B000936003F1883393601169E3B241F0100186
:10D4C000FF2B116106D01A4A0B301381FFF756FF6C
:10D4D00004281FD1C4F30723FF2B06D0144A0F20C2
:10D4E0005381FFF74BFF042814D1C4F30743FF2BEC
:10D4F00006D00F4A0F209381FFF740FF042809D17F
:10D50000240EFF2C01D1042006E0094B0F20DC8102
:10D51000FFF734FF012806D0034A41F6EF73116983
:10D5200001EA0303136110BD002002402301674597
:10D5300000F8FF1F70B504460F200E46FFF71EFFD0
:10D54000042815D10B4D0C4B0B30AB6003F1883325
:10D55000AB602B6943F010032B612680FFF70EFFB1
:10D56000012805D02A6941F6EF7302EA03032B6113
:10D5700070BD00BF002002402301674570B504461E
:10D580000F200E46FFF7FAFE042810D1084D0B308D
:10D590002B6943F001032B612680FFF7EFFE012882
:10D5A00005D02A6941F6FE7302EA03032B6170BDC0
:10D5B0000020024070B504460F200E46FFF7DEFE45
:10D5C000042818D10C4DB3B22A690B3042F0010285
:10D5D0002A612380FFF7D2FE042804D1360C66802E
:10D5E0000B30FFF7CBFE012805D02A6941F6FE7308
:10D5F00002EA03032B6170BD0020024010B540F623
:10D60000FF70FFF7BBFE04282CD1174C174B40F6D8
:10D61000FF70A36003F18833A360236943F0200304
:10D620002361236943F040032361FFF7A7FE042829
:10D6300010D1226941F6DF7302EA030323612369F3
:10D640004FF0A50243F010032361094B0B301A8001
:10D65000FFF794FE012805D0226941F6EF7302EA34
:10D660000303236110BD00BF002002402301674572
:10D6700000F8FF1F10B540F6FF70FFF77FFE04288B
:10D6800014D10B4C40F6FF70236943F0040323616F
:10D69000236943F040032361FFF770FE012805D0A2
:10D6A000226941F6FB7302EA0303236110BD00BF48
:10D6B0000020024038B5054640F6FF70FFF75EFED9
:10D6C000042815D10B4C40F6FF70236943F0020388
:10D6D00023616561236943F040032361FFF74EFE38
:10D6E000012805D0226941F6FD7302EA0303236194
:10D6F00038BD00BF00200240CB78F0B513F0100F0A
:10D7000018BF8A78098803F00F0C18BF4CEA020C86
:10D7100011F0FF0F1AD0046800220126964006EA95
:10D720000105B5420ED196000F27B7400CFA06F658
:10D7300024EA07043443282B01D1456102E0482B39
:10D7400008BF05610132082AE7D10460FF291CD90E
:10D750004468002202F108050126AE4006EA0105F0
:10D76000B5420ED196000F27B7400CFA06F624EA10
:10D7700007043443282B01D1456102E0482B08BF40
:10D7800005610132082AE5D14460F0BD0423C3706D
:10D79000022383704FF0FF33038070478368194280
:10D7A0000CBF002001207047806880B2704700BF26
:10D7B000C36819420CBF002001207047C06880B2C6
:10D7C000704700BF01617047416170470AB1016154
:10D7D00000E04161704700BFC160704741F4803391
:10D7E000836181618361836983697047064A10B5EB
:10D7F00014684FF6807341EA001104EA030341EA1A
:10D800000303136010BD00BF00000140014B18600E
:10D81000704700BF1C0020420304154A00F4401C5E
:10D820001B0CBCF5401F30B5546806D1556824F078
:10D83000706425F07065556011E010F4801F06D00B
:10D84000C0F303424FF0030C0CFA02F203E0420D66
:10D85000120113FA02F224EA020444F0706419B1CE
:10D86000400D000183401C43014B5C6030BD00BF94
:10D870000000014001F003039B000F229A4010FAC0
:10D8800003F310B58908074C023154F8210020EA4F
:10D89000020244F8212054F82120134344F8213097
:10D8A00010BD00BF000001400120014608B500F096
:10D8B00047FB0120002100F043FB08BD08B5264BC3
:10D8C00098422BD00CD8A3F5006398421AD003F5E8
:10D8D000806398421CD0A3F5006398423AD10BE0D4
:10D8E0001E4B984226D003F58063984228D0A3F5BA
:10D8F000006398422ED117E00420012100F020FBA4
:10D90000042024E00820012100F01AFB08201EE07A
:10D910001020012100F014FB102018E0202001212C
:10D9200000F00EFB202012E04020012100F008FB57
:10D9300040200CE08020012100F002FB802006E066
:10D940004FF48070012100F0FBFA4FF48070002149
:10D9500000F0F6FA08BD00BF00140140001C0140B1
:10D960000B4B4FF0FF316FF07042C3F88010C3F8DB
:10D970008420C3F88011C3F88421002303F1C0017F
:10D98000034A013300200F2B42F82100F6D17047E3
:10D9900000E100E0094B4FF0206058600848002289
:10D9A0004FF0FF319A60D8601A615A619A61DA616A
:10D9B0001A625A629962D9621963704700ED00E0F9
:10D9C0000000FA0540F0BE60024B40F42020D86011
:10D9D000704700BF00ED00E030B5C27803787AB33D
:10D9E0001C4A4178D2684FF00F0CD243C2F3022296
:10D9F0002CFA02FCC2F104029140807803F0030289
:10DA00000CEA000C4CEA010CD2004FEA0C1CFF207F
:10DA100090400CFA02FC012403F01F029440990884
:10DA20000D4AC03152F821500CEA000C25EA0000E2
:10DA30004CEA00005B0942F8210042F8234008E06C
:10DA400003F01F02012191405B09034A203342F891
:10DA5000231030BD00ED00E000E100E00023C370C2
:10DA60000370437083707047024B5868C0F30930ED
:10DA7000704700BF00ED00E0012200F01F0312FA22
:10DA800003F34009044A403052F8200018409842FD
:10DA900014BF00200120704700E100E0014B186036
:10DAA000704700BF00EF00E000F01F0301229A4022
:10DAB0004009024B603043F82020704700E100E04D
:10DAC000024B58688005800D704700BF00ED00E0F4
:10DAD000012200F01F0312FA03F34009044A8030C8
:10DAE00052F820001840984214BF002001207047CF
:10DAF00000E100E0014B1868704700BF00ED00E056
:10DB000021F0604121F07F01014B01439960704792
:10DB100000ED00E0014A024BDA6070470400FA05AC
:10DB200000ED00E0014A024BDA6070470100FA059F
:10DB300000ED00E019B1054B1A69104303E0034BF7
:10DB40001A6922EA00001861704700BF00ED00E08A
:10DB500000F01F00012313FA00F019B1044B5A6AB8
:10DB6000104303E0024B5A6A22EA000058627047F1
:10DB700000ED00E0144B70B5DC684FF0FF0CE4439F
:10DB8000C4F302242CFA04F5C4F1040411FA04F4D9
:10DB9000C0F30126F6000CFA06FC02EA050545EA88
:10DBA0000404240114FA06F6C0F38110063053F879
:10DBB000202022EA0C0243F8202053F820201643AC
:10DBC00043F8206070BD00BF00ED00E0C0F383208B
:10DBD00001238340044A506A03EA0000984214BFBC
:10DBE00000200120704700BF00ED00E000F01F00A2
:10DBF00001228240024B59680A435A60704700BFB5
:10DC000000ED00E000F01F020123013A13FA02F2D6
:10DC1000024B59680A435A60704700BF00ED00E0AC
:10DC2000C0F3833001238340044A506A03EA0000B2
:10DC3000984214BF00200120704700BF00ED00E0B3
:10DC4000C0F3814313B90A4BD86A10E0012B0CD101
:10DC5000074AC0F30153906ADA00D040022B14BF88
:10DC600000F00F0000F0FF0001E0014B186B70475F
:10DC700000ED00E010F4800F0BBF024B014B586B1E
:10DC8000986B704700ED00E008B5F6F771FA08BD33
:10DC900008B50001F6F769FA08BD00BF08B5F6F748
:10DCA00062FA08BD08B5F6F75CFA08BD08B5F6F7E4
:10DCB00056FA08BD08B5F6F750FA08BD0D4B0E4AE6
:10DCC000196841F001011960596801EA02025A60BD
:10DCD0001A6822F0847222F480321A601A6822F4E0
:10DCE00080221A605A6822F4FE025A6000229A606A
:10DCF000704700BF001002400000FFF80C4BB0F569
:10DD0000803F1A6822F480321A601A6822F4802256
:10DD10001A6003D0B0F5802F08D103E01A6842F4EE
:10DD2000803202E01A6842F4A0221A60704700BFF5
:10DD300000100240034B1A6822F0F80242EAC002C7
:10DD40001A60704700100240014B1860704700BF16
:10DD500000004242044B5A6822F47C1240EA02025C
:10DD60000A435A60704700BF00100240014B186020
:10DD7000704700BF60004242034B5A6822F0030222
:10DD800040EA02025A60704700100240024B586895
:10DD900000F00C00704700BF00100240034B5A68AF
:10DDA00022F0F00240EA02025A607047001002407E
:10DDB000034B5A6822F4E06240EA02025A6070475C
:10DDC00000100240034B5A6822F4605242EAC0023B
:10DDD0005A6070470010024019B1054B1A78104381
:10DDE00003E0034B1A7822EA00001870704700BF66
:10DDF00009100240014B1860704700BFD800424232
:10DE0000034B5A6822F4404240EA02025A607047CB
:10DE100000100240064B002201281A701A7002D02E
:10DE2000042804D101E0187001E005221A7070473F
:10DE300020100240014B1860704700BF800442422E
:10DE4000024B1A6A40EA02021A627047001002404E
:10DE5000014B1860704700BF3C0442421F4B10B595
:10DE60005A6802F00C02042A13D0082A11D15A6809
:10DE70005968C2F38342023211F4803F03D05B68D9
:10DE800013F4003F01D0164B00E0164B5A430260DA
:10DE900001E0144B0360114A134B51680468C1F34D
:10DEA0000311595C34FA01F141605468C4F3022C47
:10DEB00013F80C4031FA04F484605468C4F3C22CA3
:10DEC00013F80CC021FA0CF1C1605268C2F3813220
:10DED0009B181B7CB1FBF3F1016110BD00100240E7
:10DEE00000093D0000127A003828010819B1054BDD
:10DEF0005A69104303E0034B5A6922EA0000586153
:10DF0000704700BF0010024019B1054B9A691043D9
:10DF100003E0034B9A6922EA00009861704700BF52
:10DF20000010024019B1054BDA69104303E0034BBE
:10DF3000DA6922EA0000D861704700BF0010024091
:10DF400019B1054BDA68104303E0034BDA6822EAA3
:10DF50000000D860704700BF0010024019B1054BA7
:10DF60001A69104303E0034B1A6922EA00001861A2
:10DF7000704700BF00100240014B1860704700BF9F
:10DF800040044242014B1860704700BF4C004242BF
:10DF9000014B1870704700BF071002404309012B66
:10DFA00002D1084B1B6805E0022B0BBF054B054B4C
:10DFB0001B6A5B6A00F01F0033FA00F000F00100FA
:10DFC000704700BF0010024008B53120FFF7E6FFA0
:10DFD000094B18705A6801325A601A7822B95A6887
:10DFE00040F2FF139A42F0D13120FFF7D7FF0038FB
:10DFF00018BF012008BD00BF88060020024B5A6AE6
:10E0000042F080725A62704700100240034B9B68D6
:10E0100018420CBF00200120704700BF00100240D2
:10E02000014B1870704700BF0A1002400B884A88E5
:10E03000B1F804C01A43CB8842EA0C02B1F808C018
:10E040001A434B8930B542EA0C028D89B0F800C002
:10E05000CC891A432A4322430CF4415313439BB205
:10E060000380838B23F400631B041B0C83830B8AC4
:10E07000038230BD00234FF00702C3810282038078
:10E0800043808380C380038143818381704700BFC5
:10E0900000234381038043808380C3804FF00203C9
:10E0A0000381704721B103889BB243F0400304E031
:10E0B000038823F040031B041B0C0380704700BF40
:10E0C00021B1838B9BB243F4806304E0838B23F400
:10E0D00080631B041B0C8383704700BF0909012365
:10E0E00013FA01F189B21AB183889BB2194303E094
:10E0F00083889BB223EA0101818070471AB183882B
:10E100009BB2194303E083889BB223EA010181801B
:10E11000704700BF81817047808980B2704700BF1F
:10E120004FF6FF63994205D003889BB243F4807396
:10E13000038002E0038819400180704721B1838881
:10E140009BB243F0040304E0838823F004031B0420
:10E150001B0C8380704700BF038823F400631B04FB
:10E160001B0C038003889BB241EA030303807047C2
:10E1700003889BB243F480530380704721B1038826
:10E180009BB243F4005304E0038823F400531B04C0
:10E190001B0C0380704700BF012914BF008B808ACD
:10E1A00080B27047008A80B2704700BFB1F5804FDF
:10E1B00004D103889BB243F4804304E0038823F432
:10E1C00080431B041B0C0380704700BF0389194266
:10E1D0000CBF002001207047202906D10389038845
:10E1E0009BB243F04003038008E0402901D0082996
:10E1F00001D1038902E0C94389B20181704700BFA0
:10E20000012301F00F0213FA02F2B0F804C00089F2
:10E210001FFA8CFC80B2104006D009098B401CEA22
:10E22000030F0CBF00200120704700BF552906D105
:10E23000038903889BB243F0400303800DE0562915
:10E2400001D0532901D1038907E001F00F01012317
:10E2500013FA01F1C94389B201817047838BF0B58C
:10E2600023F47A6323F01F031B041B0C83834FF0FA
:10E27000020303840B89868B022B87B004460D466C
:10E28000B6B201D1002225E001A88F88FFF7E6FD94
:10E29000EB88002F0CBF01270227B3F5007F2989E7
:10E2A000019A06D1A3F5FB7353430902B3FBF1F3C3
:10E2B00005E00A2349015A434F43B2FBF7F3053304
:10E2C0000A229BB2B3FBF2F303F001021202C3F382
:10E2D0004F0392B2991E89B2FE2928BF002228BF9F
:10E2E0000223E98842EA03030B439BB223842B8871
:10E2F0006A8846EA0303A98843F4006313436A89E2
:10E300000B4313439BB2A38307B0F0BD08B5154B75
:10E3100098421BD003F57443984204D0A3F5784388
:10E3200098421DD10AE001214FF48050FFF708FE0A
:10E330004FF480500021FFF703FE11E04FF48040BE
:10E340000121FFF70BFE4FF4804006E04FF4004040
:10E350000121FFF703FE4FF400400021FFF7FEFD0F
:10E3600008BD00BF003C0040042804D1054B1A68DA
:10E3700042F0040203E0034B1A6822F004021A6020
:10E38000704700BF10E000E0014B5860704700BFCD
:10E3900010E000E0012804D1084B1A6842F00102A5
:10E3A00006E010F1020F05D1044B1A6822F00102B9
:10E3B0001A6002E0014B00229A60704710E000E012
:10E3C00020B1054B1A6842F0020203E0024B1A68C2
:10E3D00022F002021A60704710E000E0014B9868DA
:10E3E000704700BF10E000E0C308022B0BBF044BD6
:10E3F000034B1B68DB6833FA00F000F00100704744
:10E4000010E000E0038803F08F0303800388B1F875
:10E4100006C04A889BB243EA0C0313439BB20380B5
:10E420008B8883850B880385064B984203D003F5C0
:10E430000063984201D10B7A03864FF00103838277
:10E44000704700BF002C0140038C2DE9F04123F000
:10E4500001031B041B0C0384038C0A894C8823F0E2
:10E4600002031C4E14431B048288B1F806C0058BBE
:10E470001B0CA4B2B04244EA030392B20C88ADB2C2
:10E48000A0F834C003D006F50066B04218D18E89DA
:10E490004F89B1F80E804FF6F77C03EA0C0C4CEA7A
:10E4A000070748EA06064FF6FB73898847F6FF4CD4
:10E4B00002EA0C0C07EA0303B2B20B4342EA0C0275
:10E4C0004FF68F7105EA01012143828001830384A5
:10E4D000BDE8F081002C0140038C2DE9F04123F0D0
:10E4E00010031B041B0C0384028CB1F808C022F03B
:10E4F000200212048488120C4B8842EA0C1242EA71
:10E500000313A2B21B4C068BB1F806C0A0420D88C3
:10E51000B6B29BB2A0F838C003D004F50064A042A4
:10E520001BD1B1F80A804FF67F748F8903EA040487
:10E5300047F2FF3C02EA0C0C44EA0814CA894FF681
:10E54000BF73898804EA03034CEA870C43EA01138A
:10E550004CEA82023C469BB292B248F6FF7106EA50
:10E56000010141EA052189B2828001830384BDE86B
:10E57000F08100BF002C0140038C2DE9F04123F411
:10E5800080731B041B0C0384028CB1F808C022F4B6
:10E59000007212048488120C4B8842EA0C2242EA70
:10E5A0000323A2B21A4C868BB1F806C0A0420D8894
:10E5B000B6B29BB2A0F83CC003D004F50064A04200
:10E5C0001BD1B1F80A804FF2FF748F8903EA04046B
:10E5D00044F6FF7C02EA0C0C44EA0824CA894FF690
:10E5E000FF33898804EA03034CEA071C43EA01234A
:10E5F0004CEA02123C469BB292B24FF68F7106EA89
:10E6000001012943828081830384BDE8F08100BF3A
:10E61000002C0140038CF0B523F480531B041B0C29
:10E620000384B1F806C0078C0C8882880D89868B1C
:10E630004B88A0F840C0DFF848C0BFB2604592B236
:10E64000B6B203D00CF5006C604505D192048989FF
:10E65000920C42EA811292B24DF6FF7C07EA0C0C52
:10E6600048F6FF7106EA01014CEA053C41EA042143
:10E670004CEA033389B29BB2828081830384F0BD6C
:10E68000002C0140B1F802C00B888A884CEA0303D1
:10E69000B1F806C013430A8943EA0C03B1F80AC073
:10E6A00013438A8943EA0C0313439BB2A0F8443016
:10E6B000704700BF00234FF0FF3203724380828017
:10E6C0000380C380704700BF0023C3810380438061
:10E6D0008380C380038143818381704700234FF08F
:10E6E00001020381038043808280C380704700BFA2
:10E6F00000238381038043808380C380038143811F
:10E70000704700BF21B103889BB243F0010304E0CE
:10E71000038823F001039B059B0D0380704700BF16
:10E7200039B1B0F844306FEA43436FEA53439BB2C8
:10E7300003E0B0F844305B045B0CA0F84430704751
:10E740001AB183899BB2194303E083899BB223EA00
:10E7500001018181704700BF818270470A43A0F8A0
:10E76000482070471AB183899BB2194303E083891B
:10E770009BB223EA01018181704700BF038923F026
:10E7800007031B041B0C0381704700BFB0F808C0CF
:10E790005FFA8CFC41EA0C0C42EA0C0C4CEA032CAC
:10E7A0001FFA8CFCA0F808C0704700BF10B50446E3
:10E7B000FFF7ECFF23899BB243F48043238110BD14
:10E7C00010B50446FFF7E2FF238923F077031B040B
:10E7D0001B0C43F07703238110BD00BF01858282AB
:10E7E000704700BF038823F070039B059B0D41EA2F
:10E7F00003030380704700BF038923F070031B04E9
:10E800001B0C41EA03030381704700BF10B50446A7
:10E81000FFF7F2FF23899BB243F00703238110BD6A
:10E8200030B50489B0F818C0058C2CF4407CADB22A
:10E830002CF0030C24F007044FEA0C4C25F02205C1
:10E8400042EA050524044FEA1C4C45EA0315240C52
:10E850004CF4807C21434CF0010CADB20181A0F856
:10E8600018C0058430BD00BF038B23F070031B0468
:10E870001B0C41EA03030383704700BF038B23F49F
:10E88000E0431B041B0C43EA01239BB20383704744
:10E89000838B23F070031B041B0C41EA0303838367
:10E8A000704700BF838B23F4E0431B041B0C43EA37
:10E8B00001239BB28383704721B103889BB243F04D
:10E8C000800304E0038823F080039B059B0D0380F5
:10E8D000704700BF21B183889BB243F0040304E07A
:10E8E000838823F004031B041B0C8380704700BF44
:10E8F00021B183889BB243F0080304E0838823F0AE
:10E9000008031B041B0C8380704700BF21B1838860
:10E910009BB243F0010304E0838823F001031B044E
:10E920001B0C8380704700BF038B23F008031B047C
:10E930001B0C41EA03030383704700BF038B23F4DE
:10E9400000631B041B0C43EA01239BB20383704743
:10E95000838B23F008031B041B0C41EA030383830E
:10E96000704700BF838B23F400631B041B0C43EA36
:10E9700001239BB283837047038B23F004031B04A2
:10E980001B0C41EA03030383704700BF038B23F48E
:10E9900080631B041B0C43EA01239BB20383704773
:10E9A000838B23F004031B041B0C41EA03038383C2
:10E9B000704700BF838B23F480631B041B0C43EA66
:10E9C00001239BB283837047038B23F080031B04D6
:10E9D0001B0C41EA03030383704700BF038B5B04F6
:10E9E0005B0C43EA01239BB203837047838B23F0C4
:10E9F00080031B041B0C41EA03038383704700BFA1
:10EA0000838B5B045B0C43EA01239BB283837047D7
:10EA1000038C23F002031B041B0C41EA0303038451
:10EA2000704700BF038C23F008031B041B0C41EA52
:10EA300003030384704700BF038C23F020031B04EF
:10EA40001B0C43EA01139BB203847047038C23F031
:10EA500080031B041B0C43EA01139BB20384704721
:10EA6000038C23F400731B041B0C43EA01239BB2A9
:10EA700003847047038C23F400631B041B0C43EADC
:10EA800001239BB203847047038C23F400531B04BF
:10EA90001B0C43EA01339BB20384704701238B4074
:10EAA0008A40018C89B221EA03030384018C0A4362
:10EAB00092B20284704700BF04238B408A40018CCD
:10EAC00089B221EA03030384018C0A4392B20284CF
:10EAD000704700BF01238B40B0F820C010B51FFA6B
:10EAE0008CFC2CEA0303038409B1082909D11830EE
:10EAF000490844584FF68F7304EA030343504358C0
:10EB00000CE004391830C1F34E01445848F6FF7345
:10EB100004EA030343501202435892B243EA02024A
:10EB2000425010BD21B103889BB243F0020304E0C0
:10EB3000038823F002039B059B0D0380704700BFF1
:10EB400021B103889BB243F0040304E0038823F05F
:10EB500004039B059B0D0380704700BF21B1838890
:10EB60009BB243F0800304E0838823F080031B04FE
:10EB70001B0C8380704700BF038823F008039B05AC
:10EB80009B0D038003889BB241EA03030380704717
:10EB9000838823F070031B041B0C838083889BB243
:10EBA00041EA030383807047038923F007031B04B2
:10EBB0001B0C038103899BB241EA03030381704765
:10EBC000038923F080031B041B0C038103899BB280
:10EBD00041EA030303817047818470478185704750
:10EBE000818670470187704781877047A0F8401081
:10EBF000704700BF038B23F00C031B041B0C038323
:10EC0000038B9BB241EA030303837047038B23F416
:10EC100040631B041B0C0383038B9BB243EA012359
:10EC20009BB20383704700BF838B23F00C031B044C
:10EC30001B0C8383838B9BB241EA0303838370475E
:10EC4000838B23F440631B041B0C8383838B9BB255
:10EC500043EA01239BB28383704700BF0388DBB282
:10EC6000038003889BB241EA03030380704700BF1F
:10EC7000808E80B2704700BF008F80B2704700BFA7
:10EC8000808F80B2704700BFB0F8400080B27047FC
:10EC9000808C80B2704700BF008D80B2704700BF8B
:10ECA000038A19420CBF002001207047C94389B272
:10ECB00001827047038A828911EA030092B203D06D
:10ECC00011420CBF00200120704700BFC94389B228
:10ECD00001827047B0F820C010B52CF0010C4FEA4B
:10ECE0000C4C4FEA1C4CA0F820C0048BB0F820C09C
:10ECF000A4B21FFA8CFC24F0F30442EA04042CF0C2
:10ED0000020C44EA03144CF0010C4CEA010CA4B2CE
:10ED10000483A0F820C010BDB0F820C010B52CF0BE
:10ED2000100C4FEA0C4C4FEA1C4CA0F820C0B0F875
:10ED300018C0048C2CF4407CA4B24FEA0C5C4FEA5F
:10ED40001C5C24F020044CEA022C44F010044CEA31
:10ED5000033C44EA01141FFA8CFCA4B2A0F818C0CA
:10ED6000048410BD38B50D46602D1146044603D10C
:10ED70000122FFF7D1FF02E00122FFF7ABFF294696
:10ED80002046FFF739FD23899BB243F00703238117
:10ED900038BD00BFF8B50C46A2884988B4F800C059
:10EDA000054600290CBF02270027012A0CBF0226B6
:10EDB00001262389BCF1000F10D1FFF78BFF2846F5
:10EDC000E188FFF717FF2846394632462389FFF7C7
:10EDD000A3FF2846E188FFF719FF0FE0FFF79CFF2C
:10EDE0002846E188FFF712FF284639463246238934
:10EDF000FFF770FF2846E188FFF7FCFEF8BD00BF73
:10EE000038B50B880C4605464BB94988A28823893A
:10EE1000FFF760FF2846E188FFF7ECFE53E0042B84
:10EE200009D14988A2882389FFF776FF2846E1881F
:10EE3000FFF7ECFE47E0082BB1F802C0B1F804E0A0
:10EE4000098920D1028C22F480721204120C0284EF
:10EE5000838B028C9BB292B223F0F30322F40072F4
:10EE600043EA011142EA0C2C89B21FFA8CFC41EAF8
:10EE70000E0E4CF4807CA0F81CE0A0F820C0E188C5
:10EE8000FFF7D2FE1FE0028C22F480521204120C13
:10EE90000284838B028C23F4407392B21B051B0DFA
:10EEA00022F4005243EA0E2342EA0C3C43EA0133C7
:10EEB0001FFA8CFC9BB24CF4805C8383A0F820C0CA
:10EEC000E188FFF7BDFE38BD08B52D4B984237D01D
:10EED0000BD8A3F50063984226D003F580639842CF
:10EEE00028D0B0F1804F4AD118E0264B984233D059
:10EEF00004D8A3F58063984241D127E0224B984281
:10EF000004D003F50063984239D12EE04FF400603D
:10EF10000121FFF715F84FF400602DE001200146B4
:10EF2000FFF71CF801201CE002200121FFF716F872
:10EF3000022016E004200121FFF710F8042010E061
:10EF400008200121FFF70AF808200AE0102001211B
:10EF5000FFF704F8102004E020200121FEF7FEFF57
:10EF600020200021FEF7FAFF09E04FF400500121B4
:10EF7000FEF7E6FF4FF400500021FEF7E1FF08BD69
:10EF8000000C004000140040002C0140002383814D
:10EF90004FF416528380C38003814FF00C0302604C
:10EFA000438170470A8810B54C88B1F804C0038AC1
:10EFB000C98844EA020242EA0C0223F470630A435D
:10EFC0001B041B0C92B242EA0303038210BD00BF74
:10EFD0000023C380038043808380704721B18389ED
:10EFE0009BB243F4005304E0838923F400531B04D1
:10EFF0001B0C8381704700BF01F01F034FF0010C11
:10F00000C1F3421161450CFA03F301D10C3004E065
:10F01000022901D1103000E014301AB1026842EA2E
:10F02000030302E0026822EA03030360704700BFA3
:10F030001AB1838A9BB2194303E0838A9BB223EA05
:10F0400001018182704700BF038A23F00F031B0474
:10F050001B0C0382038A9BB241EA030303827047BD
:10F06000838923F400631B041B0C838183899BB277
:10F0700041EA03038381704721B183899BB243F046
:10F08000020304E0838923F002031B041B0C838129
:10F09000704700BF038A23F020031B041B0C03826C
:10F0A000038A9BB241EA03030382704721B1038ABA
:10F0B0009BB243F4804304E0038A23F480431B049F
:10F0C0001B0C0382704700BFC905C90D81807047C2
:10F0D0008088C005C00D704783899BB243F001034F
:10F0E00083817047038BDBB20383038B9BB243EABC
:10F0F00001230383704700BF038B03F47F43038323
:10F10000038B9BB241EA03030383704721B1838AD7
:10F110009BB243F0200304E0838A23F020031B0406
:10F120001B0C8382704700BF21B1838A9BB243F0DE
:10F13000100304E0838A23F010031B041B0C83825A
:10F14000704700BF21B1838A9BB243F0080304E0FB
:10F15000838A23F008031B041B0C8382704700BFC3
:10F16000838A23F004031B041B0C8382838A9BB2D3
:10F1700041EA03038382704721B1838A9BB243F043
:10F18000020304E0838A23F002031B041B0C838226
:10F19000704700BF038819420CBF00200120704750
:10F1A000C94389B2018070474FF0010CC1F342128C
:10F1B00001F01F0362450CFA03F301D1828903E0D9
:10F1C000022A0CBF028A828A92B21340028892B24B
:10F1D0000BB9184607E0090A012313FA01F111429D
:10F1E0000CBF002001207047090A01238B40DB433C
:10F1F0009BB20380704700BF038ACA8823F4405340
:10F200001B041B0C1343038283898A8830B5044690
:10F2100008890D4623F4B053498940EA020223F0DD
:10F220000C030A431B041B0C92B242EA0303A381A2
:10F23000A38AAA8923F440731B041B0C134387B0D1
:10F24000A38201A8FEF70AFE0E4B2A689C420CBF5F
:10F25000049B039B1921594392006423B1FBF2F1F3
:10F26000B1FBF3F21201100903FB10110901323155
:10F27000B1FBF3F303F00F0343EA020292B22281DF
:10F2800007B030BD0038014008B5214B98422BD063
:10F2900008D8A3F50063984216D003F5806398421E
:10F2A00034D119E01B4B984226D003F568439842AD
:10F2B0002CD101214FF48040FEF742FE4FF48040F4
:10F2C0000021FEF73DFE21E04FF400300121FEF762
:10F2D00045FE4FF4003016E04FF480200121FEF788
:10F2E0003DFE4FF480200EE04FF400200121FEF798
:10F2F00035FE4FF4002006E04FF480100121FEF7A8
:10F300002DFE4FF480100021FEF728FE08BD00BF3F
:10F31000004C004000500040684620F007018D4638
:10F3200001B5002303E00B495958995004330A4AA8
:10F330000A4998188842F6D3094B02E0002243F8A4
:10F34000042B084A9342F9D3F4F746FFBDE8014085
:10F3500085467047902901080000002030020020F7
:10F3600030020020600E002010B5074C20B9226842
:10F370004FF00103138205E0044B1B681B6898479C
:10F3800020680A3010BD00BFF80D0020B40D002029
:10F3900010B50A4B0A4A1B685178DA7891420AD3B1
:10F3A000997841B99C8834B99A72064B1B685B689E
:10F3B0009847204600E0022010BD00BFF80D002055
:10F3C00004010020B40D002010B5074C20B92268BC
:10F3D0004FF00103138205E0044B1B689B689847BC
:10F3E00020680C3010BD00BFF80D0020B40D0020C7
:10F3F00038B50E4C0E4B22681B68D1789B6950794A
:10F40000984723689A7A7AB170B91A7962B99D7867
:10F4100055B9084B1B68DB6898472368284659791B
:10F42000DA78D9721A7300E0022038BDF80D002096
:10F43000900D0020B40D002008B50246244B20B9E1
:10F440001B684FF00201198240E0224A4FF0000190
:10F450001B681180197811F07F0113D15B7A13F0CA
:10F46000200F03D0117841F00201117013F0400F0A
:10F47000184B15BF1A781A7822F0010242F00102E7
:10F480001A701EE0012921D0022901D000221DE0BE
:10F49000597911F0800F01F00F0306D00E4951F891
:10F4A000233003F03003102B06E00B4951F82330D2
:10F4B00003F44053B3F5805F03D1137843F00103A5
:10F4C0001370064B1B681B699847024A104608BD1B
:10F4D000F80D0020580E0020005C0040B40D002004
:10F4E00010B51E4B19684A7912F0800F22F0800384
:10F4F00005D01B4850F8230000F0300004E0184805
:10F5000050F8230000F44050164C94F800C06345B6
:10F5100022D24C8804BBF8B1897AE9B112F0800F8D
:10F5200009D00F4948F6BF7251F8230000EA0202E1
:10F5300082F0100208E00A494BF68F7251F823005E
:10F5400000EA020282F4805241F82320064B1B6835
:10F550009B699847002000E0022010BDF80D0020B4
:10F56000005C004004010020B40D002008B5064BEB
:10F570001B685A7A42F020025A72044B1B68DB69FE
:10F580009847002008BD00BFF80D0020B40D0020F2
:10F59000054B1A68538A18B98988CB1A138201E07F
:10F5A00008681818704700BFF80D002030B50E4BE2
:10F5B0001C78002310E05FFA83FC4FEA8C0202F112
:10F5C000804202F5B842156848F68F7105EA0101DC
:10F5D00041EA0C0111600133A342ECD3034B40F02C
:10F5E0008000186030BD00BF040100204C5C00406A
:10F5F000704700BF08B50C4B002093F82C1000F0AA
:10F600004FFE0A4B1B68187A082807D1084B4FF4A5
:10F6100080521A80074B4FF010021A80092814BF3D
:10F620000020012008BD00BF80000020F80D002050
:10F630005A0E00205C0E002070B52D4B1C68237AFA
:10F64000032B01D0052B46D1A369228AABB1A2B10D
:10F65000A58A954228BF154628469847228A638A7C
:10F66000521BEB18064622826382002000F0E8FD60
:10F670002A460146304600F0FBFB238A5BB11D4B56
:10F680004FF4405200201A80014600F0E7FD1A4B6B
:10F690004FF030021A80A28A238A9A4203D8144B70
:10F6A00003221B6803E0124A1BB1136805221A7279
:10F6B0000DE0126806211172104A1168104A89B2D1
:10F6C0008A18520013600C4B4FF030021A80084B1E
:10F6D0001B681B7A06E0072B03D10A4B1B68DB680B
:10F6E00098470823024A12681372FFF783FF70BD20
:10F6F000F80D00205A0E00205C0E0020505C0040E7
:10F7000002300020900D0020F8B5244B1C68238A9D
:10F71000267ABBB9042E15D1214822490278012A44
:10F720000BD1214C214A24680370A0B282185200E8
:10F7300013604FF030020A802BE04FF010030B8073
:10F74000072626E0A68AA2699E4234BF35461D469A
:10F750002846B34294BF042602269047074600205D
:10F7600000F060FD2A460146384600F069FB294654
:10F77000002000F073FD638A228AEB186382094B34
:10F78000551B4FF0300225821A80094B4FF440522E
:10F790001A80024B1B681E72F8BD00BFF80D0020D6
:10F7A000900600205C0E0020505C004002300020DB
:10F7B0005A0E002008B5144B1B681A7A022A01D091
:10F7C000042A05D1FFF7A0FF0F4B1B681B7A14E03A
:10F7D000062A11D15A78052A0AD11A7812F07F0F19
:10F7E00006D1D878FFF7E2FE084B1B681B6A9847E2
:10F7F000074B1B689B6898470823034A12681372DB
:10F80000FFF7F8FE08BD00BFF80D0020B40D002082
:10F81000900D002038B5324B1B68187810F07F002F
:10F8200004D15A7A22F020025A7258E0022855D1A7
:10F830005A88002A52D11A79002A4FD15A7912F0E7
:10F84000800F22F0800405D0264951F8241001F0E1
:10F85000300104E0234951F8241001F440512248BA
:10F86000007884423AD2002938D09B7A002B35D0D8
:10F8700012F0800F0FD01B4B53F8243003F03003ED
:10F88000102B25D1E4B2204600F082FC2046302126
:10F8900000F05EFB1CE0134D55F8243003F4405398
:10F8A000B3F5805F14D134B9104B204693F82C1077
:10F8B00000F0F6FC02E0204600F056FC55F824204B
:10F8C0004BF68F7302EA030383F4405345F8243068
:10F8D000074B1B685B699847002000E0022038BD99
:10F8E000F80D0020005C0040040100208000002092
:10F8F000B40D0020F7B58D4B8D4E1A6835688D4BD1
:10F9000092B2D3182A7A5B00092A1B681BD09BB2DB
:10F9100003F1005303F540535B001C4614F8012B20
:10F9200003F10A072A705B786B70B4F8030000F0EB
:10F9300063FE6880B4F80700346800F05DFEA080C4
:10F9400033687F88DF807A4C01212368DA88197256
:10F950005D78002A62D11A7812F07F022ED1092D2B
:10F9600002D1FFF715FD3BE0052D0DD193F90320E2
:10F97000002A4EDB9A78002A4BD19A88002A48D177
:10F980009B7A002B37D044E0032D0BD1DA78012A83
:10F9900027D19A882ABB5B7A13F0200F21D0FFF77A
:10F9A000E5FD1DE0012D1CD1DA78012A19D19A88D4
:10F9B000BAB95B7A13F0200F13D00AE0012A04D100
:10F9C0000B2D0ED1FFF714FD0AE0022A09D1012DFB
:10F9D00002D1FFF71FFF03E0032D02D1FFF780FDE7
:10F9E00048B1554B28461B685B699847032801D1ED
:10F9F00009230FE068B94D4A504B12684FF03001AF
:10FA000092B2D3185B0000221A604D4B1980062376
:10FA100000E00823464A12681372E3E0062D18D16D
:10FA20001A7812F07F0F40F097809B78012B03D15A
:10FA3000414B1B68DB696EE0022B03D13E4B1B6818
:10FA40001B6A68E0032B40F087803B4B1B685B6AB6
:10FA500061E0002D3CD1598800297DD15A6822F4FB
:10FA60007F42B2F5003F77D11A7812F07F0203D1BE
:10FA70009B88002B70D129E0012A0BD158792E4B9D
:10FA80001B689B699847002866D123689B7A002BE6
:10FA900062D01BE0022A5FD15B7913F0800F03F084
:10FAA0000F0205D0274951F8221001F0300104E07F
:10FAB000244951F8221001F4405123480078824231
:10FAC0004AD213F0700F47D1002945D01F4B23E0D5
:10FAD000082D05D11B7813F07F0F3DD11C4B1BE087
:10FAE0000A2D39D11A7802F07F02012A34D19A7A8C
:10FAF000002A31D0598800292ED15A6822F47F4239
:10FB0000B2F5803F28D158790B4B1B689B69984709
:10FB100010BB104B00E0FBB1054A4FF0000112682A
:10FB20000020936151829847002020E0505C004003
:10FB3000F80D002004300020900D0020023000203D
:10FB40005C0E0020005C00400401002039F4000835
:10FB500069F30008C9F30008244C254B22681B6890
:10FB600050781B699847032801D1236806E01F4B92
:10FB70004FF6FF711B681A8A8A4201D1092203E0FD
:10FB8000022800D012B908221A722BE093F9001053
:10FB9000002921DAD98801910198824202D9019A7B
:10FBA0001A8211E08A420FD21149096891F82C108B
:10FBB0008A4201D2002105E092FBF1F001FB102204
:10FBC00012B901210B4A1170094A126892F82C20CF
:10FBD0009A82FFF799FD05E003221A72064B4FF453
:10FBE00040521A80FFF706FDFEBD00BFF80D002051
:10FBF000900D0020900600205A0E0020074A022196
:10FC000008B5074811720749074B086007490A60A1
:10FC1000074A13601B68984708BD00BF980D002075
:10FC200008010020B40D002080000020F80D002005
:10FC3000900D002008B529E047F6FF70086019888C
:10FC400001F00F018B0003F18043117003F5B843FD
:10FC5000196889B211F4004F09D0186840F68F7105
:10FC600000EA0101196012780E4B013A0BE011F025
:10FC7000800F0BD0186848F60F7100EA0101196077
:10FC80001278094B013A53F8223098470749084B3C
:10FC90000868084A80B21880188800B20028CBDBB8
:10FCA00008BD00BFE8000020CC000020445C0040FC
:10FCB0008E0D0020940D0020F8B59AE047F6FF76EF
:10FCC0001E601688564F06F00F06B30003F18043FE
:10FCD00003F5B8433E70002E64D127682668236878
:10FCE00007F4405C03EA000080F4005020602368C1
:10FCF00006F0300003EA010181F020012160138841
:10FD0000484A13F0100F1080A5F800C004D02368F3
:10FD10009BB213F0800F08D0226848F60F7302EAF6
:10FD200003032360FFF746FD16E013F4006F08D0CD
:10FD3000226840F68F7302EA03032360FFF7DAFDBF
:10FD40000AE013F4004F54D0226840F68F7302EAA1
:10FD500003032360FFF770FC21682A884BF68F733A
:10FD600001EA030312F4805F18BF83F4805312F496
:10FD7000005F2D4A18BF83F400531360294B1168AC
:10FD80001A8848F6BF7301EA030312F0100F18BF78
:10FD900083F0100312F0200F234A18BF83F02003D2
:10FDA00013603BE01C68A4B214F4004F0BD0196838
:10FDB00040F68F7201EA02021A603A781B4B013A50
:10FDC00053F82230984714F0800F12D0144948F6A7
:10FDD0000F720B789B0003F1804303F5B84318685A
:10FDE00000EA02021A600A78114B013A53F82230F5
:10FDF0009847104B104A1D680B4C1FFA85FCA2F85F
:10FE000000C0B2F800C04BF68F700FFA8CFCBCF14A
:10FE1000000F48F6BF71094DFFF650AFF8BD00BFA7
:10FE2000940D00205C0E0020005C0040E8000020E3
:10FE3000CC000020445C00408E0D00205A0E0020B3
:10FE400001F10051013201F5405110B5490052084D
:10FE5000002308E010F803C06478013A4CEA042C4F
:10FE600021F813C00233C418002AF3D110BD00BF1B
:10FE700001F10051013201F5405110B5490052081D
:10FE8000002304E031F81340013AC4520233002A3F
:10FE9000F8D110BD014B1860704700BF405C0040B6
:10FEA000014B186880B27047405C0040014B1860FD
:10FEB000704700BF445C0040014B186880B2704737
:10FEC000445C0040014B186880B27047485C0040B9
:10FED000014B1860704700BF4C5C0040014B186834
:10FEE00080B270474C5C00404FF6F873024A00EA5B
:10FEF00003031360704700BF505C0040014B18685B
:10FF000080B27047505C0040014B43F820107047AE
:10FF1000005C0040024B53F8200080B2704700BFE5
:10FF2000005C0040054B10B553F8204048F68F1296
:10FF300004EA02020A4343F8202010BD005C00409E
:10FF4000024B53F8200000F4C0607047005C004092
:10FF50000A4B10B553F8202048F6BF7402EA040497
:10FF600011F0100F18BF84F0100411F0200F18BF0B
:10FF700084F0200443F8204010BD00BF005C004026
:10FF80000A4B10B553F820204BF68F7402EA040494
:10FF900011F4805F18BF84F4805411F4005F18BF1F
:10FFA00084F4005443F8204010BD00BF005C0040C2
:10FFB00038B50D460446FFF7ADFF012D02D120F400
:10FFC000805003E0022D04D120F01000014B43F8D3
:10FFD000240038BD005C0040024B53F8200000F0C4
:10FFE00030007047005C0040024B53F8200000F4E2
:10FFF00040507047005C0040054B48F6BF7253F814
:020000040801F1
:10000000201001EA020282F0300243F820207047FB
:10001000005C0040054B4BF68F7253F8201001EA4C
:10002000020282F4405243F820207047005C0040F6
:10003000054B48F68F6253F8201001EA020242F4A1
:10004000807243F820207047005C0040044B48F663
:100050008F6253F8201001EA020243F82020704713
:10006000005C0040044B48F68F6253F8201001EA10
:10007000020243F820207047005C0040054B48F620
:100080008F6253F8201001EA020242F4807243F8B2
:1000900020207047005C0040054B48F68F6253F803
:1000A000201001EA020242F4807243F820207047D7
:1000B000005C0040044B48F68F6253F8201001EAC0
:1000C000020243F820207047005C0040044B53F8C4
:1000D000200000F03000102814BF002001207047DD
:1000E000005C0040054B53F8200000F44050B0F590
:1000F000805F14BF00200120704700BF005C0040FB
:10010000044B40F68F7253F8201001EA020243F8C4
:1001100020207047005C0040044B48F60F7253F8F3
:10012000201001EA020243F820207047005C0040E2
:10013000054B48F68F7253F8201001EA020242F490
:10014000804243F820207047005C0040054B48F691
:100150008F7253F8201001EA020242F0400243F885
:1001600020207047005C0040084B53F8202012F418
:10017000804F09D053F8201048F68F7201EA02022E
:1001800042F4804243F82020704700BF005C0040EA
:10019000084B53F8202012F0400F09D053F82010DC
:1001A00048F68F7201EA020242F0400243F8202032
:1001B000704700BF005C0040054B10B553F820406D
:1001C00048F68F7204EA02020A4343F8202010BD69
:1001D000005C0040024B53F8200000F00F00704715
:1001E000005C0040064B49081B6849009BB203EBCA
:1001F000C00303F1005303F540535B0019607047DF
:10020000505C0040054A064B1268490892B202EB66
:10021000C002D3185B00490019607047505C004071
:1002200004300020054B1B689BB203EBC00303F1B5
:10023000005303F540535B0018887047505C004042
:10024000044A054B126892B202EBC002D3185B005D
:1002500018887047505C004004300020044A054B69
:10026000126892B202EBC002D3185B0019607047AB
:10027000505C0040023000203E2909D94B0911F0A2
:100280001F0F01D1013B9BB29B0243F4004305E0E9
:100290004B0811F0010F18BF01339B020360704738
:1002A0000D4A0E4B126892B2D31803EBC0035B00E9
:1002B0003E2909D94A0911F01F0F01D1013A92B222
:1002C000920242F4004205E04A0811F0010F18BF03
:1002D000013292021A607047505C004006300020E4
:1002E000054A064B126892B202EBC002D3185B00BB
:1002F00018688005800D7047505C00400230002077
:10030000054A064B126892B202EBC002D3185B009A
:1003100018688005800D7047505C00400630002052
:100320000C4B30B51D681C68C0001FFA85FC844466
:10033000A4B2094B00190CF1005CC3180CF5405C29
:10034000490852084FEA4C0049005B005200016026
:100350001A6030BD505C004004300020064B490854
:100360001B6849009BB203EBC00303F1005303F584
:1003700040535B0019607047505C0040054A064BD3
:100380001268490892B202EBC002D3185B00490020
:1003900019607047505C004004300020054B1B681A
:1003A0009BB203EBC00303F1005303F540535B0022
:1003B00018887047505C0040044A054B126892B29E
:1003C00002EBC002D3185B0018887047505C0040F5
:1003D00004300020012910B524D1254B25491B6884
:1003E000C0009BB2591809184B003E2A09D951097F
:1003F00012F01F0F01D1013989B2890241F4004185
:1004000005E0510812F0010F18BF0131890219608F
:100410001749194B096889B2CB18181840003E2AB1
:100420001ED913E0022922D1114BC0001C681B68A1
:10043000A4B21FFA83FC0F490F4B844400194118E2
:10044000634449005B000A601A6010E0530912F02F
:100450001F0F01D1013B9BB29B0243F4004305E017
:10046000530812F0010F18BF01339B02036010BD47
:10047000505C0040023000200630002001291BD1D2
:100480001349144B096889B2CB1803EBC000400034
:100490003E2A09D9530912F01F0F01D1013B9BB22B
:1004A0009B0243F4004305E0530812F0010F18BF0C
:1004B00001339B0203600AE0022908D10449054B7D
:1004C000096889B201EBC000C3185B001A6070476D
:1004D000505C00400230002001291BD11349144B0D
:1004E000096889B2CB1803EBC00040003E2A09D945
:1004F000530912F01F0F01D1013B9BB29B0243F441
:10050000004305E0530812F0010F18BF01339B02AE
:1005100003600AE0022908D10449054B096889B241
:1005200001EBC000C3185B001A607047505C0040CC
:1005300006300020054A064B126892B202EBC00258
:10054000D3185B0018688005800D7047505C004030
:1005500002300020054A064B126892B202EBC0023C
:10056000D3185B0018688005800D7047505C004010
:10057000063000200D4BC00019680D4A89B24118A1
:100580008A185200128812F47C4F01D001200CE02E
:100590001A68084B92B28018C3185B00188880054F
:1005A000800D002814BF022000207047505C0040DE
:1005B0000630002002300020012909D10B4A48F6FC
:1005C0008F7352F8201001EA030343F040030AE05E
:1005D00002290AD1054A48F68F7352F8201001EA21
:1005E000030343F4804342F820307047005C00402E
:1005F00041EA0020704700BF030AC0B243EA00206E
:10060000704700BF08B500220A2300F045F808BD76
:1006100008B500210A2200F0DFF808BDF0B4037825
:10062000002B2DD040F23412C2F20002156802E015
:1006300010F8013FEBB15A1903F12004527812F07F
:1006400001070A7808BF1C4601F10101561C9446B7
:10065000AE5D16F0010F18BF02F1200C6445E7D023
:1006600007B1203316F0010F18BF2032981AF0BCE2
:1006700070470A786F78561C07F00107AE5DEFE708
:1006800040F234100A78C2F20000561C05686F78F8
:10069000AE5D07F00107E3E72DE9F04F40F23415B6
:1006A000C2F2000583B00C461F46D5F800800E4606
:1006B0000190009216F8015B08EB050393F801B076
:1006C0001BF0080BF6D12D2D65D02B2D08BF16F889
:1006D000015BD7F1010338BF0023102F14BF1A4666
:1006E00043F0010232B1302D66D01BB1302D0CBF6A
:1006F00008270A27BBF1000F394614BF4FF0004905
:100700006FF00049484600F059FC48468A46394691
:1007100000F026FB00218C4608EB0502A5F1300312
:10072000527812F0040F08D112F0030F20D012F00B
:10073000010F14BF37235723EB1A9F4218DD84455E
:1007400094BF0022012252EAD1714FF0FF310CD147
:10075000844514BF002201225345D4BF002202F079
:10076000010212B907FB0C3C012116F8015BD3E72B
:10077000B1F1FF3F14D0BBF1000F09D16046009BDF
:100780001BB101B1741E009A146003B0BDE8F08F74
:10079000CCF10000F3E716F8015B4FF0010B98E78E
:1007A000019ABBF1000F4FF0220314BF4FF000403D
:1007B0006FF000401360E2E73278782A14BF00211E
:1007C0000121582A14BF0A4641F00102002A8CD0A8
:1007D0007578102702368DE710B540F23814C2F252
:1007E00000048C461346014662462068FFF754FF1A
:1007F00010BD00BF2DE9F0438BB006460F4600F058
:100800007BF840F22C24C2F2000494F90030B3F1DA
:10081000FF3F8046894638D03046394600F084FA9A
:100820000546002831D1304639460022002301F028
:100830001DF8002829D1247842F68013C0F6010360
:1008400008950193CDE90267CDE90467002C21D01A
:1008500040F200030022CFF6F0733046CDE90623C4
:1008600039460022002300F0D9FF002822D00223BD
:1008700000939C4234D0684600F064FA00282FD0E0
:10088000089B002B27D1DDE90689404649460BB07D
:10089000BDE8F0834FF6FF734FF06042CCF2EF7388
:1008A0003046CDE9062339460022002300F0B6FF8A
:1008B0000028DCD10123022C009316D0684600F0FA
:1008C00041FA90B142F68410C0F6010000F03CFA03
:1008D000CDE90601D4E700F03DFA089B0360D2E7BA
:1008E00000F038FA22230360CAE700F033FA21232C
:1008F0000360E7E700000000B1F5801F0B462DE91B
:10090000F04F804687B0894604460D463EDB4FF6E1
:10091000FF720026C7F6EF72934251DC23F07F444A
:1009200045F6647C24F47004C0F2090CA44440F23F
:100930000002A6F57E760CF4801C073EC3F6F0722A
:100940008CEA020206EB235640F20003404642EADC
:100950000401C3F6F073002206EB1C5600F042FBC4
:10096000A31C23F07F4323F47003022B80468946A7
:100970002FDC0022002300F051FF002800F0CA8085
:10098000002E40F07C81002000211FE021F0004378
:10099000034300F0B5800029C0F2468140F2000315
:1009A0000022C4F250336FF0350600F0CFFC4FF652
:1009B000FF72C7F6EF720B46804693428946ADDD63
:1009C0004046494642464B4600F00EFB07B0BDE8A4
:1009D000F08F00224FF0804300F006FB4EF6863584
:1009E000CFF6F975651902460B464046494600F0B8
:1009F000D7FDCDE90201304600F042FCCDE904010B
:100A0000DDE9020102460B4600F0A0FC02460B465F
:100A1000CDE9000100F09AFCA7A3D3E900238246A8
:100A20008B4600F093FCA6A3D3E9002300F0DCFA88
:100A300052465B4600F08AFCA3A3D3E9002300F0F2
:100A4000D3FA52465B4600F081FCA1A3D3E9002310
:100A500000F0CAFADDE9002300F078FC9EA3D3E998
:100A60000023CDE900015046594600F06FFC9CA3DD
:100A7000D3E9002300F0B8FA52465B4600F066FC6A
:100A800099A3D3E9002300F0AFFA52465B4600F089
:100A90005DFC0B460246DDE9000100F0A5FA4BF6CD
:100AA0005103C0F206031B1B43EA0505002D8246D5
:100AB0008B4656DD40F200030022C3F6E073404649
:100AC000494600F043FC42464B4600F03FFC0446DA
:100AD0000D46002E75D152465B4600F085FADDE9E1
:100AE000022300F033FC02460B462046294600F064
:100AF00079FA02460B464046494600F073FA65E72C
:100B000040F20001002000220023CCF2503100F01E
:100B100047FD5BE742464B464046494600F016FC1F
:100B200073A3D3E9002304460D464046494600F02E
:100B30000DFC40F200030022C3F6E07300F054FA0B
:100B400002460B462046294600F000FC04460D46AE
:100B5000002E72D14046494622462B4600F042FA0A
:100B600034E7002E00F0D48063A3D3E90023DDE94D
:100B7000040100F0EBFB52465B4606460F4640463A
:100B8000494600F02FFADDE9022300F0DFFB5CA309
:100B9000D3E9002304460D46DDE9040100F0D6FB4D
:100BA00002460B462046294600F01EFA42464B46B6
:100BB00000F018FA02460B463046394600F012FAA9
:100BC00004E74DA3D3E90023DDE9040100F0BEFBF7
:100BD00052465B46CDE900012046294600F004FA62
:100BE000DDE9022300F0B2FB47A3D3E90023064668
:100BF0000F46DDE9040100F0A9FB02460B46304632
:100C0000394600F0F1F902460B462046294600F02D
:100C1000E9F942464B4600F0E5F902460B46DDE9AC
:100C2000000100F0DFF9D1E602460B4600F0DAF9E8
:100C30000022002300F0B4FCC8E6304600F020FBA0
:100C40002DA3D3E9002306460F4600F07FFB2CA31B
:100C5000D3E9002382468B463046394600F076FBC6
:100C600022462B4600F0C0F942464B4600F0BAF946
:100C700002460B465046594600F0B4F9A6E6304607
:100C800000F0FEFA1CA3D3E9002306460F4600F04D
:100C90005DFB1DA3D3E9002304460D4630463946CB
:100CA00000F054FB02460B462046294600F09CF912
:100CB0008CE600BFAFF3008044523EDF12F1C23F2A
:100CC000DE03CB966446C73F599322942449D23F12
:100CD000935555555555E53F9FC678D0099AC33F62
:100CE000AF788E1DC571CC3F04FA97999999D93F79
:100CF000555555555555D5BF0000E0FE422EE63FEF
:100D0000763C7935EF39EABD763C7935EF39EA3D05
:100D100002460B464046494600F064F9DDE90223ED
:100D200000F014FBE5E600BF02464042104321F00C
:100D3000004141EAD070C0F1FE4000F57000C00FE4
:100D4000704700BF0020704740F200010020C7F646
:100D5000F871704740F23813C2F200031868704708
:100D60004A1E08BF7047C0F02481884240F21681B5
:100D7000114200F01781B0FA80F3B1FA81F2A2EBD0
:100D80000303C3F11F0304A202EB03134FF000029D
:100D90009F4600BFAFF30080B0EBC17F00BF42EBC6
:100DA000020228BFA0EBC170B0EB817F00BF42EB15
:100DB000020228BFA0EB8170B0EB417F00BF42EB85
:100DC000020228BFA0EB4170B0EB017F00BF42EBF5
:100DD000020228BFA0EB0170B0EBC16F00BF42EB75
:100DE000020228BFA0EBC160B0EB816F00BF42EBF5
:100DF000020228BFA0EB8160B0EB416F00BF42EB65
:100E0000020228BFA0EB4160B0EB016F00BF42EBD4
:100E1000020228BFA0EB0160B0EBC15F00BF42EB54
:100E2000020228BFA0EBC150B0EB815F00BF42EBD4
:100E3000020228BFA0EB8150B0EB415F00BF42EB44
:100E4000020228BFA0EB4150B0EB015F00BF42EBB4
:100E5000020228BFA0EB0150B0EBC14F00BF42EB34
:100E6000020228BFA0EBC140B0EB814F00BF42EBB4
:100E7000020228BFA0EB8140B0EB414F00BF42EB24
:100E8000020228BFA0EB4140B0EB014F00BF42EB94
:100E9000020228BFA0EB0140B0EBC13F00BF42EB14
:100EA000020228BFA0EBC130B0EB813F00BF42EB94
:100EB000020228BFA0EB8130B0EB413F00BF42EB04
:100EC000020228BFA0EB4130B0EB013F00BF42EB74
:100ED000020228BFA0EB0130B0EBC12F00BF42EBF4
:100EE000020228BFA0EBC120B0EB812F00BF42EB74
:100EF000020228BFA0EB8120B0EB412F00BF42EBE4
:100F0000020228BFA0EB4120B0EB012F00BF42EB53
:100F1000020228BFA0EB0120B0EBC11F00BF42EBD3
:100F2000020228BFA0EBC110B0EB811F00BF42EB53
:100F3000020228BFA0EB8110B0EB411F00BF42EBC3
:100F4000020228BFA0EB4110B0EB011F00BF42EB33
:100F5000020228BFA0EB0110B0EBC10F00BF42EBB3
:100F6000020228BFA0EBC100B0EB810F00BF42EB33
:100F7000020228BFA0EB8100B0EB410F00BF42EBA3
:100F8000020228BFA0EB4100B0EB010F00BF42EB13
:100F9000020228BFA0EB0100104670470CBF0120E1
:100FA00000207047B1FA81F2C2F11F0220FA02F06C
:100FB000704708B14FF0FF3000F00EB80029F8D0AC
:100FC0002DE90340FFF7CCFEBDE8064002FB00F32D
:100FD000A1EB0301704700BF704700BF81F00041E3
:100FE00002E000BF83F0004330B54FEA41044FEA0E
:100FF000430594EA050F08BF90EA020F1FBF54EAA9
:10100000000C55EA020C7FEA645C7FEA655C00F044
:10101000E2804FEA5454D4EB5555B8BF6D420CDD15
:101020002C4480EA020281EA030382EA000083EA98
:10103000010180EA020281EA0303362D88BF30BD38
:1010400011F0004F4FEA01314FF4801C4CEA11318E
:1010500002D0404261EB410113F0004F4FEA0333ED
:101060004CEA133302D0524263EB430394EA050F78
:1010700000F0A780A4F10104D5F1200E0DDB02FAE7
:101080000EFC22FA05F2801841F1000103FA0EF27B
:10109000801843FA05F359410EE0A5F120050EF141
:1010A000200E012A03FA0EFC28BF4CF0020C43FA72
:1010B00005F3C01851EBE37101F0004507D54FF07F
:1010C000000EDCF1000C7EEB00006EEB0101B1F5CF
:1010D000801F1BD3B1F5001F0CD349085FEA300015
:1010E0004FEA3C0C04F101044FEA445212F5800F20
:1010F00080F09A80BCF1004F08BF5FEA500C50F1BD
:10110000000041EB045141EA050130BD5FEA4C0C9F
:10111000404141EB010111F4801FA4F10104E9D128
:1011200091F0000F04BF01460020B1FA81F308BF1F
:101130002033A3F10B03B3F120020CDA0C3208DDEB
:1011400002F1140CC2F10C0201FA0CF021FA02F1C6
:101150000CE002F11402D8BFC2F1200C01FA02F136
:1011600020FA0CFCDCBF41EA0C019040E41AA2BF5B
:1011700001EB0451294330BD6FEA04041F3C1CDA23
:101180000C340EDC04F11404C4F1200220FA04F043
:1011900001FA02F340EA030021FA04F345EA0301ED
:1011A00030BDC4F10C04C4F1200220FA02F001FAAF
:1011B00004F340EA0300294630BD21FA04F0294631
:1011C00030BD94F0000F83F4801306BF81F48011CA
:1011D0000134013D4EE77FEA645C18BF7FEA655C3D
:1011E00029D094EA050F08BF90EA020F05D054EA0F
:1011F000000C04BF1946104630BD91EA030F1EBF14
:101200000021002030BD5FEA545C05D14000494117
:1012100028BF41F0004130BD14F580043CBF01F50A
:10122000801130BD01F0004545F0FE4141F47001F0
:101230004FF0000030BD7FEA645C1ABF19461046CB
:101240007FEA655C1CBF0B46024650EA013406BFCC
:1012500052EA033591EA030F41F4002130BD00BF8B
:1012600090F0000F04BF0021704730B54FF4806448
:1012700004F132044FF000054FF0000150E700BFC9
:1012800090F0000F04BF0021704730B54FF4806428
:1012900004F1320410F0004548BF40424FF0000115
:1012A0003EE700BF42004FEAE2014FEA31014FEA58
:1012B00002701FBF12F07F4393F07F4F81F06051A7
:1012C000704792F0000F14BF93F07F4F704730B516
:1012D0004FF4607401F0004521F0004120E700BFA9
:1012E00050EA010208BF704730B54FF000050AE030
:1012F00050EA010208BF704730B511F0004502D531
:10130000404261EB41014FF4806404F132045FEA32
:10131000915C3FF4DCAE4FF003025FEADC0C18BFD7
:1013200003325FEADC0C18BF033202EBDC02C2F1CD
:10133000200300FA03FC20FA02F001FA03FE40EA5F
:101340000E0021FA02F11444C1E600BF70B54FF05F
:10135000FF0C4CF4E06C1CEA11541DBF1CEA135541
:1013600094EA0C0F95EA0C0F00F0DEF82C4481EAA9
:10137000030621EA4C5123EA4C5350EA013518BFC9
:1013800052EA033541F4801143F4801338D0A0FBB6
:1013900002CE4FF00005E1FB02E506F00042E0FB63
:1013A00003E54FF00006E1FB03569CF0000F18BF69
:1013B0004EF0010EA4F1FF04B6F5007F64F5407411
:1013C00004D25FEA4E0E6D4146EB060642EAC621A4
:1013D00041EA55514FEAC52040EA5E504FEACE2E11
:1013E000B4F1FD0C88BFBCF5E06F1ED8BEF1004F14
:1013F00008BF5FEA500E50F1000041EB045170BD90
:1014000006F0004646EA010140EA020081EA0301D3
:10141000B4EB5C04C2BFD4EB0C0541EA045170BDCF
:1014200041F480114FF0000E013C00F3AB8014F149
:10143000360FDEBF002001F0004170BDC4F1000492
:10144000203C35DA0C341BDC04F11404C4F1200513
:1014500000FA05F320FA04F001FA05F240EA02006E
:1014600001F0004221F0004110EBD37021FA04F6A4
:1014700042EB06015EEA430E08BF20EAD37070BD5E
:10148000C4F10C04C4F1200500FA04F320FA05F0BD
:1014900001FA04F240EA020001F0004110EBD370BF
:1014A00041F100015EEA430E08BF20EAD37070BD2F
:1014B000C4F1200500FA05F24EEA020E20FA04F308
:1014C00001FA05F243EA020321FA04F001F00041B7
:1014D00021FA04F220EA020000EBD3705EEA430E28
:1014E00008BF20EAD37070BD94F0000F0FD101F057
:1014F0000046400041EB010111F4801F08BF013C90
:10150000F7D041EA060195F0000F18BF704703F0CD
:101510000046520043EB030313F4801F08BF013D54
:10152000F7D043EA0603704794EA0C0F0CEA135510
:1015300018BF95EA0C0F0CD050EA410618BF52EACA
:101540004306D1D181EA030101F000414FF00000D0
:1015500070BD50EA410606BF1046194652EA4306DE
:1015600019D094EA0C0F02D150EA013613D195EA52
:101570000C0F05D152EA03361CBF104619460AD19A
:1015800081EA030101F0004141F0FE4141F47001A4
:101590004FF0000070BD41F0FE4141F4780170BD94
:1015A00070B54FF0FF0C4CF4E06C1CEA11541DBFF9
:1015B0001CEA135594EA0C0F95EA0C0F00F0A7F8FB
:1015C000A4EB050481EA030E52EA03354FEA013128
:1015D00000F088804FEA03334FF0805545EA13133B
:1015E00043EA12634FEA022245EA111545EA106503
:1015F0004FEA00260EF000419D4208BF964244F19A
:10160000FD0404F5407402D25B084FEA3202B61AB8
:1016100065EB03055B084FEA32024FF480104FF48C
:10162000002CB6EB020E75EB030E22BFB61A754600
:1016300040EA0C005B084FEA3202B6EB020E75EB93
:10164000030E22BFB61A754640EA5C005B084FEAFB
:101650003202B6EB020E75EB030E22BFB61A7546C8
:1016600040EA9C005B084FEA3202B6EB020E75EBD3
:10167000030E22BFB61A754640EADC0055EA060E94
:1016800018D04FEA051545EA16754FEA06164FEAD7
:10169000C30343EA52734FEAC2025FEA1C1CC0D183
:1016A00011F4801F0BD141EA00014FF000004FF010
:1016B000004CB6E711F4801F04BF01430020B4F1D1
:1016C000FD0C88BFBCF5E06F3FF6AFAEB5EB030C89
:1016D00004BFB6EB020C5FEA500C50F1000041EB86
:1016E000045170BD0EF0004E4EEA113114EB5C0453
:1016F000C2BFD4EB0C0541EA045170BD41F4801126
:101700004FF0000E013C90E645EA060E8DE60CEA2D
:10171000135594EA0C0F08BF95EA0C0F3FF43BAF4A
:1017200094EA0C0F0AD150EA01347FF434AF95EA01
:101730000C0F7FF425AF104619462CE795EA0C0FE5
:1017400006D152EA03353FF4FDAE1046194622E7B2
:1017500050EA410618BF52EA43067FF4C5AE50EA8C
:1017600041047FF40DAF52EA43057FF4EBAE12E77C
:101770004FF0FF3C06E000BF4FF0010C02E000BF5D
:101780004FF0010C4DF804CD4FEA410C7FEA6C5C40
:101790004FEA430C18BF7FEA6C5C1BD001B050EAE3
:1017A000410C0CBF52EA430C91EA030F02BF90EACE
:1017B000020F0020704710F1000F91EA030F58BF8D
:1017C000994208BF90422CBFD8176FEAE37040F0EF
:1017D000010070474FEA410C7FEA6C5C02D150EA8D
:1017E000013C07D14FEA430C7FEA6C5CD6D152EA48
:1017F000033CD3D05DF8040B704700BF844610460D
:1018000062468C461946634600E000BF01B5FFF70B
:10181000B7FF002848BF10F1000F01BD4DF808EDDB
:10182000FFF7F4FF0CBF012000205DF808FB00BFAC
:101830004DF808EDFFF7EAFF34BF012000205DF806
:1018400008FB00BF4DF808EDFFF7E0FF94BF012053
:1018500000205DF808FB00BF4DF808EDFFF7CEFF54
:1018600094BF012000205DF808FB00BF4DF808ED93
:10187000FFF7C4FF34BF012000205DF808FB00BF64
:101880004FEA410212F5001215D211D56FF47873A8
:10189000B3EB625212D94FEAC12343F0004343EA4B
:1018A000505311F0004F23FA02F018BF4042704726
:1018B0004FF00000704750EA013005D111F00040B0
:1018C00008BF6FF0004070474FF00000704700BF46
:1018D0004FEA4102B2F1E04324BFB3F5001CDCF152
:1018E000FE5C0DD901F0004C4FEAC0024CEA50708A
:1018F000B2F1004F40EB830008BF20F001007047B9
:1019000011F0804F21D113F13872BCBF01F00040BB
:10191000704741F480114FEA5252C2F11802C2F1ED
:10192000200C10FA0CF320FA02F018BF40F001006E
:101930004FEAC1234FEAD32303FA0CFC40EA0C0020
:1019400023FA02F34FEA4303CCE77FEA625307D15D
:1019500050EA01331EBF4FF0FE4040F44000704794
:1019600001F0004040F0FE4040F40000704700BF2E
:1019700080F0004002E000BF81F0004142001FBF44
:101980005FEA410392EA030F7FEA226C7FEA236C4D
:101990006AD04FEA1262D2EB1363C1BFD218414042
:1019A00048404140B8BF5B42192B88BF704710F0D8
:1019B000004F40F4000020F07F4018BF404211F07B
:1019C000004F41F4000121F07F4118BF494292EAE3
:1019D000030F3FD0A2F1010241FA03FC10EB0C000F
:1019E000C3F1200301FA03F100F0004302D549429C
:1019F00060EB4000B0F5000F13D3B0F1807F06D349
:101A000040084FEA310102F10102FE2A51D2B1F140
:101A1000004F40EBC25008BF20F0010040EA030035
:101A20007047490040EB000010F4000FA2F10102E2
:101A3000EDD1B0FA80FCACF1080CB2EB0C0200FA6C
:101A40000CF0AABF00EBC25052421843BCBFD040BA
:101A50001843704792F0000F81F4000106BF80F434
:101A600000000132013BB5E74FEA41037FEA226CF7
:101A700018BF7FEA236C21D092EA030F04D092F0C2
:101A8000000F08BF0846704790EA010F1CBF0020F6
:101A9000704712F07F4F04D1400028BF40F0004053
:101AA000704712F100723CBF00F50000704700F073
:101AB000004343F0FE4040F4000070477FEA22629A
:101AC00016BF08467FEA23630146420206BF5FEA6B
:101AD000412390EA010F40F4800070474FF000036B
:101AE00004E000BF10F0004348BF40425FEA000C32
:101AF00008BF704743F0964301464FF000001CE0DA
:101B000050EA010208BF70474FF000030AE000BF2F
:101B100050EA010208BF704711F0004302D540426D
:101B200061EB41015FEA010C02BF844601460020DF
:101B300043F0B64308BFA3F18053A3F50003BCFAFA
:101B40008CF2083AA3EBC25310DB01FA02FC6344A7
:101B500000FA02FCC2F12002BCF1004F20FA02F2AE
:101B600043EB020008BF20F00100704702F12002A1
:101B700001FA02FCC2F1200250EA4C0021FA02F202
:101B800043EB020008BF20EADC7070474FF0FF0C07
:101B90001CEAD0521EBF1CEAD15392EA0C0F93EA02
:101BA0000C0F6FD01A4480EA010C400218BF5FEAA4
:101BB00041211ED04FF0006343EA501043EA511117
:101BC000A0FB01310CF00040B1F5000F3EBF490011
:101BD00041EAD3715B0040EA010062F17F02FD2A15
:101BE0001DD8B3F1004F40EBC25008BF20F00100F8
:101BF000704790F0000F0CF0004C08BF49024CEA0F
:101C0000502040EA51207F3AC2BFD2F1FF0340EAA0
:101C1000C250704740F400004FF00003013A5DDC11
:101C200012F1190FDCBF00F000407047C2F1000252
:101C3000410021FA02F1C2F1200200FA02FC5FEA3F
:101C4000310040F1000053EA4C0308BF20EADC7089
:101C5000704792F0000F00F0004C02BF400010F4FB
:101C6000000F013AF9D040EA0C0093F0000F01F0A8
:101C7000004C02BF490011F4000F013BF9D041EACA
:101C80000C018FE70CEAD15392EA0C0F18BF93EACC
:101C90000C0F0AD030F0004C18BF31F0004CD8D1F6
:101CA00080EA010000F00040704790F0000F17BF7D
:101CB00090F0004F084691F0000F91F0004F14D0C3
:101CC00092EA0C0F01D142020FD193EA0C0F03D11B
:101CD0004B0218BF084608D180EA010000F000401E
:101CE00040F0FE4040F40000704740F0FE4040F4F9
:101CF000400070474FF0FF0C1CEAD0521EBF1CEA98
:101D0000D15392EA0C0F93EA0C0F69D0A2EB0302B5
:101D100080EA010C49024FEA402037D04FF080534F
:101D200043EA111143EA10130CF000408B4238BF14
:101D30005B0042F17D024FF4000C8B4224BF5B1A22
:101D400040EA0C00B3EB510F24BFA3EB510340EA70
:101D50005C00B3EB910F24BFA3EB910340EA9C001E
:101D6000B3EBD10F24BFA3EBD10340EADC001B018E
:101D700018BF5FEA1C1CE0D1FD2A3FF650AF8B4232
:101D800040EBC25008BF20F0010070470CF0004C3F
:101D90004CEA50207F32C2BFD2F1FF0340EAC2506A
:101DA000704740F400004FF00003013A37E792F02B
:101DB000000F00F0004C02BF400010F4000F013A89
:101DC000F9D040EA0C0093F0000F01F0004C02BF84
:101DD000490011F4000F013BF9D041EA0C0195E7ED
:101DE0000CEAD15392EA0C0F08D142027FF47DAF86
:101DF00093EA0C0F7FF470AF084676E793EA0C0F76
:101E000004D14B023FF44CAF08466EE730F0004C73
:101E100018BF31F0004CCAD130F000427FF45CAF03
:101E200031F000437FF43CAF5FE700BF4FF0FF3C71
:101E300006E000BF4FF0010C02E000BF4FF0010CC4
:101E40004DF804CD4FEA40024FEA41037FEA226C8D
:101E500018BF7FEA236C11D001B052EA530C18BFAF
:101E600090EA010F58BFB2EB030088BFC81738BF14
:101E70006FEAE17018BF40F0010070477FEA226C02
:101E800002D15FEA402C05D17FEA236CE4D15FEAFE
:101E9000412CE1D05DF8040B704700BF8446084632
:101EA0006146FFE70FB5FFF7C9FF002848BF10F1F3
:101EB000000F0FBD4DF808EDFFF7F4FF0CBF012038
:101EC00000205DF808FB00BF4DF808EDFFF7EAFFC2
:101ED00034BF012000205DF808FB00BF4DF808ED7D
:101EE000FFF7E0FF94BF012000205DF808FB00BF72
:101EF0004DF808EDFFF7D2FF94BF012000205DF8F8
:101F000008FB00BF4DF808EDFFF7C8FF34BF012004
:101F100000205DF808FB00BF42000ED2B2F1FE4F78
:101F20000BD34FF09E03B3EB126209D44FEA0023A8
:101F300043F0004323FA02F070474FF0000070476F
:101F400012F1610F01D1420202D14FF0FF30704710
:101F50004FF00000704700BF73B96AB9002908BF8D
:101F60000028BCBF00204FF00041C4BF6FF000410B
:101F70004FF0FF30FFF730B882B0EC462DE900504B
:101F800000F01CF8DDF804E002B00CBC704700BFA4
:101F9000F8B514461D4606460F4600F0D3F900FB7F
:101FA00005F5A0FB042304FB0154E318B61A67EB04
:101FB0000307069BC3E90067F8BD00BFF8B51446E8
:101FC0001D4606460F4600F00FF800FB05F5A0FB86
:101FD000042304FB0154E318B61A67EB0307069BBE
:101FE000C3E90067F8BD00BF00292DE9F04F85B0B7
:101FF000C0F2C9800026002BC0F2C080894614467A
:1020000005469B46002B4BD18A4258D9B2FA82F33F
:1020100053B1C3F1200001FA03F925FA00F812FACE
:1020200003F49D4048EA0909270C484639461FFA3F
:1020300084FBFEF795FE394682464846FEF7BEFF12
:102040004FEA15420BFB0AF342EA01494B4509D915
:1020500019EB04090AF1FF3A04D24B4584BF0AF197
:10206000FF3AA144C3EB090939464846ADB2FEF731
:1020700077FE394680464846FEF7A0FF0BFB08FB7B
:1020800045EA0145AB4507D92D1908F1FF3803D2C0
:10209000AB4588BF08F1FF3848EA0A48002703E04B
:1020A0008B4257D90027B84642463B4616B15242AA
:1020B00063EB43031946104605B0BDE8F08F22B923
:1020C00011460120FEF74CFE0446B4FA84F8B8F13C
:1020D000000F5ED1C4EB0908270C1FFA84F9012117
:1020E000029139464046FEF73BFE3946824640465D
:1020F000FEF764FF4FEA154809FB0AF348EA014B73
:102100005B4509D91BEB040B0AF1FF3A04D25B458E
:1021100084BF0AF1FF3AA344C3EB0B0B3946584680
:10212000ADB2FEF71DFE394680465846FEF746FF23
:1021300009FB08F945EA0145A94507D92D1908F118
:10214000FF3803D2A94588BF08F1FF3848EA0A489A
:10215000029FA9E7B3FA83F7002F67D18B422CBF08
:102160004FF000094FF0010982428CBF4C4649F004
:102170000104002C96D04FF0010895E7524263EB22
:102180004303F6433AE7404261EB41014FF0FF362B
:1021900031E704FA08F4C8F1200735FA07F329FA01
:1021A00007FA270C09FA08FB3946504643EA0B02A6
:1021B0000292FEF7D5FD39461FFA84F98346504650
:1021C000FEF7FCFE029809FB0BF2030C43EA014305
:1021D0009A4204D91B190BF1FF3BC0F0AD809B1A4A
:1021E000394618460193FEF7BBFD01998246084621
:1021F0003946FEF7E3FE029809FB0AF31FFA80FC5A
:102200004CEA0142934208D912190AF1FF3A04D26A
:10221000934284BF0AF1FF3A121905FA08F54AEA17
:102220000B4EC3EB0208CDF808E05AE7C7F12000D7
:1022300003FA07FAC24035FA00F342EA0A0B21FA20
:1022400000F801FA07F940464FEA1B4A43EA090140
:10225000029151461FFA8BF20392FEF781FD51461F
:1022600081464046FEF7AAFE0398029B00FB09F256
:10227000180C14FA07F340EA0144A24204D914EB03
:102280000B0409F1FF3951D3A41A5146204601939A
:10229000FEF766FD514680462046FEF78FFE039C02
:1022A000019B04FB08F2029C1FFA84FC4CEA0140EB
:1022B000824204D910EB0B0008F1FF3830D348EA12
:1022C00009481FFA83FC1B0C801A1FFA88FE4FEA8C
:1022D000184A0CFB0EF90CFB0AF203FB0E2103FB60
:1022E0000AF301EB19418A4288BF03F5803303EBFF
:1022F000114E704510D31FFA89F905FA07F709EB5B
:10230000014014BF0022012287422CBF002702F0A7
:102310000107002F3FF4C8AE08F1FF380027C3E6DD
:10232000824284BF584408F1FF38C8E7A24284BF04
:1023300009F1FF395C44A7E79A4284BF0BF1FF3BE8
:102340001B194CE72DE9F04F0C4683B0804616462A
:1023500089461F4615468A46002B4BD18A425CD9D6
:10236000B2FA82F35BB1C3F1200001FA03FA28FA52
:1023700000F216FA03F508FA03F842EA0A0A2E0CEC
:1023800050463146AFB2FEF7EBFC31464FEA1844F7
:1023900081465046FEF712FE07FB09F344EA014A64
:1023A000534509D91AEB050A09F1FF3904D25345FF
:1023B00084BF09F1FF39AA44C3EB0A0A31465046EB
:1023C0001FFA88F8FEF7CCFC314604465046FEF76B
:1023D000F5FD07FB04F748EA0148474506D9013CEB
:1023E00018EB050802D2474588BF013C44EA09447E
:1023F00000265CE08B4258D8B3FA83F6002E5BD1FE
:102400008B422CBF0022012285428CBF154642F030
:102410000105002D49D0012449E022B911460120CF
:10242000FEF79EFC0546B5FA85F6002E40F0BB800F
:10243000641B2F0C1FFA85FA012639462046FEF749
:102440008FFC39464FEA184B81462046FEF7B6FD11
:102450000AFB09F34BEA014B5B4509D91BEB050B62
:1024600009F1FF3904D25B4584BF09F1FF39AB4460
:10247000C3EB0B0B394658461FFA88F8FEF770FC81
:10248000394604465846FEF799FD0AFB04FA48EA25
:102490000148C24506D9013C18EB050802D2C245E5
:1024A00088BF013C44EA094401E000263446314635
:1024B000204603B0BDE8F08FC6F12000B34032FAE9
:1024C00000F721FA00FB1F4314FA06F228FA00F184
:1024D00058464FEA174A114300915146BBB2019347
:1024E000FEF73EFC5146B54081465846FEF766FD74
:1024F000019C009804FB09F34FEA104C4CEA014B95
:102500005B4505D91BEB070B09F1FF39C0F08F8044
:10251000C3EB0B0B51465846FEF722FC51460446CE
:102520005846FEF74BFD0198009A00FB04F31FFA92
:1025300082FC4CEA0142934206D9013CD21903D2F3
:10254000934201D9D219013C44EA0944A8B2D21AF3
:102550002D0C1FFA84FC4FEA144300FB0CF700FB20
:1025600003FE05FB0CE105FB03F501EB17418E456E
:1025700088BF05F5803505EB1145AA4210D3BFB2DF
:1025800008FA06F607EB014214BF4FF0000E4FF0B9
:10259000010E96422CBF00260EF00106002E86D0BA
:1025A000013C002683E7B540C6F1200124FA01F979
:1025B00028FA01F22F0CB4403946484622430092D3
:1025C000FEF7CEFB39461FFA85FA83464846FEF7EA
:1025D000F5FC009B1A0C0AFB0BF342EA0144A342F0
:1025E00003D964190BF1FF3B27D3E41A394620467F
:1025F000FEF7B6FB394681462046FEF7DFFC009821
:102600000AFB09F31FFA80FC4CEA0144A34208D9F3
:10261000641909F1FF3904D2A34284BF09F1FF39DB
:10262000641908FA06F8E41A49EA0B4605E75B451F
:1026300084BF09F1FF39BB446AE7A34284BF0BF1B1
:10264000FF3B6419D1E700BF00000000000000005C
:10265000010003E80000000000000003E8000000A3
:1026600000000200FA060003000000000037060028
:102670000000000000000000F40100006400000001
:102680000180080800000000006400000000000055
:1026900000000000C800000012011001020000400C
:1026A000D0169E05011B0102030100000902430030
:1026B000020100C0320904000001020201000524E9
:1026C0000010010524010001042402020524060073
:1026D00001070582030800FF09040100020A000047
:1026E00000070503024000000705810240000000CA
:1026F0000403090426035400720069006E0061009F
:102700006D00690063004D006F00740069006F0088
:102710006E002000430074006C000000320354007F
:102720004D0043004D002D003100310034003000D9
:1027300020002800760069007200740075006100B6
:102740006C00200043004F004D00290020000000D5
:10275000524F5200000106524F4C000002064D53EA
:1027600054000003024D565000000407534150002E
:10277000000507474150000006035354415000072D
:1027800003525341500008035347500000090747C4
:10279000475000000A0353544750000B035253475D
:1027A00050000C0352465300000D0353494F0000E4
:1027B0000E0747494F00000F0353414300001D0718
:1027C00053434F00001E0747434F00001F0343437E
:1027D0004F0000200341434F0000270355463000BF
:1027E000004007554631000041075546320000427F
:1027F000075546330000430755463400004407554B
:102800004635000045075546360000460755463711
:102810000000470752554E0000810553544F5000A9
:10282000800042494E00008B0000000000000000C4
:10283000020000000000000100000000010203048B
:1028400001020304060708090204060800202020EC
:102850002020202020202828282828202020202050
:102860002020202020202020202020202088101020
:10287000101010101010101010101010100404047C
:10288000040404040404041010101010101041413A
:102890004141414101010101010101010101010128
:1028A000010101010101010110101010101042423C
:1028B00042424242020202020202020202020202F8
:1028C0000202020202020202101010102000000098
:1028D00000000000000000000000000000000000F8
:1028E00000000000000000000000000000000000E8
:1028F00000000000000000000000000000000000D8
:1029000000000000000000000000000000000000C7
:1029100000000000000000000000000000000000B7
:1029200000000000000000000000000000000000A7
:102930000000000000000000000000000000000097
:102940000000000000000000000000000000000087
:102950003131343056313237004142530052454C08
:1029600000434F4F52440053544152540053544F6C
:1029700050005354415455530000000043000000E0
:082980006C6F6700000000000D
:0829880060F6FF7F0100000072
:1029900050290108000100000001020000080000A9
:1029A0000100000002000000000000000000000024
:1029B0000000000000000000000000000000000017
:1029C0000000000000000000000000000000000007
:1029D000000000000000000000C20100000008002C
:1029E000F026010804000000F4260108260000007B
:1029F0001C27010832000000B00000201A0000006F
:102A0000AC260108430000009826010812000000CF
:102A1000699B00088599000895970008A997000808
:102A2000AD9700080D9800083198000875990008C6
:102A3000659900084199000800000000400000006E
:102A40001A0354004D0043003100310034003000BF
:102A50000000000000000000000000009596000843
:102A6000F1F50008F1F50008F1F50008F1F50008AE
:102A7000F1F50008F1F50008F1F50008F1F500089E
:102A8000D59A0008F1F50008F1F50008F1F5000805
:102A9000F1F5000804010000F1F500087197000845
:102AA000F1F50008F1F50008F1F50008F1F500086E
:102AB000F1F50008F1F50008899700080100000011
:102AC0004D2801084C2801083C01002000000000AE
:102AD00000000000000000000000000000000000F6
:102AE0000000000000000000000000007C29010838
:102AF00000000000000000000000000000000000D6
:102B000000000000000000000000000000000000C5
:102B100000000000000000000000000000000000B5
:102B200000000000000000000000000000000000A5
:102B30000000000000000000000000000000000095
:102B40000000000000000000000000000000000085
:102B50000000000000000000000000000000000075
:102B60000000000000000000000000000000000065
:102B70000000000000000000000000000000000055
:102B80000000000000000000000000000000000045
:102B90000000000000000000000000000000000035
:102BA0000000000000000000000000000000000025
:102BB0000000000000000000000000000100000014
:04000005080041109E
:00000001FF
